:020000040800F2
:2000000000500020190200082102000825020008290200082D02000831020008000000004E
:200020000000000000000000000000003502000839020008000000003D02000841020008AC
:20004000450200084502000845020008450200084502000845020008450200084502000828
:20006000450200084502000845020008450200084502000845020008450200084502000808
:200080004502000845020008450200084502000845020008450200084502000845020008E8
:2000A000450200084502000845020008450200089D3400084502000845020008450200083E
:2000C000450200084502000845020008450200084502000845360008450200084502000874
:2000E000450200084502000845020008000000000000000000000000000000000000000013
:2001000000000000000000005FF808F100B583B0304B314A1360314A1360314B3149002238
:2001200001E01A6004338B42FBD32B4B1B6813B92A4B1B6803B1FEE7264B2B4A13602B4A6E
:2001400013602B4B2B4A2C4803E011681960043304328342F9D3244B1A68284B9A4204D1E5
:20016000224B1A681B689A4200D0FEE701F0E8FB01A8694601F0A8FB214B224EF61AB6100A
:2001800000241D4603E055F8243098470134A642F9DC1D4B1D4EF61AB61000241D4603E070
:2001A00055F8243098470134A642F9DC0198009904F0B0F90546164B164CE41AA4101E46DA
:2001C00003E0013C56F824309847002CF9DC284601F052FBBABADECACC000020081200208F
:2001E000CC0000200C12002000000020C800002000000020445A0008CC0000207856341207
:2002000048020008480200084802000848020008480200084802000808B5FFF777FF00BF0A
:20022000FEE700BFFEE700BFFEE700BFFEE700BFFEE700BFFEE700BFFEE700BFFEE700BF9E
:20024000FEE700BFFEE700BF10B50446C378012B03D92048752101F06FFB63780F2B03D9BA
:200260001C48762101F068FBA3780F2B03D91948772101F061FBE37803B3174BDB68DB43E4
:20028000C3F30223C3F104020F2121FA03F3617801FA02F2A1781940114309012278C9B2DB
:2002A0000E4B1A4482F800132278510902F01F02012000FA02F243F8212010BD237859099E
:2002C00003F01F03012202FA03F32031034A42F8213010BDD056000800ED00E000E100E042
:2002E00010B50446022804D9054840F2031101F023FB044B1A6802F0380214431C6010BDA9
:20030000F85600080020024010B50446102805D020B1074840F22F1101F00EFB054B1A68AB
:2003200022F010021A601A6814431C6010BD00BFF856000800200240034B044A5A6002F13D
:2003400088325A60704700BF0020024023016745024B1A6942F080021A6170470020024069
:2003600010B5044630F0350300D120B9034840F2CC5101F0E1FA024BDC6010BDF85600085A
:20038000002002400B4BDB6813F0010F0DD1094BDB6813F0040F0AD1064BDB6803F010034F
:2003A000002B0CBF042003207047012070470220704700BF0020024010B50446FFF7E2FF91
:2003C00002E0FFF7DFFF013C012801D1002CF8D1002C08BF052010BD38B5044600F1784273
:2003E000114B9A4204D9114840F2A71101F0A4FA4FF43020FFF7E0FF042813D10C4D2B69B1
:2004000043F002032B616C612B6943F040032B614FF43020FFF7D0FF2B6923F00203DB04D2
:20042000DB0C2B6138BD00BFFEFF0F00F85600080020024030B583B004460D460023019365
:2004400000F178421A4B9A4204D91A4840F2B52101F072FA4FF40050FFF7AEFF042824D1B5
:20046000154B1A6942F001021A61ABB223804FF40050FFF7A1FF042810D102340194019B4C
:200480002D0C1D804FF40050FFF796FF0A4B1A6922F00102D204D20C1A6106E0064B1A6992
:2004A00022F00102D204D20C1A6103B030BD00BFFEFF0F00F8560008002002402DE9F0418E
:2004C00005460C46494B98421BD003F58063984217D003F58063984213D003F5806398423D
:2004E0000FD003F5806398420BD003F58063984207D003F58063984203D03D48B22101F030
:200500001BFAE3788BB1042B0FD0282B0DD0482B0BD0142B09D0102B07D01C2B05D0182B1A
:2005200003D03348B32101F007FA23881BB93048B42101F001FAE37803F00F073E4613F004
:20054000100F0AD0A378013BDBB2022B03D92848BB2101F0F1F9A6783E432378FBB12F6811
:20056000002301204FF00F0C16E000FA03F22188114091420FD199000CFA01F827EA080793
:2005800006FA01F10F43E178282901D16A6102E0482908BF2A610133072BE6D92F602388CC
:2005A000FF2B21D96F68002301204FF00F0C18E003F1080200FA02F22188114091420FD111
:2005C00099000CFA01F827EA080706FA01F10F43E178282908BF6A61E178482908BF2A61C7
:2005E0000133072BE4D96F60BDE8F081000801402C57000838B504460D462A4B98421CD05A
:2006000003F58063984218D003F58063984214D003F58063984210D003F5806398420CD07E
:2006200003F58063984208D003F58063984204D01D484FF48F7101F07FF96B1E9BB2012B91
:2006400028D9042D26D0082D24D0102D22D0202D20D0402D1ED0802D1CD0B5F5807F19D057
:20066000B5F5007F16D0B5F5806F13D0B5F5006F10D0B5F5805F0DD0B5F5005F0AD0B5F503
:20068000804F07D0B5F5004F04D0074840F21F1101F052F9A36803EA0500003018BF0120D5
:2006A00038BD00BF000801402C57000838B504460D46144B98421CD003F58063984218D066
:2006C00003F58063984214D003F58063984210D003F5806398420CD003F58063984208D0CE
:2006E00003F58063984204D0074840F2691101F023F925B904484FF4B57101F01DF9256149
:2007000038BD00BF000801402C57000838B504460D46144B98421CD003F58063984218D005
:2007200003F58063984214D003F58063984210D003F5806398420CD003F58063984208D06D
:2007400003F58063984204D0074840F2791101F0F3F825B904484FF4BD7101F0EDF86561F2
:2007600038BD00BF000801402C5700080D4B1A6842F001021A6059680B4A0A405A601A68CC
:2007800022F0847222F480321A601A6822F480221A605A6822F4FE025A604FF41F029A606B
:2007A000704700BF001002400000FFF810B5044650B1B0F5803F07D0B0F5802F04D01048AF
:2007C00040F2111101F0B8F80E4B1A6822F480321A601A6822F480221A60B4F5803F03D018
:2007E000B4F5802F06D010BD064B1A6842F480321A6010BD034B1A6842F4A0221A6010BDED
:20080000605700080010024038B50C46054650B1B0F5803F07D0B0F5403F04D01E4840F271
:200820007F1101F089F874B3B4F5802F2BD0B4F5002F28D0B4F5402F25D0B4F5801F22D025
:20084000B4F5A01F1FD0B4F5C01F1CD0B4F5E01F19D0B4F5001F16D0B4F5101F13D0B4F52A
:20086000201F10D0B4F5301F0DD0B4F5401F0AD0B4F5501F07D0B4F5601F04D006484FF426
:20088000C07101F059F8054B5A6822F47C122C4314435C6038BD00BF6057000800100240E8
:2008A00010B50446012804D903484FF4CA7101F043F8024B1C6010BD6057000860004242F5
:2008C00010B50446022804D905484FF40E7101F033F8044B5A6822F0030214435C6010BDCF
:2008E0006057000800100240024B586800F00C00704700BF0010024010B50446A0B180280E
:2009000012D0902810D0A0280ED0B0280CD0C0280AD0D02808D0E02806D0F02804D0064859
:200920004FF4197101F008F8044B5A6822F0F00214435C6010BD00BF605700080010024034
:2009400010B5044680B1B0F5806F0DD0B0F5A06F0AD0B0F5C06F07D0B0F5E06F04D0064897
:2009600040F27E2100F0E8FF044B5A6822F4E06214435C6010BD00BF6057000800100240B6
:2009800010B5044680B1B0F5806F0DD0B0F5A06F0AD0B0F5C06F07D0B0F5E06F04D0064857
:2009A0004FF4267100F0C8FF044B5A6822F4605242EAC4045C6010BD60570008001002403F
:2009C00010B4284B5B6803F00C03042B05D0082B06D0F3B9244B03601DE0244B03601AE0C7
:2009E000204B5A685B68C2F38342023213F4803F04D11F4B03FB02F202600CE0194B5B68ED
:200A000013F4003F14BF1B4B184B03FB02F2026001E0154B0360134B5A68C2F303121649B3
:200A20008A5CD2B2046824FA02F242605C68C4F302240C5DE4B222FA04F484605C68C4F319
:200A4000C224095DC9B2CA40C2605B68C3F381330A49CB5CDBB2B2FBF3F202615DF8044BD6
:200A6000704700BF0010024000127A00001BB70000093D00808D5B00080000200400002056
:200A800038B504460D460E4B034003B920B90D4840F24A4100F050FF012D04D9094840F2BC
:200AA0004B4100F049FF25B1074B9A6914439C6138BD054B9A6922EA04049C6138BD00BFE6
:200AC0000200C0FF605700080010024038B504460D460E4B184200D120B90D4840F269412C
:200AE00000F02AFF012D04D9094840F26A4100F023FF25B1074BDA691443DC6138BD054B4E
:200B0000DA6922EA0404DC6138BD00BF00360181605700080010024010B50446212818D084
:200B2000312816D0392814D0412812D0612810D07A280ED07B280CD07C280AD07D2808D083
:200B40007E2806D07F2804D00A4840F2345100F0F3FE6309012B02D1074B186804E0022B66
:200B6000054B0CBF186A586A04F01F04E04000F0010010BD605700080010024010B582B019
:200B80000023019331242046FFF7C6FF019B01330193019BB3F5A06F01D00028F3D0312064
:200BA000FFF7BAFF003018BF012002B010BD00BF2DE9F84305460C46464B98420BD0A3F554
:200BC0007843984207D003F58063984203D04248A32100F0B1FE238863B1B3F5806F09D005
:200BE000B3F5004F06D0B3F5404F03D03A48A62100F0A2FE6388B3F5827F04D01BB1364893
:200C0000A72100F099FEA388B3F5006F04D01BB13148A82100F090FEE3882BB1022B03D09C
:200C20002D48A92100F088FE2389012B03D92A48AA2100F081FE6389B3F5007F04D01BB1EC
:200C40002548AB2100F078FEA3898BB1082B0FD0102B0DD0182B0BD0202B09D0282B07D0F7
:200C6000302B05D0382B03D01B48AC2100F064FEE3892BB1802B03D01748AD2100F05CFE4F
:200C8000238A1BB91448AE2100F056FE2A8802F44152B4F800906388B4F80480B4F806C060
:200CA00027896689A089E18949EA030348EA03034CEA03033B43334303430B4313432B80CC
:200CC000AB8B23F400631B041B0CAB83238A2B82BDE8F883003001409057000838B50446DF
:200CE0000D46124B98420CD0A3F57843984208D003F58063984204D00D4840F2B71100F0C1
:200D00001BFE012D04D90A484FF4DC7100F014FE2DB123889BB243F04003238038BD23883C
:200D200023F040031B041B0C238038BD003001409057000838B504460D46094B98420CD08B
:200D4000A3F57843984208D003F58063984204D0044840F23A2100F0EFFDA58138BD00BF76
:200D6000003001409057000810B50446094B98420CD0A3F57843984208D003F58063984240
:200D800004D0054840F24A2100F0D6FDA08980B210BD00BF003001409057000838B5054653
:200DA0000C46164B98420CD0A3F57843984208D003F58063984204D0114840F2163100F07A
:200DC000BBFD802C12D0402C10D0202C0ED0102C0CD0082C0AD0042C08D0022C06D0012CF8
:200DE00004D0074840F2173100F0A6FD2B8904EA0300003018BF012038BD00BF00300140D1
:200E00009057000838B504460D46524B984242D0B0F1804F3FD0A3F5943398423BD003F515
:200E20008063984237D003F58063984233D003F5806398422FD003F5806398422BD003F5DA
:200E40009033984227D003F5C053984223D003F5806398421FD003F5806398421BD0A3F54A
:200E60009E33984217D003F58063984213D003F5806398420FD003F5903398420BD003F54C
:200E80008063984207D003F58063984203D03248E72100F051FD6B885BB1102B09D0202B18
:200EA00007D0402B05D0602B03D02B48E82100F043FDEB884BB1B3F5807F06D0B3F5007FFE
:200EC00003D02548E92100F037FD23889BB2214A944212D002F5006294420ED0B4F1804F08
:200EE0000BD0A2F59832944207D002F58062944203D002F58062944203D123F070036A888C
:200F00001343164A944208D002F58062944204D023F440739BB2EA8813432380AB88A3850D
:200F20002B8823850B4B9C420FD003F500639C420BD003F540639C4207D003F580639C4226
:200F400003D003F580639C4201D12B7A23860123A38238BD002C0140C057000800100040CB
:200F600038B504460D462E4B984243D0B0F1804F40D0A3F5943398423CD003F58063984207
:200F800038D003F58063984234D003F58063984230D003F5806398422CD003F59033984295
:200FA00028D003F5C053984224D003F58063984220D003F5806398421CD0A3F59E339842D7
:200FC00018D003F58063984214D003F58063984210D003F5903398420CD003F580639842D5
:200FE00008D003F58063984204D00E4840F2293100F0A2FC012D04D90A4840F22A3100F046
:201000009BFC2DB123889BB243F00103238038BD238823F001031B041B0C238038BD00BF35
:20102000002C0140C057000870B504460D461646314B984243D0B0F1804F40D0A3F59433BE
:2010400098423CD003F58063984238D003F58063984234D003F58063984230D003F58063A4
:2010600098422CD003F59033984228D003F5C053984224D003F58063984220D003F58063B4
:2010800098421CD0A3F59E33984218D003F58063984214D003F58063984210D003F5903376
:2010A00098420CD003F58063984208D003F58063984204D0114840F26B3100F03DFC15F40B
:2010C0007F4F00D125B90D484FF45B7100F034FC012E04D9094840F26D3100F02DFC26B1F2
:2010E000A3899BB21D43A58170BDA389ED43ADB21D40A58170BD00BF002C0140C05700080E
:2011000070B504460E461546284B984243D0B0F1804F40D0A3F5943398423CD003F58063B1
:20112000984238D003F58063984234D003F58063984230D003F5806398422CD003F59033F3
:20114000984228D003F5C053984224D003F58063984220D003F5806398421CD0A3F59E3335
:20116000984218D003F58063984214D003F58063984210D003F5903398420CD003F5806333
:20118000984208D003F58063984204D0084840F29B4100F0D1FB012D04D9054840F29C4193
:2011A00000F0CAFB2685A58270BD00BF002C0140C057000838B504460D46334B984243D03B
:2011C000B0F1804F40D0A3F5943398423CD003F58063984238D003F58063984234D003F5DC
:2011E0008063984230D003F5806398422CD003F59033984228D003F5C053984224D003F523
:201200008063984220D003F5806398421CD0A3F59E33984218D003F58063984214D003F5C4
:201220008063984210D003F5903398420CD003F58063984208D003F58063984204D013482F
:2012400040F6582100F078FB6B1E9BB2012B10D9042D0ED0082D0CD0102D0AD0202D08D035
:20126000402D06D0802D04D0084840F6592100F063FB238AA08928401D4203D0003018BFE5
:20128000012038BD002038BD002C0140C057000838B504460D462A4B984243D0B0F1804F3B
:2012A00040D0A3F5943398423CD003F58063984238D003F58063984234D003F580639842AE
:2012C00030D003F5806398422CD003F59033984228D003F5C053984224D003F58063984242
:2012E00020D003F5806398421CD0A3F59E33984218D003F58063984214D003F580639842E4
:2013000010D003F5903398420CD003F58063984208D003F58063984204D00A4840F682213B
:2013200000F00AFB15F47F4F00D125B9054840F6832100F001FBED43ADB2258238BD00BF35
:20134000002C0140C057000830B587B004460D46644B984213D0A3F5744398420FD003F5DC
:20136000806398420BD003F58063984207D003F58063984203D05C48B82100F0DDFA2B68EA
:20138000013B5A4A934203D95748B92100F0D4FAAB8833B1B3F5805F03D05348BA2100F0AE
:2013A000CBFAEB8863B1B3F5805F09D0B3F5005F06D0B3F5405F03D04B48BB2100F0BCFA75
:2013C0002B894BB1B3F5806F06D0B3F5C06F03D04548BC2100F0B0FA6B8923F00C0292B2E9
:2013E00002B91BB94048BD2100F0A6FAAB8963B1B3F5807F09D0B3F5007F06D0B3F5407F3C
:2014000003D03948BE2100F097FAAB8973B1354B9C420BD0A3F574439C4207D003F58063A8
:201420009C4203D03048C22100F086FA238A23F440531B041B0CEA8813432382A28992B2B7
:2014400022F4B05222F00C02A8882B89698903430B431343A381A38A23F440731B041B0C33
:20146000AA891343A38201A8FFF7AAFA1D4B9C420CBF049A039AA3891BB2002B08DA02EB3C
:20148000820202EB82022B685B00B2FBF3F207E002EB820202EB820229688900B2FBF1F264
:2014A000134BA3FB02135B091801642103FB1123A18909B2002908DADB0032330C4DA5FBBE
:2014C0000323C3F34213034307E01B013233084DA5FB0313C3F3431303439BB2238107B028
:2014E00030BD00BF00380140F05700081FAA44001F85EB5170B505460C46234B98420CD0A5
:20150000A3F57443984208D003F58063984204D01E484FF4997100F00FFA23883BB1B3F556
:20152000006F04D0194840F2331100F005FA63883BB1B3F5806F04D014484FF49A7100F0C6
:20154000FBF9A3883BB1B3F5007F04D00F4840F2351100F0F1F9E3883BB1B3F5807F04D00A
:201560000A484FF49B7100F0E7F92B8A23F470631B041B0C26886288A088E1883243024332
:201580000A4313432B8270BD00380140F057000838B504460D46164B984214D0A3F574430E
:2015A000984210D003F5806398420CD003F58063984208D003F58063984204D00D484FF432
:2015C000B17100F0B9F9012D04D90A4840F2631100F0B2F92DB1A3899BB243F40053A381A4
:2015E00038BDA38923F400531B041B0CA38138BD00380140F057000870B505460C4616461B
:20160000364B984214D0A3F57443984210D003F5806398420CD003F58063984208D003F56C
:201620008063984204D02E4840F2891100F084F9282C1ED040F227739C421AD040F22663D9
:201640009C4216D040F225539C4212D040F224439C420ED040F646039C420AD040F66A131D
:201660009C4206D0602C04D01D484FF4C57100F063F9012E04D91A4840F28B1100F05CF9AB
:2016800040F66A139C420FD1144B9D420CD0A3F574439D4208D003F580639D4204D01048D3
:2016A00040F28F1100F048F9C4F3421304F01F04012202FA04F4934201D10C3503E0022BF5
:2016C0000CBF103514351EB12B681C432C6070BD2B6823EA04042C6070BD00BF003801409E
:2016E000F057000838B504460D46124B984214D0A3F57443984210D003F5806398420CD05C
:2017000003F58063984208D003F58063984204D0094840F25F2100F00FF9B5F5007F04D3B8
:2017200005484FF4187100F007F9C5F30805A58038BD00BF00380140F057000810B504462B
:201740000D4B984214D0A3F57443984210D003F5806398420CD003F58063984208D003F554
:201760008063984204D005484FF41C7100F0E4F8A088C0F3080010BD00380140F057000877
:2017800038B505460C463A4B984214D0A3F57443984210D003F5806398420CD003F5806307
:2017A000984208D003F58063984204D0314840F2D93100F0C1F8282C25D040F227739C429D
:2017C00021D040F226639C421DD040F225539C4219D040F224439C4215D040F646039C4268
:2017E00011D040F66A139C420DD0B4F5587F0AD0B4F5187F07D0B4F5B07F04D01D4840F2E6
:20180000DA3100F099F840F66A139C420FD1184B9D420CD0A3F574439D4208D003F58063CC
:201820009D4204D0134840F2DE3100F085F8C4F3421304F01F0201219140012B03D1AA89A5
:2018400092B20A4005E0022B0CBF2A8AAA8A92B20A40240A012000FA04F4288880B2204024
:201860001AB1003018BF012038BD002038BD00BF00380140F0570008FEE700BF08B5012062
:20188000FFF7FAFF08B50D4B1B6813B90C4A0B4B1A600A4B1B68033020F003001844094A02
:2018A000904206D902F074FE0C2303604FF0FF3008BD024A1060184608BD00BFD0000020C0
:2018C0000C120020004C002001230360014B0B60704700BF1800002008B502F059FE5823F1
:2018E00003604FF0FF3008BD08B502F051FE582303604FF0FF3008BD08B502F049FE5823D2
:201900000360002008BD00BF08B502F041FE582303604FF0FF3008BD08B502F039FE582360
:2019200003604FF0FF3008BD08B502F031FE582303604FF0FF3008BD08B5FFF79FFF00BF12
:2019400008B500F067F808BD82B000230193009303F1804303F504331A6842F480321A6070
:201960001A46136803F400330093019B01330193009B1BB9019BB3F5A06FF2D1214B1B68F7
:2019800013F4003F14BF012300230093009B012B36D11D4B1A6842F010021A601A6822F04A
:2019A00003021A601A6842F002021A60A3F580535A685A605A685A605A6842F480625A607F
:2019C0005A6822F47C125A605A6842F4E8125A601A6842F080721A601A46136813F0007FBE
:2019E000FBD0084B5A6822F003025A605A6842F002025A601A46536803F00C03082BFAD169
:201A000002B07047001002400020024008B5FFF79BFF08BD08B5104B1A6842F001021A604E
:201A200059680E4A0A405A601A6822F0847222F480321A601A6822F480221A605A6822F431
:201A4000FE025A604FF41F029A60FFF7DFFF4FF00062034B9A6008BD001002400000FFF8A3
:201A600000ED00E0030A43EA002080B2704700BFC0F30722120442EA0062030A03F47F4351
:201A8000134343EA1060704708B5FFF7EBFF08BD08B5FFF7EDFF08BD08B5FFF7F5FF08BD6A
:201AA00008B5FFF7E5FF08BD00230A4A13700A4A13600A4A13800A4A13800A4A13600A4A20
:201AC00013800A4A13600A4A13600A4A13600A4A13707047DC000020D8000020FC00002080
:201AE000FE00002000010020F400002008010020F800002004010020F6000020054B1B6844
:201B000033B10023034A1360034A1360034A1360704700BF08010020F800002004010020A2
:201B2000054B1B683BB90122034B1A600023034A1360034A1360704708010020F800002058
:201B40000401002030B583B0054602214CF23872012300F0A7FBC4B2AC420CD10A25204666
:201B600029460DF1070200F0C5FD9DF80730222BF5D1204601E04FF0FF3003B030BD00BF4A
:201B800070B584B006460D46144603931846FFF77FFF04AB43F8040DBDF820200092F0B267
:201BA0002946A2B200F00AFCA0420CBF20464FF0FF3004B070BD00BF10B584B004460420E4
:201BC000FFF762FFADF80C002046FFF75DFFADF80E00074B1B68074A128807490868009280
:201BE00003A90422FFF7CCFFFFF79AFF04B010BDD8000020FC0000202000002008B50B4BDB
:201C00001B68012B02D0022B09D008BD0522074B1A60FFF773FF0020FFF7CEFF08BD04224F
:201C2000024B1A60FFF76AFF08BD00BF0001002008B503460A460248194602F0BEFC08BD69
:201C4000DC0000202DE9F047ADF5BF6D81460C46174698460120FFF717FFADF80C000DF13D
:201C60000E00494602F0DCFC484602F0E1FC01300DF10E0505442846214602F0D1FC20461B
:201C800002F0D6FC01300544002418E007EBC40A57F834602846314602F0C2FC304602F04A
:201CA000C7FC01300544DAF804602846314602F0B7FC304602F0BCFC013005440134A04573
:201CC000E4D803AA0C4B1B680C490868452100911146AA1AFFF754FF0122094B1A60484622
:201CE00002F0A6FC411C4846FFF7A2FFFFF718FF0DF5BF6DBDE8F087D8000020200000203F
:201D000000010020F0B585B00F4616461D46C4B220460A210DF10F0200F0ECFC01281ED1AE
:201D20009DF80F30222B1DD12046092103AA00F0E1FC012819D1BDF80C30CBB10A9B0093D2
:201D400020463946B2B22B4600F0DCFBADF80C002868FFF7A5FE2860BDF80C000AE04FF0B6
:201D6000FF3007E04FF0FF3004E04FF0FF3001E04FF0FF3005B0F0BD10B504460088FFF74F
:201D80008BFE20806088FFF787FE6080FFF78CFE0122014B1A7010BDF600002038B5044644
:201DA0000D460088FFF778FE20806088FFF774FE82B26280194B1B68032B14D0052B01D0DC
:201DC000012B29D1012A0AD10321144B1960144B1A80201D291F01F073F8FFF78FFE608896
:201DE000FFF7EAFE38BD0E4B1B8801339A4207D10B4B1A80201D291F01F062F8FFF77EFEFA
:201E00006088FFF7D9FE043DB5F5007F04D2FFF74BFE0222034B1A7038BD00BF00010020BD
:201E2000F4000020F6000020F8B505460E461F46124C2468A2421FD10088FFF72DFE104B05
:201E40001B68022B01D0012B01D10E4B1F8080B205280DD0062806D003280DD128463146DD
:201E6000FFF79CFFF8BD28463146FFF7C7FEF8BD28463146FFF780FFF8BD00BFD800002001
:201E800000010020FC00002038B505460C46FFF70BFE2846FFF756FE024B1860024B1C6036
:201EA00038BD00BF20000020F000002010B584B01E4B1B681BB31E4B1B68042B1FD91D4BF0
:201EC0001B68032B09D0052B07D0012B09D11A481A491B4AFFF7B6FE03E01A4B1888FFF7B9
:201EE0006BFE0022124B1A60174A136801331360042B04D9FFF7D8FD0122144B1A70144BBB
:201F00001868144C21680DF10E03009340F2EA5202ABFFF7F7FE81B22068029ABDF80E3066
:201F2000FFF782FF094B187804B010BD08010020F800002000010020DC00002024580008E3
:201F400024000020F400002004010020F600002020000020F000002008B5064B18600022F6
:201F6000054B1A7008460549054A0123FFF76AFE08BD00BFD8000020F60000202458000804
:201F800024000020034B1B681BB1034B1A6801321A60704708010020F800002038B50546B3
:201FA0000C4CA368984723699847E369C5F307409847E369C5F307209847E369E8B298477B
:201FC000A3699847054663699847E3689847284638BD00BF30000020F8B505460E460D4CDF
:201FE000A36898472369984745F00407E369C5F307409847E369C5F307209847E369F8B222
:202000009847E3693046984763699847E3689847F8BD00BF30000020F8B506460F461546FE
:202020000F4CA368984723699847E369C6F307409847E369C6F307209847E369F0B29847ED
:202040000024074E04E0B369984738550134A4B2AC42F8D3024C63699847E3689847F8BD7F
:20206000300000202DE9F04106460F461546124CA36898472369984746F00408E369C6F3D3
:2020800007409847E369C6F307209847E3695FFA88F098470024084E04E0385DF3699847E5
:2020A0000134A4B2AC42F8D3034C63699847E3689847BDE8F08100BF30000020F8B50025C1
:2020C000400100F1080606F5005706F504563846FFF764FF000284B23046FFF75FFF2044DC
:2020E00084B24CB13846FFF759FF000285B23046FFF754FF284485B2A542E8D12846F8BD83
:20210000F8B50025400100F1080606F5185706F51C563846FFF742FF000284B23046FFF77D
:202120003DFF204484B24CB13846FFF737FF000285B23046FFF732FF284485B2A542E8D109
:202140002846F8BD2DE9F8430D46144632B34FEA800909F10106F60006F510573846FFF7EA
:202160001DFF804606F514563046FFF717FF00EB08201FFA80F809F10200C00000EB082023
:2021800029462246FFF76EFF4444A4B23846210AFFF722FF3046E1B2FFF71EFFBDE8F8832B
:2021A0002DE9F8430D46144632B34FEA800909F10106F60006F520573846FFF7EFFE8046EA
:2021C00006F524563046FFF7E9FE00EB08201FFA80F809F10300C00000EB082029462246EC
:2021E000FFF71AFF4444A4B23846210AFFF7F4FE3046E1B2FFF7F0FEBDE8F883F8B50F4652
:20220000400100F1080505F520563046FFF7C6FE044605F524552846FFF7C0FE00EB0420F1
:20222000C419A4B23046210AFFF7D6FE2846E1B2FFF7D2FEF8BD00BF70B50546082827D826
:202240004601083606F5807420461021FFF7C4FE2046FFF7A3FE0028FAD106F500701F2120
:20226000FFF7BAFE0122AA400B4B198821EA02021A800023094A22F81530094A535506F538
:2022800040742046FFF78AFE0028FAD1012000E0FF2040B270BD00BF0E010020180100204D
:2022A000100100202DE9F04105460F4614461E4608286BD800296BD0022901D9042967D107
:2022C00016F0060F66D1A6B1012F02D0022F04D00FE016F0210F0CD15EE016F0200F02D007
:2022E00016F0800F5AD016F0100F02D016F0800F56D02846FFF7A0FF4FEA451808F10808CB
:2023000026F00F0140463943FFF766FE64B9264A1488631C9BB213804FF6F072934203D163
:202320004FF44042204B1A8008F58060210AFFF753FE08F5A060E1B2FFF74EFE08F58074C1
:2023400020460121FFF748FE2046FFF727FE0028FAD106F00106AE40144B1A8816431E8062
:202360000122AA40124B198821EA02021A800023104A22F81530104A535508F540742046B4
:20238000FFF70CFE0028FAD0E8B20AE0FF2008E0FB2006E0FA2004E0FA2002E0FA2000E0CB
:2023A000FA2040B2BDE8F0812C0000200C0100200E01002018010020100100202DE9F84F8C
:2023C00006468B4691461D46BDF82840082878D880464FEA401A0AF1080A5046FFF7DEFD3C
:2023E00000F00F00022801D004286ED1B9F1000F6FD02B68002B70D0002C72D00AF540775E
:202400003846FFF7CBFD422801D022286DD10AF5406029460422FFF725FE0AF58050210A76
:20242000FFF7DAFD0AF58850E1B2FFF7D5FD0AF5F850FFF7B3FD850205F47C454D4528BFF6
:202440004D46DFF8BC903046FFF738FE04463846FFF7A4FD00284CD0B9F8003043FA08F368
:2024600013F0010F01D0AC4247D3AC42EBD3304659462A46FFF766FE0AF58074204620214B
:20248000FFF7AAFD2046FFF789FD0028FAD10AF5007A5046FFF782FD10F0100F06D05046BB
:2024A0001021FFF799FD2846BDE8F88F10F0080FEFD050460821FFF78FFD6FF00C00BDE89E
:2024C000F88F4FF0FF30BDE8F88F6FF00400BDE8F88F6FF00D00BDE8F88F6FF00B00BDE8A5
:2024E000F88F6FF00A00BDE8F88F6FF00600BDE8F88F6FF00300BDE8F88F0020BDE8F88F55
:202500000C0100202DE9F04F85B00546009193460193082800F2D88006464FEA401909F169
:2025200008094846FFF73AFD824600F00F03022B02D0042B40F0CB80BBF1000F00F0CA8067
:20254000694B33F81530CBB909F54077DFF8A0812846FFF7D5FD04463846FFF71FFD0028EE
:2025600000F0BB80B8F80030334113F0010F02D0002C00F0B580002CEAD000E0002400229A
:202580005A4B5A550AF0070ABAF1020F03D0BAF1040F41D077E0544B33F8153083BB28466C
:2025A00002A90822FFF7FCFD09F5807420464021FFF712FD2046FFF7F1FC0028FAD19DF8C8
:2025C0000830019A13709DF8093053709DF80A3093709DF80B30D3709DF80C209DF80D309C
:2025E00003EB02220E9B1A809DF80E209DF80F3003EB02223C4B23F8152080223B4B5A552F
:20260000394B33F815405C4528BF5C46284600992246FFF7C5FD3DE0334B33F8153033BB6C
:20262000284602A90222FFF7BBFD09F5807420464021FFF7D1FC2046FFF7B0FC0028FAD138
:202640009DF808209DF8093003EB02239BB2264A22F8153040F2EA52934205D92846FFF73B
:20266000EBFD6FF47A703CE08022204B5A551E4B33F815405C4528BF5C46284600992246CB
:20268000FFF78EFD06E028462146FFF7B7FD164B23F8154009F5807948464021FFF79CFC0F
:2026A0004846FFF77BFC0028FAD10F4A32F815301B1B9BB222F8153023B10C4B5A5D42F06E
:2026C00001025A5520460CE04FF0FF3009E06FF0040006E06FF00D0003E06FF0030000E0C5
:2026E000002005B0BDE8F08F18010020100100200C01002070B504461546082800F2888056
:202700000C2900F28780DFE801F0071019222D36854656595D65770040010830FFF73EFCC2
:2027200020F00F002870012079E0400100F5B0500830FFF733FC2870012070E0400100F596
:20274000A8500830FFF72AFC2870012067E04601083606F59050FFF721FC06F59850FFF7E1
:202760001DFC2870600100F6084029460422FFF753FC012053E04401083404F58050FFF79B
:202780000DFC064604F58850FFF708FC00EB06202880012043E0440108342046FFF7FEFB46
:2027A00000F00F00012837D104F53C50FFF7F6FB2880012033E0FFF781FC28802046FFF72A
:2027C0009FFC2880600100F54270FFF7E7FB2870012024E040010830FFF7E0FB012805D1D0
:2027E0002046FFF78DFC2880012018E00D4B33F814302B80012012E040010830FFF7CEFB76
:2028000000F00F00012809D1074B1B5D2B7006E0FF2004E0FE2002E0FB2000E0FB2040B260
:2028200070BD00BF1801002010010020704700BF704700BF704700BF704700BF007870473B
:202840000170704700207047704700BF00B129B9044B054A1A61054A5A617047014B1861D1
:2028600059617047300000203528000839280008094A138803F400739BB2002BF9D000B17F
:2028800029B9054B054A9A61054ADA617047024B9861D961704700BF3000002045280008C0
:2028A0004928000800B587B04FF4106001A90622FFF7B2FB4FF4807005A90422FFF7ACFBE7
:2028C0004FF4A06004A90422FFF7A6FB4FF4706003A90422FFF7A0FB00208021FFF77CFBA7
:2028E0000020FFF75BFB4FF4106001A90622FFF7B9FB4FF4807005A90422FFF7B3FB4FF44F
:20290000A06004A90422FFF7ADFB4FF4706003A90422FFF7A7FB07B05DF804FB70B506464D
:202920000D46FFF7BFFF3EB91DE059B2715C0A44D2B20133DBB201E00022134659B207299A
:20294000F3DD52B2102A31DC002409E063B2580100F5F8500830F15CFFF73EFB0134E4B225
:2029600063B2072BF2DD00201DB306E059B2695C0A44D2B20133DBB201E00022134659B2A1
:202980000729F3DD52B2102A12DC002409E063B2580100F5F0500830E95CFFF71DFB01349B
:2029A000E4B263B2072BF2DD002002E0FF2000E0FF2040B270BD00BF10B50146040A4FF410
:2029C000A85001F0F001FFF707FB4FF4B8502146FFF702FB10BD00BF10B54FF4A850FFF7FE
:2029E000DDFA00F0F0044FF4B850FFF7D7FA000280B20444A0B210BD10B50146040A4FF412
:202A0000B050C9B2FFF7E8FA4FF4C0502146FFF7E3FA10BD10B54FF4B050FFF7BFFA044608
:202A20004FF4C050FFF7BAFA04EB002080B210BD08B54FF43850FFF7B1FA00F0010008BDAC
:202A400008B54FF43850FFF7A9FA00F03000003018BF012008BD00BF08B54FF43850FFF70B
:202A60009DFA00F07F014FF43850FFF7B5FA4FF43850FFF793FA60F07F014FF43850C9B27B
:202A8000FFF7AAFA08BD00BF08B50378012B14BF002140214378012B03D141F03801C9B2BF
:202AA0000FE0C378012B07D18378012B0CBF41F0180141F0080104E08378012B08BF41F06F
:202AC00010014FF43850FFF787FAFFF7C5FF08BD10B504464FF43850FFF760FAC0F38013B4
:202AE000237000F03803202B01D0382B02D10122627001E000226270182B03D0202B01D0CA
:202B0000102B02D10122A27001E00022A270182B03D0202B01D0082B02D10123E37010BDE1
:202B20000023E37010BD00BF10B504464FF43850FFF734FA10F0400F1CD000F0C701012C75
:202B40000CBF41F0300141F038014FF43850FFF743FAFFF781FF4FF43850FFF71FFA012C63
:202B60000CBF00F0300000F03800002814BF0020FF2000E0FF2040B210BD00BF30B583B073
:202B80000C460023009301930F2809D8DFE800F00A0E1D1822272C394755595E7763676FCC
:202BA000FF2071E0FFF77EFE00206DE019B1009101F10804019400980199FFF7AFFE63E0C0
:202BC0000888FFF7F9FE00205EE0FFF705FF2080002059E00888FFF70FFF002054E0FFF749
:202BE00019FF208000204FE009884FF49850090AFFF7F2F94FF4A0502178FFF7EDF9002056
:202C000042E04FF49850FFF7C9F905464FF4A050FFF7C4F900EB05202080002034E01C4B33
:202C20009A780A70DA784A701A798A705A79CA709B790B710020487126E0FFF70DFF0020D1
:202C400022E00846FFF720FF00201DE00846FFF73FFF002018E00878FFF766FF14E0FFF793
:202C6000EFFEC0B2FF280CD0207000200CE0FFF7DFFEC0B2FF2806D02070002004E0002060
:202C800002E0FF2000E0FF2040B203B030BD00BF3000002010B504464FF410602146062242
:202CA000FFF7E0F94FF4807004F10E010422FFF7D9F94FF4A06004F10A010422FFF7D2F9F6
:202CC0004FF47060A11D0422FFF7CCF9A27C064B1A70E27C5A70227D9A70627DDA70A27D30
:202CE000024B1A7010BD00BF2C0100202801002010B504464FF4106021460622FFF78CF90F
:202D00004FF4807004F10E010422FFF785F94FF4A06004F10A010422FFF77EF94FF47060F9
:202D2000A11D0422FFF778F9064B1A78A2745A78E2749A782275DB786375034B1B78A3755A
:202D400010BD00BF2C0100202801002010B5044630F03A030AD10020FFF720F940EA0401AC
:202D60000020C9B2FFF738F9002000E0FF2040B210BD00BF08B50020FFF710F908BD00BF94
:202D800010B504464FF4D8502178FFF725F961884FF4C850090AFFF71FF94FF4D050A1782B
:202DA000FFF71AF910BD00BF38B504464FF4D850FFF7F4F820704FF4C850FFF7EFF80546E7
:202DC0004FF4D050FFF7EAF800EB0520608038BD10B50C46052821D8DFE800F003080D11B6
:202DE000161B0846FFF756FF002018E00846FFF77FFF002013E00878FFF7A8FF0FE0FFF71A
:202E0000B9FF207000200AE00846FFF7B9FF002005E00846FFF7C8FF002000E0FF2040B243
:202E200010BD00BF10B5044672B6FDF785FA3520FDF796FA2046FDF7CFFA042802D0034817
:202E400000F098FCFDF784FA62B610BD385800082DE9F04105460F46904672B6960812F07A
:202E6000030F18BF0136FDF767FA3520FDF778FA00240FE0284657F82410FDF7DBFA042829
:202E800006D0084800F076FC4FF0FF30BDE8F08104350134B442EDDBFDF75AFA62B6404614
:202EA000BDE8F0815058000810B4002302E0C45CCC5401339342FAD318465DF8044B7047B4
:202EC0002DE9F04180460F46012A0DD107E068682E8904FB0600FFF7A5FF013401E0002440
:202EE000154DEB89A342F2DC144B1A683A441A60B7F5007F15D208EB0700FF21C7F5007216
:202F000001F064FB0E4C206841464FF40072FFF79FFF094B5B6823600022084B1A60BDE881
:202F2000F081074C206841463A46FFF791FF23681F442760BDE8F081CC09002030010020E7
:202F40005000002008B51A4B1B88FF2B17D9194800F010FC184B4FF000621A6002F5C0424E
:202F60005A604FF400621A8140225A810C221A7303225A733122DA81104A1A6108BD1048CD
:202F800000F0F8FB0C4B4FF000621A6002F5C0425A604FF480621A8180225A8118221A7325
:202FA00003225A736522DA81064A1A6108BD00BFE0F7FF1F6C580008CC09002000F001083F
:202FC0008858000800F8010810B582B004460C4B53F820000121FDF753FD0A4B33F81430DB
:202FE000ADF8043010238DF8073003238DF80630054B53F8240001A9FDF760FA02B010BDF2
:20300000A8580008B85800085400002008B50346044A52F82000044A32F81310FDF776FB5E
:2030200008BD00BF54000020B858000808B50346044A52F82000044A32F81310FDF736FB02
:2030400008BD00BF54000020B8580008044B53F82030D968034A32F810204A40DA60704713
:2030600054000020B858000800B583B04FF48053ADF8043028238DF8073003238DF8063005
:20308000034801A9FDF71AFA03B05DF804FB00BF0010014008B503484FF48051FDF7AAFA68
:2030A00008BD00BF0010014010B5FDF75FFB4FF48030FDF77BFBFDF761FD012833D110201C
:2030C000FDF722F90220FDF70BF90020FDF714FC0020FDF755FC4FF48060FDF731FC4FF4B7
:2030E00080304FF48011FDF78FFB0120FDF7D8FB39242046FDF710FD0028FAD00220FDF71A
:20310000DFFBFDF7F1FB0828FBD101200146FDF7DDFC4FF480400121FDF7D8FC44F21D0084
:203120000121FDF7ADFC10BD01604360826000230361C3600120704738B504460568C268CD
:203140000369D21A43689A420DDAC268013B02EA0300A26802FB005001F02FFAE368013364
:20316000E360012038BD002038BD00BFF8B504460F460068E1682369C91A6368994231DA05
:20318000E6682169761A9E1BE1685D1E29408D199D422CBFC1EB03053546761BAA42B8BF4E
:2031A0001546521BB242B8BF1646A26802FB0100394602FB05F201F000FAE3682B44E3601D
:2031C00020686268013A1340A26802FB030002FB057102FB06F201F0F0F9E3683344E360BE
:2031E000A819F8BD0020F8BD38B504460568C26803699A420ED003694268013A1340826802
:20320000084602FB035101F0D8F9236901332361012038BD002038BDF8B504460F46016829
:20322000C0682369984231D0E6682369F61A23696568681E03409819A8422CBFC3EB0505B5
:203240003546761BAA42B8BF1546521BB242B8BF1646A268384602FB031102FB05F201F0F2
:20326000ACF923692B44236121686268013A1340A26802FB057002FB031102FB06F201F0D6
:203280009CF9236933442361A819F8BD0020F8BD08B503484FF48051FDF738FA08BD00BF01
:2032A000000C014008B503484FF48051FDF7FEF908BD00BF000C014070B506460C4D0224F9
:2032C00028462146FDF76AFD0028F9D008483146FDF730FD064D012428462146FDF75EFD49
:2032E0000028F9D00248FDF73FFDC0B270BD00BF0038004008B5FFF7DFFF08BD08B5FF205B
:20330000FFF7DAFF08BD00BF82B0019002E0019B013B0193019B002BF9D102B0704700BF90
:2033200030B587B04FF40053ADF8143003238DF8163018238DF81730234C204605A9FDF783
:20334000BDF84FF40043ADF81430204605A9FDF7B5F84FF48043ADF8143004238DF81730B2
:20336000204605A9FDF7AAF84FF48053ADF8143010238DF81730204605A9FDF79FF80023E3
:20338000ADF800304FF48272ADF80220ADF804300222ADF806200124ADF808404FF40072CB
:2033A000ADF80A20ADF80C30ADF80E300723ADF81030064D28466946FDF7FAFB284621463D
:2033C000FDF78CFC07B030BD000C01400038004010B584B0184B6C46186859689A68DB6874
:2033E0000FC4FFF75FFF154C20464FF40071FDF78DF94FF47A70FFF787FF20464FF40071EE
:20340000FDF754F90E480F49FFF720FA0E480F49FFF72EFA01206946FFF7B0FBB0F1FF3F91
:2034200003D10B4800F0A6F903E042F21070FFF76BFF04B010BD00BFC0580008000C014032
:2034400091320008A5320008FD320008F5320008D058000808B50128044B03BF18891B6910
:20346000C0181869FFF720FD08BD00BFCC09002070B50E4615460128074B03BF1C891B692D
:20348000E4181C692046FFF7CDFC204631462A46FFF7DEFC70BD00BFCC09002008B54FF08C
:2034A00080400121FDF786FE30B34FF080400121FDF7EEFE114B1A6801321A60104BA3FB4A
:2034C00002135B09642101FB13232BB90020FFF7BDFD0120FFF7BAFD084B1A68094BA3FB73
:2034E00002139B094FF47A7101FB132323B90022024B1A60FEF746FD08BD00BF34010020DD
:203500001F85EB51D34D621030B585B01C238DF8003000258DF8015001248DF802408DF8BF
:2035200003406846FCF790FE4FF47A73ADF80830ADF80450ADF80A50ADF806504FF080401A
:2035400001A9FDF75FFC4FF0804047212246FDF7D7FD4FF080402146FDF702FD4FF0804083
:2035600021462246FDF760FD05B030BDF8B505460F4616461C4640F227710022FEF73CF869
:20358000384631462246FFF7F1FD0446284640F227710122FEF730F82046F8BD2DE9F843BC
:2035A00007460C4691469846E6682569AE42FBD0384640F225510022FEF71EF820464946D8
:2035C0004246FFF729FE0446384640F225510122FEF712F82046BDE8F88300BF70B582B018
:2035E00005460C46164640F22771FEF7C9F888B130460DF10701FFF7F7FD28B128469DF8D7
:203600000710FEF76FF805E0284640F227710022FDF7F2FF284640F22551FEF7B1F870B13E
:20362000E2682369D21A63689A4208DA2846FEF785F802A901F8010D2046FFF77DFD02B025
:2036400070BD00BF08B503480349044AFFF7C6FF08BD00BF00380140F4090020E0090020FE
:2036600070B588B03148324901224FF48063FFF75BFD3048304901224FF48063FFF754FDE1
:2036800025238DF8003000248DF801408DF8024001258DF803506846FCF7D6FD4FF49053E4
:2036A000ADF8043018238DF8073003238DF80630224E304601A9FCF701FF04238DF80730F3
:2036C0004FF44063ADF80430304601A9FCF7F6FE4FF4E1330493ADF81440ADF81640ADF89D
:2036E0001840ADF81C400C23ADF81A30ADF80840ADF80A404FF40073ADF80C30ADF80E40ED
:203700000F4C204604A9FDF71FFE204602A9FDF7F1FE204640F225512A46FDF76DFF2046F2
:203720002946FDF735FF08B070BD00BFF409002038050020E0090020380100200008014029
:203740000038014008B502460B4602480249FFF70DFF08BD00380140E009002008B50246B7
:203760000B4602480249FFF719FF08BD00380140F40900200FB400B5A3B024AA52F8041BF8
:20378000219201A801F06EFB01A800F051FF014601A8FFF7D7FF23B05DF804EB04B070474C
:2037A0000048704738090020F8B53F4C852323804FF0010E84F802E00223E3700025257147
:2037C000DFF8E8C066460FCEC4F80500C4F80910C4F80D20C4F8113003CEC4F81500C4F807
:2037E0001910337863776523A377E57784F82050C02184F82710A82284F828200B2384F865
:203800002930642084F82A0084F82B1084F82C2084F82D3084F82EE0FF2384F82F3084F8CA
:20382000303084F8313084F8325084F83350636B03F07F4343F4E1736363082384F837306C
:2038400084F8385084F839E084F83A5084F83B50E26B02F07F4242F4E172E26384F83F3009
:2038600084F8405084F841E084F842500CF11C0203CAC4F84300C4F847101288A4F84B20F6
:2038800084F84D5084F84E5084F84F3084F8503084F8513084F8523004F1530029463222F8
:2038A00000F094FEF8BD00BF38090020EC58000810B50E4C012021468522FFF7CBFD2288AF
:2038C000013A92B24FF6FD739A4206D9FFF76CFF012021468522FFF7CBFD044B65229A77C4
:2038E0000022DA7783F8202010BD00BF3809002008B5012002498522FFF7BAFD08BD00BFAC
:203900003809002008B500F058FE08BD08B500F054FE08BD30B58BB0012004A9FFF758FA84
:203920009DF810109DF811209DF812309DF813509DF814409DF815000095019402901A488C
:2039400000F04CFE9DF816109DF817209DF818309DF819000090154800F040FE9DF81E103D
:203960009DF81F209DF820309DF821000090104800F034FE9DF81A109DF81B209DF81C305E
:203980009DF81D0000900B4800F028FE9DF822109DF823209DF824309DF82500009006485C
:2039A00000F01CFE0BB030BD145900083C59000850590008645900087859000810B586B0F9
:2039C000FFF7EEFE0446684604F121010622FFF799FF0DF1060004F127010422FFF792FF72
:2039E0000DF10E0004F12B010422FFF78BFF0DF10A0004F12F010422FFF784FF0DF1120018
:203A000004F14F010422FFF77DFF94F84D301BB102238DF8163002E001238DF81630002013
:203A20006946FFF7D5F9FFF775FF06B010BD00BF3038C3B258B20928C4BFD81F40B20F28AC
:203A4000C4BF203840B2704738B50D4640B2FFF7EFFF000100F0F00468B2FFF7E9FF20448B
:203A6000C0B238BDF0B585B0264B93F821305BB9244B93F82230082B08D1224B93F8233001
:203A8000DC2B3CD0002402E0002400E000241E4E1E4F3046FFF76EFE68460121FFF75EFE12
:203AA0009DF80030532B0ED13846FFF763FE0024012505E000A820442946FFF74FFE0134ED
:203AC0000B2CF7D90124002CE3D000252C460D4E0CE004AA2A4412F8100C12F80F1CFFF790
:203AE000B3FF331983F8210001340235062CF0D9FFF75AFEFFF7FCFE0548FFF73BFE05B056
:203B0000F0BD00BF380900208C5900089C590008A0590008BFF34F8F044AD16801F4E061A0
:203B2000034B0B43D360BFF34F8FFEE700ED00E00400FA0510B4002304E0CC5C4440CC54DA
:203B400001339BB29342F8D35DF8044B704700BF10B4002304E0CC5C4440CC5401339BB212
:203B60009342F8D35DF8044B704700BF2DE9F041CEB0054688461446FFF712FE0746284692
:203B80000B210DF59B72FEF7B5FDB4F80560BDF83621964257D10DF10A030093284627A94A
:203BA000062203ABFEF7AEFC607810F0800F06D000F07F0027A9BDF83621FFF7C9FF27A87B
:203BC00007F12101062200F0E9FC00283BD16FF0740363710023A371552323713B4653F8E1
:203BE000210F04909B88ADF814300DF116003946852200F0E2FC607810F0800F05D000F0C1
:203C00007F0004A98B22FFF795FF20682990A288A379ADF8A8208DF8AA300DF1AB0004A998
:203C20008B2200F0CAFCA37823B94046FF21042200F0CCFCB8F804300093284629A992223B
:203C40004346FEF7BBFB4EB0BDE8F0812DE9F043A5B0054688461446FFF7A2FD07462846BB
:203C60000B210DF18E02FEF745FDB4F80560BDF88E20964240F0FC80E378A13B042B00F203
:203C8000F780DFE803F0AE03207B9A000DF13E030093284602A9072210ABFEF733FC607842
:203CA00010F0800F06D000F07F0002A9BDF88E20FFF74EFF02A8B91C032200F06FFC0028B8
:203CC00000F08F80D4E00DF13E030093284602A90C2210ABFEF716FC607810F0800F06D019
:203CE00000F07F0002A9BDF88E20FFF731FF9DF8082097F821309A4200F2BA809DF80910CE
:203D000097F82220914200F2B3809DF80A0097F82310884200F2AC809DF80B6097F82400DE
:203D2000864200F2A5809DF80CC097F82560B44500F29E809DF80D9097F826C0E14500F267
:203D400097809DF80E904B4500F292809DF80F309A4200F28D809DF81030994200F288802C
:203D60009DF81130984200F283809DF812309E427ED89DF813309C4533D979E00DF13E0334
:203D80000093284602A9212210ABFEF7BBFB607810F0800F06D000F07F0002A9BDF88E2014
:203DA000FFF7D6FE7E1D02A800F042FC024602A8314600F0F3FBA0B15AE00DF13E03009322
:203DC000284602A9342210ABFEF79CFB607810F0800F06D000F07F0002A9BDF88E20FFF77D
:203DE000B7FE0C2363710023A371552323713B4633F8022F9B78ADF844208DF846303B4653
:203E000033F81E2F9B78ADF847208DF8493057F8213FCDF84A30BB88ADF84E30607810F0E1
:203E2000800F05D000F07F0011A90C22FFF782FE20681490A288A379ADF854208DF85630BB
:203E400011AB07CBCDF85700CDF85B10CDF85F20A37823B94046FF21042200F0B7FBB8F82F
:203E600004300093284614A913224346FEF7A6FA25B0BDE8F08300BF2DE9F04190B005467F
:203E800088461446FFF78CFC074628460B210DF13E02FEF72FFCB4F80560BDF83E2096423B
:203EA0005BD10DF10A030093284606A9172203ABFEF728FB607810F0800F06D000F07F0070
:203EC00006A9BDF83E20FFF743FE06A807F12101062200F063FB00283FD10DF11F0007F15E
:203EE000430100F093FB002837D1062363710023A3715523237157F8210F0490BB88ADF895
:203F00001430607810F0800F05D000F07F0004A90622FFF70FFE20680C90A288A379ADF8CB
:203F200034208DF8363010AB53F8300DCDF837009B88ADF83B30A37823B94046FF2104220D
:203F400000F044FBB8F80430009328460CA90D224346FEF733FAFFF7DDFD10B0BDE8F08118
:203F60002DE9F041F4B0054688461446FFF718FC074628460B210DF5E772FEF7BBFBB4F840
:203F80000560BDF8CE2196426ED10DF10E030093284628A99C2204ABFEF7B4FA607810F038
:203FA000800F06D000F07F0028A9BDF8CE21FFF7CFFD28A807F12101062200F0EFFA0028E3
:203FC00052D10DF1A70007F1430100F01FFB00284AD138460DF1B7018522FFF797FC6523A4
:203FE000BB770026FE7787F82060FFF781FC6FF074036371A671552323713B4653F8210FB9
:2040000005909B88ADF818300DF11A003946852200F0D3FA607810F0800F05D000F07F0055
:2040200005A98B22FFF786FD20684F90A288A379ADF840218DF842310DF2431005A98B2254
:2040400000F0BBFAA37823B94046FF21042200F0BDFAB8F80430009328464FA99222434637
:20406000FEF7ACF9FFF756FD74B0BDE8F08100BF2DE9F043B7B0054688461446FFF790FBC0
:204080008146FFF78DFB074628460B210DF1C202FEF730FBB4F80560BDF8C220964240F062
:2040A000B4800DF10A03009328461CA94F2203ABFEF728FAE378D12B40F0A780607810F03F
:2040C000800F06D000F07F001CA9BDF8C220FFF73FFD1CA807F12101062200F05FFA002807
:2040E00040F093800DF1770007F1430100F08EFA002840F08A800DF1C40E4E4656F8210F10
:204100007168B268F368AEE80F00338AAEF80030FFF7CEFB0DF1C40EBEE80F00C9F82100F3
:204120007160B260F360BEF800303382FFF7E0FB20680490A288A379ADF814208DF81630D7
:20414000D8F80030CDF81730B8F80430ADF81B30DDF88730CDF81D30BDF88B30ADF821307B
:204160000DF18D030DF123020DF1BD01D3F800C0D3F804E09E68D868C2F800C0C2F804E03A
:204180009660D060103310328B42EFD11B881380002004A94522FFF76BF906236371002303
:2041A000A3715523237157F8210F1690BB88ADF85C30607810F0800F05D000F07F0016A9DC
:2041C0000622FFF7B7FC20681890A288A379ADF864208DF8663036AB53F8800DCDF867006F
:2041E0009B88ADF86B30A37823B94046FF21042200F0ECF9B8F804300093284618A90D22EF
:204200004346FEF7DBF8FFF785FC37B0BDE8F0832DE9F04190B0054688461446FFF7C0FA2D
:20422000074628460B210DF13E02FEF763FAB4F80560BDF83E2096425FD10DF10A0300933D
:20424000284606A9172203ABFEF75CF9607810F0800F06D000F07F0006A9BDF83E20FFF7AC
:2042600077FC06A807F12101062200F097F9002843D10DF11F0007F1430100F0C7F90028EE
:204280003BD1FFF791FAFFF733FB062363710023A3715523237157F8210F0490BB88ADF832
:2042A0001430607810F0800F05D000F07F0004A90622FFF73FFC20680C90A288A379ADF8FA
:2042C00034208DF8363010AB53F8300DCDF837009B88ADF83B30A37823B94046FF2104226A
:2042E00000F074F9B8F80430009328460CA90D224346FEF763F8FFF70DFC10B0BDE8F081EA
:2043000030B59DB00446FFF74BFA05462046FDF793FF2046022141F696120023FDF7C2FF6F
:20432000002004A94522FFF795F8059A062363F317220592D2238DF8133055238DF81430DA
:204340002B4653F8210F16909B88ADF85C309DF8110010F0800F05D000F07F0016A9062217
:20436000FFF7E8FB04AB93E803001890ADF86410090C8DF866101CAB53F8180DCDF8670003
:204380009B88ADF86B309DF812302BB90DF11700FF21042200F01AF9DDF817000390BDF86D
:2043A0001B30ADF80A30BDF80A300093204618A90D2203ABFEF702F81DB030BD10B588B0A7
:2043C00004460A210DF11F02FEF794F99DF81F30002B51D0222B56D12046092107AAFEF7ED
:2043E00089F9BDF81C30062B4DD906AB0093204603A9072205ABFEF785F89DF80C30A52BA1
:2044000041D19DF81030AA2B3DD19DF80F3003F0F003C02B18D004D8A02B09D0B02B0DD00D
:2044200031E0E02B1CD0F02B20D0D02B2BD111E0204605A903AAFFF709FC24E0204605A9AD
:2044400003AAFFF793FB1EE0204605A903AAFFF787FD18E0204605A903AAFFF709FE12E04A
:20446000204605A903AAFFF707FD0CE0204605A903AAFFF7CDFE06E02046022141F69612C5
:204480000123FDF70FFF08B010BD00BF72B60348006885460248006887467047006000086E
:2044A0000460000830B593B0002069464522FEF7D1FF9DF80030A52B28D19DF80D309DF878
:2044C0000E00000440EA03609DF80F3040EA03209DF8103018430DF11301FDF73DFDFDF7B8
:2044E000E5FC04460028FAD002280DD10020FFF707FF4525684600212A4600F067F8002063
:2045000069462A46FEF7B4FF204600E0002013B030BD00BF10B5FEF7C7FD0020FEF754FD1B
:204520000120FEF751FD0020FEF770FD0120FEF77DFDFEF799FDFFF793F8FEF703FDFFF70E
:20454000B7F9FFF78FFAFEF7EBFEFEF741FFFEF7DBFFFFF733FA01200B49FDF795FCFFF737
:20456000A1FF0446FEF796FD48B9012C07D0074B5B681B68B3F1FF3F01D0FFF787FF0024D9
:204580002046FFF71BFFFBE7080A0020CC090020014B1868704700BFC400002030B500236E
:2045A000934208D0C55C0133CC1814F8014CA542F6D0281B30BD002030BD10B50023934215
:2045C00003D0CC5CC4540133F9E710BD02440346934202D003F8011BFAE770470FB40A4BEA
:2045E00013B51C6824B1A36913B9204600F00CFE05AB2046A168049A019300F091F902B0E5
:20460000BDE8104004B07047C400002010F8012B11F8013B012A28BF9A42F7D0D01A704787
:20462000034611F8012B03F8012B002AF9D17047034613F8012B002AFBD1181A0138704792
:204640002DE9F0478D688146AB420C4692461F4643D38B8913F4906F3DD026680969022274
:20466000C1EB0608666906EB460696FBF2F608F101023A44964238BF16465B050FD531469B
:2046800000F0E6FE054698B121694246FFF795FFA38923F4906343F08003A38113E032469B
:2046A00000F02AFF054670B94846216900F08CFE0C23C9F80030A3894FF0FF3043F04003AB
:2046C000A381BDE8F087256166614544C8EB06062560A6603D46AF4200D23D462A462068B9
:2046E000514600F055FEA36800205B1BA36023681D442560BDE8F0872DE9F0439DB0039383
:204700008B8907461C060D4616460CD50B6953B9402100F09DFE2860286110B90C233B6076
:20472000C7E040236B610023099320238DF8293030238DF82A3033461C4613F8012B1AB9AC
:20474000B4EB06090FD002E0252AF5D1F8E73846294632464B46FFF773FF013000F0A48053
:20476000099B4B4409932378002B00F09D8000234FF0FF3204930793059206938DF853309B
:204780001A9304F101094D4E4C4630462178052200F0F0FD09F10109049B28B1861B0120EF
:2047A000B04003430493EEE7D90644BF20228DF853201A0744BF2B228DF8532022782A2AE4
:2047C00002D0079B21460EE0039A111D12680391002A01DB079204E0524243F0020307924F
:2047E000049301340AE00C4622780131303A092A03D80A2000FB0323F5E7079323782E2BB8
:2048000019D163782A2B09D1039B02341A1D1B680392002BB8BF4FF0FF330BE0611C0023E3
:204820000C4622780131303A092A03D80A2000FB0323F5E70593224E21783046032200F08F
:2048400099FD30B1861B4020B040049B01340343049321781B480622661C8DF8281000F0EC
:2048600089FD88B1184B33B9039B073323F007030833039314E003AB0093384604A92A4694
:20488000124BAFF3008007E003AB0093384604A92A460E4B00F0BAF9B0F1FF3F804603D062
:2048A000099B4344099346E7AB895B0601D4099801E04FF0FF301DB0BDE8F083B0590008B4
:2048C000B6590008BA5900080000000041460008936810B5013B002B936005DA9469A3423C
:2048E00008DBCBB20A2B05D01368581C10601970C8B210BDBDE8104000F0C2BAF8B50546C6
:204900000E461446D718BC4208D0284614F8011B3246FFF7DDFF431CF5D100E00020F8BD6A
:204920002DE9F0439DB00D4617460393064618B183690BB900F068FC734B9D4201D1756836
:2049400008E0724B9D4201D1B56803E0704B9D4208BFF568AB8918070AD52B6943B1002366
:20496000099320238DF8293030238DF82A3038E03046294600F0D8FA0028F0D04FF0FF3033
:20498000BEE0039A111D12680391002A70DB0792013423782E2B7DD05E4F21783846032233
:2049A00000F0E8FC30B1C71B4020B840049B013403430493217858480622671C8DF82810B6
:2049C00000F0D8FC002800F08980544B002B7CD1039B073323F0070308330393099B4344EA
:2049E00009933B461C4613F8012B1AB9B4EB07090ED002E0252AF5D1F8E7304629463A4666
:204A00004B46FFF77BFF013075D0099B4B4409932378002B6FD000234FF0FF320493079387
:204A2000059206938DF853301A9304F101093C4F4C4638462178052200F09CFC09F10109AB
:204A4000049B28B1C71B0120B84003430493EEE7D90644BF20228DF853201A0744BF2B22A4
:204A60008DF8532022782A2A8BD0079B214605E0524243F002030792049389E70C462278AF
:204A80000131303A092A03D80A2000FB0323F5E707937EE763782A2B09D1039B02341A1D31
:204AA0001B680392002BB8BF4FF0FF330BE0611C00230C4622780131303A092A03D80A2080
:204AC00000FB0323F5E7059366E703AB0093304604A92A46134BAFF3008007E003AB009378
:204AE000304604A92A460F4B00F090F8B0F1FF3F80467FF473AFAB895B063FF53FAF0998BF
:204B00001DB0BDE8F08300BFE4590008045A0008245A0008B6590008BA590008000000008E
:204B2000B0590008FD4800082DE9F84315461F468A680B6906469A42A8BF13462B6091F8A4
:204B400043200C46DDF820800AB101332B602368990602D52B6802332B60236813F00609C0
:204B60001DD094F843302268003318BF012392061FD5E118302081F843005A1C94F84510A9
:204B80002244023382F8431013E03046394604F119020123C047013007D009F10109E26834
:204BA0002B68D31A9945F0DBDBE74FF0FF30BDE8F8833046394604F14302C0470130F4D051
:204BC00023682A6803F00603E168042B08BFC2EB01052369A2680CBF25EAE57500259A42FF
:204BE000C4BFC3EB0203ED184FF00009A9450ADA3046394604F11A020123C0470130D4D05A
:204C000009F10109F2E70020BDE8F8832DE9FF470E7E80466E2E0C4691469A460C9D01F189
:204C2000430000F0A58011D8632E22D009D8002E00F0AF80582E40F0BF8081F845607B4AAA
:204C40004FE0642E1ED0692E1CD0B5E0732E00F0A48009D86F2E2BD0702E40F0AD800B68F1
:204C600043F020030B6038E0752E21D0782E34D0A2E02B6801F142071A1D1B682A6081F810
:204C800042309DE022682B6812F0800F03D01A1D2A601D6805E05106F9D51A1D2A60B3F9E7
:204CA0000050002D39DA2D236D4284F8433034E022682B6812F0800F03D01A1D2A601D689B
:204CC00004E05206F9D51A1D2A601D88237E574A6F2B14BF0A2308231BE07823544A84F8AD
:204CE00045302368296813F0800F01F104062E6001D00D6802E05F06FBD50D88DE0744BF2D
:204D000043F0200323601DB9236823F0200323601023002184F8431001E0444A0A23666813
:204D2000002EA66003DB216821F00401216005B96EB104F14201B5FBF3F603FB1655555D78
:204D40000F4601F801593546002EF4D100E00746082B0AD12368DD0707D5626823699A4285
:204D600003DC302307F8013C013FC01B20612CE009682B6811F0800F626904D0191D29602B
:204D80001B681A6005E04906F8D5191D29601B681A8000232361074617E02B681A1D2A60FA
:204DA0001F683846FFF744FC63682061984288BF23612369636005E004F1420784F8426037
:204DC00001232361002384F84330CDF800A04046214603AA4B46FFF7A7FE013002D14FF0AB
:204DE000FF301FE0404649463A462369D0470130F5D023689B0705D4E068039B9842B8BF1A
:204E000018460FE00025E268039BD31A9D42F3DA4046494604F119020123D0470130DED060
:204E20000135F0E704B0BDE8F08700BFC1590008D259000810B59AB0009104916FF00041AC
:204E4000029105914FF6FF71ADF80E104FF402746946ADF80C40FFF74FFC009B00221A70D0
:204E60001AB010BD30B51346044A05460C46106829462246BDE83040FFF7DCBFC400002099
:204E800070B50E461446054618B183690BB900F0BBF9224B9C4201D16C6808E0204B9C42B5
:204EA00001D1AC6803E01F4B9C4208BFEC68A369A360A3891A0709D523693BB12369206800
:204EC000F6B2C01A636998420FDB08E02846214600F02AF80028F1D04FF0FF3070BD2846FF
:204EE000214600F013F90028F6D1A3680130013BA36023685A1C22601E706369984204D05A
:204F0000A389DB0707D50A2E05D12846214600F0FDF80028E0D1304670BD00BFE45900085F
:204F2000045A0008245A0008324B70B51D6806460C4625B1AB6913B9284600F065F92E4BD5
:204F40009C4201D16C6808E02C4B9C4201D1AC6803E02B4B9C4208BFEC68A28993B21907C8
:204F600020D4DD0605D4092342F040023360A2813BE0580712D5616B41B104F144039942F5
:204F800002D0304600F020FA00236363A38923F02403A3810023636023692360A38943F0F8
:204FA0000803A38123694BB9A38903F42073B3F5007F03D03046214600F090F9A38913F0FD
:204FC000010205D00022A26062695242A26103E0990758BF6269A26022694AB903F080000B
:204FE00080B230B143F04003A3814FF0FF3070BD002070BDC4000020E4590008045A00088D
:20500000245A00088A892DE9F041054610070C4657D44B68002B02DC0B6C002B18DDE66A2E
:20502000B6B102F48052002392B22F682B600AB1626D10E0216A28460123B047411C024685
:2050400009D12B683BB11D2B01D0162B46D12F600020BDE8F081A3895B0705D56368D21AA2
:20506000636B0BB1236CD21AE66A2846216A0023B047461CA28905D12B681BB11D2B01D0ED
:20508000162B19D1002363602369D104236004D5421C01D12B6803B96065616B2F6000297A
:2050A000D6D004F14403994202D0284600F08CF900206063BDE8F08142F04002A281BDE849
:2050C000F0810E69002EC3D00B680E60C6EB030893070CBF4B6900238B6012E0A3894FF006
:2050E000FF3043F04003A381BDE8F081A76A2846216A32464346B8470028EFDD0644C0EBDE
:205100000808B8F1000FF1DCA2E7000038B50B6905460C46DBB118B183690BB900F074F812
:205120000C4B9C4201D16C6808E00B4B9C4201D1AC6803E0094B9C4208BFEC68B4F90C3079
:205140002BB128462146BDE83840FFF75BBF002038BD00BFE4590008045A0008245A00086C
:20516000F8B5074600F1480494B1A5686668013E0CD4AB89012B07D9B5F90E30013303D086
:2051800038462946FFF7C2FF6835F0E72468EBE7F8BD0000002310B50446036043608360C9
:2051A00081814366C28103614361836119465C300822FFF70BFA054B24626362044BA36216
:2051C000044BE362044B236310BD00BF6555000887550008BF550008E355000870B54B1E4A
:2051E00068255D430E4605F1740100F031F9044640B1002180E842000C30A06005F1680207
:20520000FFF7E4F9204670BD836910B5044633BB8364C3640365124B124A1B6882629842CF
:2052200004BF0123836100F01FF86060204600F01BF8A060204600F017F80421E060002287
:205240006068FFF7A7FFA06809210122FFF7A2FFE06812210222FFF79DFF0123A36110BDD8
:20526000AC59000861510008F8B51B4B07461E68B36913B93046FFF7C7FF4836B4687368F2
:20528000013B04D4B4F90C5075B16834F8E733682BB938460421FFF7A1FF306008B13668B1
:2052A000ECE70C233B60F8BD4FF6FF73E3810123A38165662560A560656025616561A561CD
:2052C00004F15C0029460822FFF780F96563A563A564E5642046F8BDAC590008F0B58B8972
:2052E00091B09E0705460C4625D4B1F90E10002908DAA389002713F0800F14BF40264FF4FE
:2053000080660DE001AA00F093F90028F1DB029F4FF4806607F47047B7F500514F424F4105
:205320002846314600F094F860B9A3899A051DD443F00203A38104F1470323602361012371
:20534000636113E00A4BAB62A389206043F08003A381206166614FB12846B4F90E1000F03D
:2053600079F918B1A38943F00103A38111B0F0BD6151000810B5C9B202449042034605D0CD
:205380001C7801308C42F8D1184610BD002010BD814270B501D300230EE08C18A042FAD27A
:2053A0008518134613F1FF3305D351426618F65C2944CE54F6E770BD934203D0CC5CC45405
:2053C0000133F9E770BD000030B500293CD051F8042C0B1F1D49002AB8BF9B180A680C4651
:2053E00012B95A600B6030BD93420DD219685818904203D15A581144426819605A6023601E
:2054000030BD994203D80A4651680029F9D1146815199D420AD11B682344D018884213607A
:2054200012D10868034413604B680CE002D90C23036030BD18681C188C4203D10C684968EB
:20544000204418605960536030BD00BFC409002070B5CD1C25F0030508350C2D38BF0C25A2
:20546000002D06463FDB8D423DD3214B1C6818462146A1B10B685B1B0ED40B2B03D90B606B
:20548000CC18CD501FE08C4202D1626802601AE04B6863600C4616E00C464968E9E7154C53
:2054A00023681BB9304600F04DF820602946304600F048F8431C014615D0C41C24F00304C7
:2054C00084420AD1256004F10B00231D20F00700C31A0BD05A42E25070BD3046611A00F0BB
:2054E00031F80130EED10C233360002070BD00BFC4090020C0090020F8B5064614460D4649
:2055000021B91146BDE8F840FFF7A2BF1AB9FFF75BFF2046F8BD00F0BFF8A0420ED2304609
:205520002146FFF795FF074650B129462246FFF744F830462946FFF747FF01E02846F8BDFE
:205540003846F8BD38B5064C0023054608462360FCF798F9431C02D1236803B12B6038BD25
:20556000C809002010B50C46B1F90E1000F09EF8002803DB636D0344636510BDA38923F4E0
:205580008053A38110BD2DE9F0411D468B890746DB050C46164605D5B1F90E1000220223C5
:2055A00000F068F8A389384623F48053A381B4F90E1032462B46BDE8F04100F017B810B5D5
:2055C0000C46B1F90E1000F055F8431CA38903D123F48053A38110BD43F48053A381606547
:2055E00010BDB1F90E1000F013B8000038B5074C054600202060084611461A46FCF794F9AB
:20560000431C02D1236803B12B6038BDC809002038B5064C0023054608462360FCF75CF9E2
:20562000431C02D1236803B12B6038BDC809002038B5074C00230546084611462360FCF7BF
:2056400053F9431C02D1236803B12B6038BD00BFC809002038B5064C0023054608462360DF
:20566000FCF74AF9431C02D1236803B12B6038BDC809002038B5074C054600202060084699
:2056800011461A46FCF740F9431C02D1236803B12B6038BDC809002051F8040C002802DAE8
:2056A00004390B58184404387047000038B5074C054600202060084611461A46FCF72CF9B3
:2056C000431C02D1236803B12B6038BDC80900202E2E2F73797374656D2F7372632F73742B
:2056E0006D333266312D7374647065726970682F6D6973632E6300002E2E2F737973746512
:205700006D2F7372632F73746D333266312D7374647065726970682F73746D333266313077
:20572000785F666C6173682E630000002E2E2F73797374656D2F7372632F73746D333266FE
:20574000312D7374647065726970682F73746D3332663130785F6770696F2E630000000052
:205760002E2E2F73797374656D2F7372632F73746D333266312D7374647065726970682FD4
:2057800073746D3332663130785F7263632E63002E2E2F73797374656D2F7372632F73742C
:2057A0006D333266312D7374647065726970682F73746D3332663130785F7370692E63001D
:2057C0002E2E2F73797374656D2F7372632F73746D333266312D7374647065726970682F74
:2057E00073746D3332663130785F74696D2E63002E2E2F73797374656D2F7372632F7374BA
:205800006D333266312D7374647065726970682F73746D3332663130785F75736172742E3C
:20582000630000006F6374657400000074696D656F75740035000000464C4153485F457226
:2058400061736550616765204572726F720D0A00464C4153485F50726F6772616D576F7274
:2058600064204572726F720D0A000000484947482044656E7369747920466C617368206DC8
:20588000656D6F72790D0A004D656469756D2044656E7369747920466C617368206D656DF7
:2058A0006F72790D0A00000010000000100000000000000000000000100020000000000027
:2058C0000202020202020202020202020202020257495A4348495020496E697469616C6937
:2058E0007A6564206661696C2E0D0A0057495A3535305745420000000000000000000000F2
:20590000000000000000000057495A6E65740000000000004D41433A20253032583A2530AD
:2059200032583A253032583A253032583A253032583A253032580D0A0000000049503A206F
:2059400025642E25642E25642E25640D0A00000047573A2025642E25642E25642E25640DCF
:205960000A000000534E3A2025642E25642E25642E25640D0A000000444E533A2025642E67
:2059800025642E25642E25640D0A0000496E707574204D4143203F20000000005200000027
:2059A0000D0A4F4B0D0A00004300000064000020232D302B2000686C4C0065666745464769
:2059C00000303132333435363738394142434445460030313233343536373839616263648E
:2059E0006566000000000000000000000000000000000000000000000000000000000000DC
:205A0000000000000000000000000000000000000000000000000000000000000000000086
:205A2000000000000000000000000000000000000000000000000000000000000000000066
:205A400000000000785634120204060800000000010203040102030406070809D4000020F8
:205A600000000000FFFFFFFF2C5800083458000800C0000001025735353030002D280008C9
:205A80003128000835280008392800083D28000841280008006000080010014000100140EF
:205AA000000000000000000000000000E4590008045A0008245A00080000000000000000B5
:205AC0000000000000000000A85900080000000000000000000000000000000000000000BD
:205AE0000000000000000000000000000000000000000000000000000000000000000000A6
:105B0000000000000000000064000020325476987D
:20600000005000201962000885710108897101088D7101089171010895710108000000006A
:20602000000000000000000000000000997101089D71010800000000A1710108A5710108FC
:206040004562000845620008456200084562000845620008456200084562000845620008C8
:206060004562000845620008456200084562000845620008456200084562000845620008A8
:20608000456200084562000845620008456200084562000845620008456200084562000888
:2060A00045620008456200084562000845620008E11001084562000845620008456200081D
:2060C0004562000845620008456200084562000845620008251201087115010845620008D7
:2060E000456200084562000845620008000000000000000000000000000000000000000093
:2061000000000000000000005FF808F100B583B0304B314A1360314A1360314B31490022D8
:2061200001E01A6004338B42FBD32B4B1B6813B92A4B1B6803B1FEE7264B2B4A13602B4A0E
:2061400013602B4B2B4A2C4803E011681960043304328342F9D3244B1A68284B9A4204D185
:20616000224B1A681B689A4200D0FEE702F0E0FB01A8694602F05CFB214B224EF61AB610FC
:2061800000241D4603E055F8243098470134A642F9DC1D4B1D4EF61AB61000241D4603E010
:2061A00055F8243098470134A642F9DC0198009910F0E6FE0546164B164CE41AA4101E4633
:2061C00003E0013C56F824309847002CF9DC284602F000FBBABADECA8C020020684500202B
:2061E0008C0200206C45002000000020880200200000002010B801088C02002078563412A3
:2062000048620008486200084862000848620008486200084862000808B5FFF777FF00BF6A
:20622000FEE700BFFEE700BFFEE700BFFEE700BFFEE700BFFEE700BFFEE700BFFEE700BF3E
:20624000FEE700BFFEE700BF10B50446B0F5E06F0FD0B0F5C06F0CD0B0F5A06F09D0B0F532
:20626000806F06D0B0F5407F03D00548632102F007FB44F0BF6444F40034024BDC6010BD44
:20628000E487010800ED00E010B50446C378012B03D92048752102F0F3FA63780F2B03D99D
:2062A0001C48762102F0ECFAA3780F2B03D91948772102F0E5FAE37803B3174BDB68DB433C
:2062C000C3F30223C3F104020F2121FA03F3617801FA02F2A1781940114309012278C9B23B
:2062E0000E4B1A4482F800132278510902F01F02012000FA02F243F8212010BD23785909FE
:2063000003F01F03012202FA03F32031034A42F8213010BDE487010800ED00E000E100E05B
:2063200038B504460D46B0F1005F06D0B0F1006F03D00948AA2102F0A3FA084B9D4203D961
:206340000548AB2102F09CFA25F0604121F07F012143034B996038BDE4870108FEFF0F0035
:2063600000ED00E010B50446042806D010F1050F03D00748D52102F083FA042C054B1A68A1
:206380000CBF42F0040222F004021A6010BD00BFE487010810E000E038B505460C464D4B76
:2063A00098420BD003F58063984207D003F5A053984203D04848E52102F062FA2368F3B1F1
:2063C000B3F5803F1BD0B3F5003F18D0B3F5403F15D0B3F5802F12D0B3F5A02F0FD0B3F559
:2063E000C02F0CD0B3F5E02F09D0B3F5002F06D0B3F5102F03D03848E62102F041FA23798B
:20640000012B03D93448E72102F03AFA6379012B03D93148E82102F033FAA36843B3B3F59C
:20642000003F25D0B3F5802F22D0B3F5C02F1FD0B3F5002F1CD0B3F5202F19D0B3F5402F9F
:2064400016D0B3F5602F13D093B1B3F5003F0FD0B3F5C02F0CD0B3F5002F09D0B3F5202F18
:2064600006D0B3F5402F03D01B48E92102F008FAE36833B1B3F5006F03D01748EA2102F086
:20648000FFF9237C013BDBB20F2B03D91248EB2102F0F6F96B6823F4702323F4807322682E
:2064A000217942EA012213436B60AA680B4B1340E168A2680A43617942EA41021343AB60CD
:2064C000EA6A22F47002237C013BDBB242EA0353EB6238BD002401400C880108FDF7F1FFCE
:2064E00038B504460D46114B98420CD003F58063984208D003F5A053984204D00C484FF443
:206500009A7102F0BDF9012D04D9094840F2351102F0B6F925B1A36843F00103A36038BD43
:20652000A36823F00103A36038BD00BF002401400C88010838B504460D460F4B984208D0EA
:2065400003F5C053984204D00C4840F24D1102F097F9012D04D909484FF4A77102F090F9EA
:2065600025B1A36843F48073A36038BDA36823F48073A36038BD00BF002401400C8801084A
:2065800010B504460A4B98420CD003F58063984208D003F5A053984204D006484FF4C271F7
:2065A00002F06EF9A36843F00803A36010BD00BF002401400C88010810B504460B4B984269
:2065C0000CD003F58063984208D003F5A053984204D007484FF4C97102F052F9A06800F0B8
:2065E0000800003018BF012010BD00BF002401400C88010810B504460A4B98420CD003F5CB
:206600008063984208D003F5A053984204D006484FF4D57102F034F9A36843F00403A3600E
:2066200010BD00BF002401400C88010810B504460B4B98420CD003F58063984208D003F52C
:20664000A053984204D007484FF4DC7102F018F9A06800F00400003018BF012010BD00BF07
:20666000002401400C88010838B504460D46114B98420CD003F58063984208D003F5A05304
:20668000984204D00C484FF4E97102F0F9F8012D04D9094840F2D31102F0F2F825B1A36849
:2066A00043F4A003A36038BDA36823F4A003A36038BD00BF002401400C880108F8B5044693
:2066C0000D4616461F46374B98420CD003F58063984208D003F5A053984204D032484FF48B
:2066E000167102F0CDF8112D04D92F4840F2592102F0C6F8731EDBB20F2B04D92A4840F295
:206700005A2102F0BDF8072F04D9274840F25B2102F0B6F8092D0DD9E168A5F10A0303EB91
:20672000430307229A4021EA02029F4042EA0703E3600AE0216905EB450307229A4021EAEF
:2067400002029F4042EA07032361062E0CD8626B013E06EB86061F23B34022EA0303B540BF
:2067600043EA05066663F8BD0C2E0DD8226B073E06EB86061F23B34022EA030305FA06F6B3
:2067800043EA06052563F8BDE26A0D3E06EB86061F23B34022EA0303B54043EA0506E662B4
:2067A000F8BD00BF002401400C88010810B504464F4B984225D01433984222D014339842B7
:2067C0001FD0143398421CD01433984219D01433984216D01433984213D003F56273984201
:2067E0000FD0143398420CD01433984209D01433984206D01433984203D03E486F2102F0D0
:206800003FF8236823F001031B041B0C2360002323606360A360E360354B9C4205D1083BB0
:206820005A6842F00F025A6010BD334B9C4205D11C3B5A6842F0F0025A6010BD2F4B9C427E
:2068400005D1303B5A6842F470625A6010BD2C4B9C4205D1443B5A6842F470425A6010BDCB
:20686000284B9C4205D1583B5A6842F470225A6010BD254B9C4205D16C3B5A6842F4700218
:206880005A6010BD214B9C4205D1803B5A6842F070625A6010BD1E4B9C4205D1083B5A6827
:2068A00042F00F025A6010BD1A4B9C4205D11C3B5A6842F0F0025A6010BD174B9C4205D11B
:2068C000303B5A6842F470625A6010BD134B9C4205D1443B5A6842F470425A6010BD104BDF
:2068E0009C4204D1583B5A6842F470225A6010BD080002403C8801081C000240300002405A
:2069000044000240580002406C00024080000240080402401C040240300402404404024037
:206920005804024038B505460C46504B984225D01433984222D0143398421FD01433984281
:206940001CD01433984219D01433984216D01433984213D003F5627398420FD0143398428F
:206960000CD01433984209D01433984206D01433984203D03E48CF2101F082FFA368102B28
:2069800004D01BB13A48D02101F07AFFE368013B4FF6FE72934203D93548D12101F070FFBE
:2069A0002369402B04D01BB13148D22101F068FF6369802B04D01BB12D48D32101F060FFAC
:2069C000A3694BB1B3F5807F06D0B3F5007F03D02748D42101F054FFE3694BB1B3F5806FB1
:2069E00006D0B3F5006F03D02148D52101F048FF236A202B04D01BB11D48D62101F040FF3C
:206A0000636AB3F5405F0AD0B3F5005F07D0B3F5805F04D01BB11648D72101F031FFA36AFF
:206A2000B3F5804F04D01BB11148D82101F028FF2B6823F4FF4323F07003A168226A11437A
:206A40002269114362691143A2691143E2691143626A1143A26A0A4313432B60E3686B60CA
:206A60002368AB606368EB6038BD00BF080002403C88010838B504460D461F4B984226D0DB
:206A80001433984223D01433984220D0143398421DD0143398421AD01433984217D0143369
:206AA000984214D003F56273984210D0143398420DD0143398420AD01433984207D0143359
:206AC000984204D00D4840F2291101F0D9FE012D04D90A484FF4957101F0D2FE25B12368B7
:206AE00043F00103236038BD236823F001031B041B0C236038BD00BF080002403C880108B1
:206B000010B50446431E012B40F29B80042800F09880082800F09580102800F092802028A1
:206B200000F08F80402800F08C80802800F08980B0F5807F00F08580B0F5007F00F08180A3
:206B4000B0F5806F7DD0B0F5006F7AD0B0F5805F77D0B0F5005F74D0B0F5804F71D0B0F589
:206B6000004F6ED0B0F5803F6BD0B0F5003F68D0B0F5802F65D0B0F5002F62D0B0F5801FFA
:206B80005FD0B0F5001F5CD0B0F5800F59D0B0F5000F56D0B0F1807F53D0B0F1007F50D09C
:206BA000B0F1806F4DD0B0F1006F4AD02B4B984247D00133984244D00233984241D004331E
:206BC00098423ED0083398423BD01033984238D02033984235D04033984232D0803398427A
:206BE0002FD003F5807398422BD003F50073984227D003F58063984223D0B0F1102F20D022
:206C000003F5C05398421CD003F50053984218D003F58043984214D003F50043984210D028
:206C200003F5803398420CD003F50033984208D003F58023984204D0094840F2B71101F091
:206C40001FFE14F0805F14BF064B074B1B6803EA0400003018BF012010BD00BF0100001085
:206C60003C880108000402400000024010B50446022804D9054840F2031101F001FE044BD7
:206C80001A6802F0380214431C6010BD6C8801080020024010B50446102805D020B107480B
:206CA00040F22F1101F0ECFD054B1A6822F010021A601A6814431C6010BD00BF6C8801083A
:206CC00000200240034B044A5A6002F188325A60704700BF0020024023016745024B1A691D
:206CE00042F080021A6170470020024010B5044630F0350300D120B9034840F2CC5101F0B0
:206D0000BFFD024BDC6010BD6C880108002002400B4BDB6813F0010F0DD1094BDB6813F0DE
:206D2000040F0AD1064BDB6803F01003002B0CBF042003207047012070470220704700BF67
:206D40000020024010B50446FFF7E2FF02E0FFF7DFFF013C012801D1002CF8D1002C08BF15
:206D6000052010BD38B5044600F17842114B9A4204D9114840F2A71101F082FD4FF43020E4
:206D8000FFF7E0FF042813D10C4D2B6943F002032B616C612B6943F040032B614FF4302067
:206DA000FFF7D0FF2B6923F00203DB04DB0C2B6138BD00BFFEFF0F006C88010800200240F1
:206DC00030B583B004460D460023019300F178421A4B9A4204D91A4840F2B52101F050FDD6
:206DE0004FF40050FFF7AEFF042824D1154B1A6942F001021A61ABB223804FF40050FFF720
:206E0000A1FF042810D102340194019B2D0C1D804FF40050FFF796FF0A4B1A6922F001027D
:206E2000D204D20C1A6106E0064B1A6922F00102D204D20C1A6103B030BD00BFFEFF0F00BA
:206E40006C880108002002402DE9F04105460C46494B98421BD003F58063984217D003F502
:206E60008063984213D003F5806398420FD003F5806398420BD003F58063984207D003F5CA
:206E80008063984203D03D48B22101F0F9FCE3788BB1042B0FD0282B0DD0482B0BD0142BC2
:206EA00009D0102B07D01C2B05D0182B03D03348B32101F0E5FC23881BB93048B42101F0D7
:206EC000DFFCE37803F00F073E4613F0100F0AD0A378013BDBB2022B03D92848BB2101F0C9
:206EE000CFFCA6783E432378FBB12F68002301204FF00F0C16E000FA03F2218811409142FA
:206F00000FD199000CFA01F827EA080706FA01F10F43E178282901D16A6102E0482908BF34
:206F20002A610133072BE6D92F602388FF2B21D96F68002301204FF00F0C18E003F10802D8
:206F400000FA02F22188114091420FD199000CFA01F827EA080706FA01F10F43E1782829F0
:206F600008BF6A61E178482908BF2A610133072BE4D96F60BDE8F08100080140A0880108E1
:206F800038B504460D462A4B98421CD003F58063984218D003F58063984214D003F580631B
:206FA000984210D003F5806398420CD003F58063984208D003F58063984204D01D484FF4C8
:206FC0008F7101F05DFC6B1E9BB2012B28D9042D26D0082D24D0102D22D0202D20D0402D3B
:206FE0001ED0802D1CD0B5F5807F19D0B5F5007F16D0B5F5806F13D0B5F5006F10D0B5F54A
:20700000805F0DD0B5F5005F0AD0B5F5804F07D0B5F5004F04D0074840F21F1101F030FCE6
:20702000A36803EA0500003018BF012038BD00BF00080140A088010838B504460D462A4BFE
:2070400098421CD003F58063984218D003F58063984214D003F58063984210D003F58063C4
:2070600098420CD003F58063984208D003F58063984204D01D484FF4A27101F001FC6B1E12
:207080009BB2012B28D9042D26D0082D24D0102D22D0202D20D0402D1ED0802D1CD0B5F51C
:2070A000807F19D0B5F5007F16D0B5F5806F13D0B5F5006F10D0B5F5805F0DD0B5F5005FF5
:2070C0000AD0B5F5804F07D0B5F5004F04D0074840F2451101F0D4FBE36803EA05000030B5
:2070E00018BF012038BD00BF00080140A088010838B504460D46144B98421CD003F58063E0
:20710000984218D003F58063984214D003F58063984210D003F5806398420CD003F5806313
:20712000984208D003F58063984204D0074840F2691101F0A5FB25B904484FF4B57101F004
:207140009FFB256138BD00BF00080140A088010838B504460D46144B98421CD003F5806357
:20716000984218D003F58063984214D003F58063984210D003F5806398420CD003F58063B3
:20718000984208D003F58063984204D0074840F2791101F075FB25B904484FF4BD7101F0BC
:2071A0006FFB656138BD00BF00080140A088010838B504460D46431E012B40F290800428EC
:2071C00000F08D80082800F08A80624B984200F086802033984200F082805F4B98427ED01A
:2071E000803398427BD05D4B984278D003F58073984274D003F58073984270D0584B984262
:207200006DD003F58063984269D0B0F5805F66D0B0F5EA1F63D0B0F5EB1F60D0B0F5004FD5
:207220005DD0504B98425AD00133984257D00233984254D00433984251D0083398424ED0B5
:20724000B0F1201F4BD03033984248D0464B984245D003F58073984241D003F50073984243
:207260003DD0424B98423AD003F57063984236D0B0F5011F33D03E4B984230D001339842AC
:207280002DD0023398422AD00433984227D00833984224D01033984221D0203398421ED0AE
:2072A000403398421BD08033984218D003F58073984214D003F50073984210D003F5806378
:2072C00098420CD003F50063984208D003F58053984204D0274840F22A2101F0D1FA012D9C
:2072E00004D9244840F22B2101F0CAFA002C224BB4BFDB695B68C4F30340A1B204F4401268
:20730000B2F5401F07D123F070631B4A506820F07060506012E014F4801F07D0032202FA6B
:2073200000F023EA000343F0706307E0620D120101FA02F223EA020343F070631DB1620D9A
:20734000120191400B43002C0B4AB4BFD361536038BD00BF100014004000160000011800D9
:2073600000081A0001002000000130000011200001000080A08801080000014010B5044666
:2073800045F25553984204D018B103485F2101F077FA024B1C6010BDD488010800300040FF
:2073A00010B50446062803D90348732101F068FA024B5C6010BD00BFD48801080030004018
:2073C00010B50446B0F5805F03D30348802101F057FA024B9C6010BDD4880108003000402B
:2073E0004AF6AA22014B1A60704700BF003000404CF6CC42014B1A60704700BF00300040D9
:207400000D4B1A6842F001021A6059680B4A0A405A601A6822F0847222F480321A601A687B
:2074200022F480221A605A6822F4FE025A604FF41F029A60704700BF001002400000FFF86B
:2074400010B5044650B1B0F5803F07D0B0F5802F04D0104840F2111101F012FA0E4B1A6835
:2074600022F480321A601A6822F480221A60B4F5803F03D0B4F5802F06D010BD064B1A680D
:2074800042F480321A6010BD034B1A6842F4A0221A6010BD088901080010024038B50C4683
:2074A000054650B1B0F5803F07D0B0F5403F04D01E4840F27F1101F0E3F974B3B4F5802FD9
:2074C0002BD0B4F5002F28D0B4F5402F25D0B4F5801F22D0B4F5A01F1FD0B4F5C01F1CD0CF
:2074E000B4F5E01F19D0B4F5001F16D0B4F5101F13D0B4F5201F10D0B4F5301F0DD0B4F54C
:20750000401F0AD0B4F5501F07D0B4F5601F04D006484FF4C07101F0B3F9054B5A6822F4C0
:207520007C122C4314435C6038BD00BF088901080010024010B50446012804D903484FF4F8
:20754000CA7101F09DF9024B1C6010BD088901086000424210B50446022804D905484FF4AF
:207560000E7101F08DF9044B5A6822F0030214435C6010BD0889010800100240024B586814
:2075800000F00C00704700BF0010024010B50446A0B1802812D0902810D0A0280ED0B02827
:2075A0000CD0C0280AD0D02808D0E02806D0F02804D006484FF4197101F062F9044B5A681B
:2075C00022F0F00214435C6010BD00BF088901080010024010B5044680B1B0F5806F0DD06B
:2075E000B0F5A06F0AD0B0F5C06F07D0B0F5E06F04D0064840F27E2101F042F9044B5A682E
:2076000022F4E06214435C6010BD00BF088901080010024010B5044680B1B0F5806F0DD0D6
:20762000B0F5A06F0AD0B0F5C06F07D0B0F5E06F04D006484FF4267101F022F9044B5A6804
:2076400022F4605242EAC4045C6010BD088901080010024010B4284B5B6803F00C03042BCE
:2076600005D0082B06D0F3B9244B03601DE0244B03601AE0204B5A685B68C2F38342023247
:2076800013F4803F04D11F4B03FB02F202600CE0194B5B6813F4003F14BF1B4B184B03FB9E
:2076A00002F2026001E0154B0360134B5A68C2F3031216498A5CD2B2046824FA02F24260FD
:2076C0005C68C4F302240C5DE4B222FA04F484605C68C4F3C224095DC9B2CA40C2605B68E1
:2076E000C3F381330A49CB5CDBB2B2FBF3F202615DF8044B704700BF0010024000127A002C
:20770000001BB70000093D00808D5B00080000200400002038B504460D4620F4AA6323F0DF
:20772000070303B920B90C4840F22B4101F0A8F8012D04D9084840F22C4101F0A1F825B1CD
:20774000064B5A6914435C6138BD044B5A6922EA04045C6138BD00BF088901080010024089
:2077600038B504460D460E4B034003B920B90D4840F24A4101F084F8012D04D9094840F241
:207780004B4101F07DF825B1074B9A6914439C6138BD054B9A6922EA04049C6138BD00BF6B
:2077A0000200C0FF088901080010024038B504460D460E4B184200D120B90D4840F2694104
:2077C00001F05EF8012D04D9094840F26A4101F057F825B1074BDA691443DC6138BD054BA5
:2077E000DA6922EA0404DC6138BD00BF00360181088901080010024010B50446212818D05D
:20780000312816D0392814D0412812D0612810D07A280ED07B280CD07C280AD07D2808D036
:207820007E2806D07F2804D00A4840F2345101F027F86309012B02D1074B186804E0022BEA
:20784000054B0CBF186A586A04F01F04E04000F0010010BD088901080010024010B582B0F1
:207860000023019331242046FFF7C6FF019B01330193019BB3F5A06F01D00028F3D0312017
:20788000FFF7BAFF003018BF012002B010BD00BF024B5A6A42F080725A62704700100240D9
:2078A0002DE9F84305460C46464B98420BD0A3F57843984207D003F58063984203D042487E
:2078C000A32100F0DDFF238863B1B3F5806F09D0B3F5004F06D0B3F5404F03D03A48A621C9
:2078E00000F0CEFF6388B3F5827F04D01BB13648A72100F0C5FFA388B3F5006F04D01BB1BB
:207900003148A82100F0BCFFE3882BB1022B03D02D48A92100F0B4FF2389012B03D92A482B
:20792000AA2100F0ADFF6389B3F5007F04D01BB12548AB2100F0A4FFA3898BB1082B0FD0E7
:20794000102B0DD0182B0BD0202B09D0282B07D0302B05D0382B03D01B48AC2100F090FF8E
:20796000E3892BB1802B03D01748AD2100F088FF238A1BB91448AE2100F082FF2A8802F4D8
:207980004152B4F800906388B4F80480B4F806C027896689A089E18949EA030348EA0303E8
:2079A0004CEA03033B43334303430B4313432B80AB8B23F400631B041B0CAB83238A2B8284
:2079C000BDE8F883003001403889010838B504460D46124B98420CD0A3F57843984208D0AA
:2079E00003F58063984204D00D4840F2B71100F047FF012D04D90A484FF4DC7100F040FF5D
:207A00002DB123889BB243F04003238038BD238823F040031B041B0C238038BD0030014032
:207A20003889010870B504460D461646164B98420CD0A3F57843984208D003F5806398428D
:207A400004D012484FF4087100F01AFF012E04D90E4840F2212100F013FF25F003039BB2F3
:207A600003B925B9094840F2222100F009FF26B1A3889BB21D43A58070BDA388ED43ADB2F3
:207A80001D40A58070BD00BF003001403889010838B504460D46094B98420CD0A3F5784356
:207AA000984208D003F58063984204D0044840F23A2100F0E5FEA58138BD00BF0030014094
:207AC0003889010810B50446094B98420CD0A3F57843984208D003F58063984204D00548E8
:207AE00040F24A2100F0CCFEA08980B210BD00BF003001403889010838B505460C46164B22
:207B000098420CD0A3F57843984208D003F58063984204D0114840F2163100F0B1FE802C04
:207B200012D0402C10D0202C0ED0102C0CD0082C0AD0042C08D0022C06D0012C04D007486B
:207B400040F2173100F09CFE2B8904EA0300003018BF012038BD00BF003001403889010865
:207B600038B504460D46524B984242D0B0F1804F3FD0A3F5943398423BD003F5806398427A
:207B800037D003F58063984233D003F5806398422FD003F5806398422BD003F5903398422D
:207BA00027D003F5C053984223D003F5806398421FD003F5806398421BD0A3F59E3398426F
:207BC00017D003F58063984213D003F5806398420FD003F5903398420BD003F5806398426D
:207BE00007D003F58063984203D03248E72100F047FE6B885BB1102B09D0202B07D0402BCF
:207C000005D0602B03D02B48E82100F039FEEB884BB1B3F5807F06D0B3F5007F03D025483B
:207C2000E92100F02DFE23889BB2214A944212D002F5006294420ED0B4F1804F0BD0A2F511
:207C40009832944207D002F58062944203D002F58062944203D123F070036A881343164A7A
:207C6000944208D002F58062944204D023F440739BB2EA8813432380AB88A3852B8823859B
:207C80000B4B9C420FD003F500639C420BD003F540639C4207D003F580639C4203D003F5E9
:207CA00080639C4201D12B7A23860123A38238BD002C0140688901080010004038B50446B7
:207CC0000D462E4B984243D0B0F1804F40D0A3F5943398423CD003F58063984238D003F571
:207CE0008063984234D003F58063984230D003F5806398422CD003F59033984228D003F5D8
:207D0000C053984224D003F58063984220D003F5806398421CD0A3F59E33984218D003F519
:207D20008063984214D003F58063984210D003F5903398420CD003F58063984208D003F517
:207D40008063984204D00E4840F2293100F098FD012D04D90A4840F22A3100F091FD2DB1E5
:207D600023889BB243F00103238038BD238823F001031B041B0C238038BD00BF002C014070
:207D80006889010870B504460D461646314B984243D0B0F1804F40D0A3F5943398423CD09D
:207DA00003F58063984238D003F58063984234D003F58063984230D003F5806398422CD0E7
:207DC00003F59033984228D003F5C053984224D003F58063984220D003F5806398421CD0F7
:207DE000A3F59E33984218D003F58063984214D003F58063984210D003F5903398420CD0B9
:207E000003F58063984208D003F58063984204D0114840F26B3100F033FD15F47F4F00D15D
:207E200025B90D484FF45B7100F02AFD012E04D9094840F26D3100F023FD26B1A3899BB25C
:207E40001D43A58170BDA389ED43ADB21D40A58170BD00BF002C01406889010870B504466F
:207E60000E461546284B984243D0B0F1804F40D0A3F5943398423CD003F58063984238D071
:207E800003F58063984234D003F58063984230D003F5806398422CD003F59033984228D036
:207EA00003F5C053984224D003F58063984220D003F5806398421CD0A3F59E33984218D078
:207EC00003F58063984214D003F58063984210D003F5903398420CD003F58063984208D076
:207EE00003F58063984204D0084840F29B4100F0C7FC012D04D9054840F29C4100F0C0FCD5
:207F00002685A58270BD00BF002C01406889010838B504460D462A4B984243D0B0F1804FE0
:207F200040D0A3F5943398423CD003F58063984238D003F58063984234D003F580639842C1
:207F400030D003F5806398422CD003F59033984228D003F5C053984224D003F58063984255
:207F600020D003F5806398421CD0A3F59E33984218D003F58063984214D003F580639842F7
:207F800010D003F5903398420CD003F58063984208D003F58063984204D00A4840F636219B
:207FA00000F06EFC15F4614F00D125B9054840F6372100F065FCED43ADB2258238BD00BFE9
:207FC000002C01406889010838B504460D46334B984243D0B0F1804F40D0A3F5943398428C
:207FE0003CD003F58063984238D003F58063984234D003F58063984230D003F58063984295
:208000002CD003F59033984228D003F5C053984224D003F58063984220D003F580639842A4
:208020001CD0A3F59E33984218D003F58063984214D003F58063984210D003F59033984266
:208040000CD003F58063984208D003F58063984204D0134840F6582100F012FC6B1E9BB250
:20806000012B10D9042D0ED0082D0CD0102D0AD0202D08D0402D06D0802D04D0084840F645
:20808000592100F0FDFB238AA08928401D4203D0003018BF012038BD002038BD002C01406F
:2080A0006889010838B504460D462A4B984243D0B0F1804F40D0A3F5943398423CD003F51D
:2080C0008063984238D003F58063984234D003F58063984230D003F5806398422CD003F5C4
:2080E0009033984228D003F5C053984224D003F58063984220D003F5806398421CD0A3F534
:208100009E33984218D003F58063984214D003F58063984210D003F5903398420CD003F535
:208120008063984208D003F58063984204D00A4840F6822100F0A4FB15F47F4F00D125B9E1
:20814000054840F6832100F09BFBED43ADB2258238BD00BF002C01406889010830B587B005
:2081600004460D46644B984213D0A3F5744398420FD003F5806398420BD003F580639842A9
:2081800007D003F58063984203D05C48B82100F077FB2B68013B5A4A934203D95748B92104
:2081A00000F06EFBAB8833B1B3F5805F03D05348BA2100F065FBEB8863B1B3F5805F09D048
:2081C000B3F5005F06D0B3F5405F03D04B48BB2100F056FB2B894BB1B3F5806F06D0B3F533
:2081E000C06F03D04548BC2100F04AFB6B8923F00C0292B202B91BB94048BD2100F040FB65
:20820000AB8963B1B3F5807F09D0B3F5007F06D0B3F5407F03D03948BE2100F031FBAB89AF
:2082200073B1354B9C420BD0A3F574439C4207D003F580639C4203D03048C22100F020FBEB
:20824000238A23F440531B041B0CEA8813432382A28992B222F4B05222F00C02A8882B8989
:20826000698903430B431343A381A38A23F440731B041B0CAA891343A38201A8FFF7EAF991
:208280001D4B9C420CBF049A039AA3891BB2002B08DA02EB820202EB82022B685B00B2FB0F
:2082A000F3F207E002EB820202EB820229688900B2FBF1F2134BA3FB02135B091801642153
:2082C00003FB1123A18909B2002908DADB0032330C4DA5FB0323C3F34213034307E01B01C9
:2082E0003233084DA5FB0313C3F3431303439BB2238107B030BD00BF0038014098890108C5
:208300001FAA44001F85EB5170B505460C46234B98420CD0A3F57443984208D003F58063AE
:20832000984204D01E484FF4997100F0A9FA23883BB1B3F5006F04D0194840F2331100F000
:208340009FFA63883BB1B3F5806F04D014484FF49A7100F095FAA3883BB1B3F5007F04D007
:208360000F4840F2351100F08BFAE3883BB1B3F5807F04D00A484FF49B7100F081FA2B8A26
:2083800023F470631B041B0C26886288A088E188324302430A4313432B8270BD00380140D4
:2083A0009889010838B504460D46164B984214D0A3F57443984210D003F5806398420CD050
:2083C00003F58063984208D003F58063984204D00D484FF4B17100F053FA012D04D90A4833
:2083E00040F2631100F04CFA2DB1A3899BB243F40053A38138BDA38923F400531B041B0CCB
:20840000A38138BD003801409889010870B505460C461646364B984214D0A3F5744398421A
:2084200010D003F5806398420CD003F58063984208D003F58063984204D02E4840F2891173
:2084400000F01EFA282C1ED040F227739C421AD040F226639C4216D040F225539C4212D055
:2084600040F224439C420ED040F646039C420AD040F66A139C4206D0602C04D01D484FF401
:20848000C57100F0FDF9012E04D91A4840F28B1100F0F6F940F66A139C420FD1144B9D42F6
:2084A0000CD0A3F574439D4208D003F580639D4204D0104840F28F1100F0E2F9C4F342134B
:2084C00004F01F04012202FA04F4934201D10C3503E0022B0CBF103514351EB12B681C435C
:2084E0002C6070BD2B6823EA04042C6070BD00BF003801409889010838B504460D46124B19
:20850000984214D0A3F57443984210D003F5806398420CD003F58063984208D003F580639B
:20852000984204D0094840F25F2100F0A9F9B5F5007F04D305484FF4187100F0A1F9C5F39D
:208540000805A58038BD00BF003801409889010810B504460D4B984214D0A3F57443984244
:2085600010D003F5806398420CD003F58063984208D003F58063984204D005484FF41C7157
:2085800000F07EF9A088C0F3080010BD003801409889010838B505460C46264B984214D068
:2085A000A3F57443984210D003F5806398420CD003F58063984208D003F58063984204D00B
:2085C0001D4840F2863100F05BF9012C18D0802C16D0402C14D0202C12D0102C10D0B4F51F
:2085E000807F0DD0B4F5007F0AD0082C08D0042C06D0022C04D0104840F2873100F040F91E
:20860000B4F5007F0FD10B4B9D420CD0A3F574439D4208D003F580639D4204D0064840F22D
:208620008B3100F02DF92B8804EA0300003018BF012038BD003801409889010838B50546CC
:208640000C463A4B984214D0A3F57443984210D003F5806398420CD003F58063984208D05E
:2086600003F58063984204D0314840F2D93100F007F9282C25D040F227739C4221D040F2B6
:2086800026639C421DD040F225539C4219D040F224439C4215D040F646039C4211D040F645
:2086A0006A139C420DD0B4F5587F0AD0B4F5187F07D0B4F5B07F04D01D4840F2DA3100F0D3
:2086C000DFF840F66A139C420FD1184B9D420CD0A3F574439D4208D003F580639D4204D0A0
:2086E000134840F2DE3100F0CBF8C4F3421304F01F0201219140012B03D1AA8992B20A4056
:2087000005E0022B0CBF2A8AAA8A92B20A40240A012000FA04F4288880B220401AB1003088
:2087200018BF012038BD002038BD00BF003801409889010838B504460D46244B984214D01E
:20874000A3F57443984210D003F5806398420CD003F58063984208D003F58063984204D069
:208760001B4840F2224100F08BF840F226639D4210D040F225539D420CD040F646039D4251
:2087800008D040F66A139D4204D0114840F2234100F076F840F66A139D420FD10B4B9C42A8
:2087A0000CD0A3F574439C4208D003F580639C4204D0074840F2274100F062F82D0A0123BD
:2087C00003FA05F5ED43ADB2258038BD0038014098890108FEE700BF08B5034800F076F8CC
:2087E0000120FFF7F7FF00BFCC89010808B50D4B1B6813B90C4A0B4B1A600A4B1B680330BA
:2088000020F003001844094A904206D90EF0D0FC0C2303604FF0FF3008BD024A106018463C
:2088200008BD00BF900200206C4500200048002001230360014B0B60704700BF18000020DD
:2088400008B50EF0B5FC582303604FF0FF3008BD08B50EF0ADFC582303604FF0FF3008BD26
:2088600008B50EF0A5FC58230360002008BD00BF08B50EF09DFC582303604FF0FF3008BDB5
:2088800008B503460A460348194600F005F8FFF7A3FF00BF208A01080FB400B583B004AB87
:2088A00053F8042B0193084880210FF0CFFB011E03DD054800F038F80146084603B05DF8E7
:2088C00004EB04B0704700BF9802002010B504460EF04EFE0146204600F026F80248012145
:2088E00000F022F810BD00BFCC92010810B400244FF0604212E0D2F8803E13F0010F04D051
:20890000D2F8003E13F0010F01D1204609E01368002BFCD003781370013401308C42EAD3BA
:2089200008465DF8044B704708B5FFF7DFFF08BD08B500F067F808BD82B0002301930093EB
:2089400003F1804303F504331A6842F480321A601A46136803F400330093019B0133019351
:20896000009B1BB9019BB3F5A06FF2D1214B1B6813F4003F14BF012300230093009B012BC9
:2089800036D11D4B1A6842F010021A601A6822F003021A601A6842F002021A60A3F5805378
:2089A0005A685A605A685A605A6842F480625A605A6822F47C125A605A6842F4E8125A605F
:2089C0001A6842F080721A601A46136813F0007FFBD0084B5A6822F003025A605A6842F075
:2089E00002025A601A46536803F00C03082BFAD102B07047001002400020024008B5FFF7CE
:208A00009BFF08BD08B5104B1A6842F001021A6059680E4A0A405A601A6822F0847222F4F1
:208A200080321A601A6822F480221A605A6822F4FE025A604FF41F029A60FFF7DFFF4FF053
:208A40000062034B9A6008BD001002400000FFF800ED00E008B54FF4C060FDF7F5FB4FF04E
:208A600000604FF4C041FDF75BFC62B608BD00BF08B57D20FEF7C0FE08B1FEF709FF45F271
:208A80005550FEF77BFC0520FEF78AFC40F6FF70FEF796FCFEF7ACFC08BD00BF10B582B0E1
:208AA00004460C4B53F820000121FEF759FE0A4B33F81430ADF8043010238DF8073003238A
:208AC0008DF80630054B53F8240001A9FEF7BCF902B010BD788A0108888A010820000020E3
:208AE00008B50346044A52F82000044A32F81310FEF72EFB08BD00BF20000020888A010820
:208B000008B50346044A52F82000044A32F81310FEF7EEFA08BD00BF20000020888A010840
:208B200008B50346044A52F82000044A32F81310FEF782FA08BD00BF20000020888A01088C
:208B400082B0019002E0019B013B0193019B002BF9D102B0704700BF10B586B004460420E2
:208B6000FDF700FC01A8FEF775FD1048029BA0FB0320800C04FB00F00138B0F1807F09D213
:208B80000B4B5860F0210B4A82F8231000229A6007221A60064B1A6822F002021A601A4632
:208BA000136813F4803FFBD006B010BD83DE1B4310E000E000ED00E008B54FF47A7303FBDF
:208BC00000F0FFF7C9FF08BD10B5094C20464FF4DB7108F06FFD94F8B431AE2B05D194F803
:208BE000B501AE3818BF012010BD012010BD00BFD428002008B50548AE2380F8B43180F89B
:208C0000B5314FF4DB7108F061FD08BDD428002008B50548FF2380F8B43180F8B5314FF47E
:208C2000DB7108F053FD08BDD428002008B5082007F03CFF012815D1092007F037FF01281A
:208C400010D1094B1B686BB908480EF029FC08480EF026FC07480EF023FC0122024B1A60FF
:208C6000FFF7D6FF08BD00BF18030020908A0108B88A0108E48A010808B5FEF7B1FB08BD62
:208C8000002070470020704710B5BBB101280DD1012B03D1104600F023FB03E01046DAB2C5
:208CA00000F09AFB003018BF012010BD28B950025A0200F0FFFD002010BD10BD042010BD14
:208CC00010B51C46DBB101280DD1012B03D1104600F01EFB03E01046DAB200F0AFFB0030EC
:208CE00018BF012010BD48B9074B1B68012B08D15002620200F054FE002010BD10BD0420FE
:208D000010BD002010BD00BF2C13002038B5154601281FD1012918D011B1032910D032E028
:208D20001B484FF48061FEF713FA00F005FC041C18BF012416484FF48061FEF7D9F925E04F
:208D40004FF400731380002420E000F07FFA286000241BE0D0B9032917D8DFE801F0020F29
:208D6000060B00F0E7FC002410E04FF40073138000240BE001231380002407E04FF400633B
:208D80001360002402E0042400E00424204638BD000C01400C4B1A68A2F2BC720B4B1B680E
:208DA0005B0543EA42630A4A126843EA0243094A128843EAC223084A128843EA4213074A83
:208DC000108843EA40007047300000203C00002034000020440000204000002038000020BB
:208DE00000B583B04FF48063ADF8043003238DF8063010238DF80730034801A9FEF724F8B6
:208E000003B05DF804FB00BF000C014070B5064640F6FF74FF2501E0013CA4B2284600F02F
:208E2000CDFBB04201D0002CF6D1002C14BF0020FF2070BD70B50024FF264FF6FE753046AD
:208E400000F0BCFB00F01F00AC421AD001340B2807D00D2817D0052818BFFF20FF28EED021
:208E600001E00B2070BD0024FF2503E0013414F1030F0AD8284600F0A1FB0028F6D0002058
:208E800070BD012070BD0D2070BDFF2070BD00BFF8B507460C4616461F4D28464FF480614C
:208EA000FEF726F9FF2000F089FBFF2000F086FBFF2000F083FB28464FF48061FEF748F926
:208EC00047F0400000F07AFB200E00F077FBC4F3074000F073FBC4F3072000F06FFBE0B200
:208EE00000F06CFB304600F069FB0024FF2603E00134A4B2FF2C05D8304600F05FFB054687
:208F0000FF28F5D004484FF48061FEF7F1F8FF2000F054FB2846F8BD000C014070B50646D8
:208F20000C461546FF2000F049FBFF2000F046FB13484FF48061FEF70BF946F0400000F003
:208F40003DFB200E00F03AFBC4F3074000F036FBC4F3072000F032FBE0B200F02FFB284652
:208F600000F02CFB0024FF2503E00134A4B2FF2C04D8284600F022FBFF28F6D070BD00BFC9
:208F8000000C014070B5002301E001339BB2B3F5706FFAD30024FF2504E0284600F00EFBF3
:208FA0000134A4B2092CF8D9002426469525304631462A46FFF76CFF0134A4B2012801D093
:208FC000FE2CF4D9FF2C14BF0020012070BD00BFF0B587B075484FF48061FEF789F8002319
:208FE000ADF804304FF48272ADF80620ADF808300222ADF80A200124ADF80C404FF40072FB
:20900000ADF80E203822ADF81020ADF812300723ADF81430664D284601A9FEF741FC2846E9
:209020002146FEF7D3FC042000F090FAFF2000F0C5FAFFF7A7FF002840F0B1805B484FF48E
:209040008061FEF785F808204FF4D5718722FFF765FF044605284BD10222564B1A7053488C
:209060004FF48061FEF774F8FF2000F0A7FA0024372625462927304629462A46FFF708FF2D
:20908000FF2800F09180384629462A46FFF700FF0134A4B208B1FE2CEDD9FF2C11D10024F1
:2090A00001262546304629462A46FFF7F1FE0134A4B208B1FE2CF5D9FF2C72D001223D4B90
:2090C0001A70012000F042FAFF2000F077FA3B2000219522FFF7DCFE002864D110204FF466
:2090E00000719522FFF7D4FE0446002855D05BE0012852D1FF2000F061FAFF2000F05EFA91
:20910000FF2000F05BFAFF2000F058FA27484FF48061FDF7EDFFFF2000F050FA372500243E
:209120002926284621462246FFF7B2FE01283BD130464FF080412246FFF7AAFE0028F0D163
:209140003A2000210A46FFF7E9FE044630B117484FF48061FDF7CCFF204625E0FF2000F080
:209160002DFA0546FF2000F029FAFF2000F026FAFF2000F023FA0D484FF48061FDF7B8FFCC
:20918000FF2000F01BFA15F0400F14BF04220322084B1A70012000F0D9F9204604E001200E
:2091A00002E0012000E0FFE707B0F0BD000C0140003800401C0300202DE9F84305460C4690
:2091C000914619484FF48061FDF7C2FFFE20FFF71DFE804670B114484FF48061FDF788FF6D
:2091E0004FF001081CE0384600F0E8F905F8010B344600E0FF27631E9EB2002CF3D1FF2073
:2092000000F0DCF9FF2000F0D9F9B9F1010F07D105484FF48061FDF76BFFFF2000F0CEF971
:209220004046BDE8F88300BF000C014010B5044609200021FF22FFF72BFE30B92046102163
:209240000122FFF7B9FF002010BD10BD00B585B06846FFF7EBFF00283ED19DF8003003F01C
:20926000C003402B08D19DF808009DF8093003EB00200130C00430E09DF8060000F00300DB
:209280009DF8073003EB00209DF808309B0903EB80009DF8092002F003029DF80A30DB09AD
:2092A00003EB42030233012203E0520092B2013BDBB2002BF9D100FB02229DF8053003F010
:2092C0000F03012103E0490089B2013B9BB2002BF9D102FB01F000E0002005B05DF804FB7E
:2092E00010B503460C46094A1278042A18BF4302112019460022FFF7CBFD30B920464FF4E5
:2093000000710122FFF758FF10BD10BD1C03002070B503460C462E4A1278042A18BF430287
:20932000182019460022FFF7B3FD00284FD129484FF48061FDF70CFFFF2000F03FF9FF208C
:2093400000F03CF9FF2000F039F9FE2000F036F9002506E0661C207800F030F90135ADB297
:209360003446B5F5007FF5D3FF2000F027F9FF2000F024F9FF2000F021F9044600F01F03A2
:20938000052B11D013484FF48061FDF7B1FE204670BD0134A4B2B4420AD10E484FF4806131
:2093A000FDF7A6FE012070BD0024FF254FF6FF76284600F003F90028EBD006484FF4806116
:2093C000FDF796FEFF2000F0F9F8002070BD70BD1C030020000C0140F8B503460C4615465C
:2093E000144A1278042A18BF4302122019460022FFF74EFDE8B94FF40077002620463946E1
:209400003246FFF7D9FE28B904F50074681E10F0FF05F3D10C2000210A46FFF739FD064854
:209420004FF48061FDF764FEFF2000F0C7F82846F8BDF8BD1C030020000C01402DE9F04733
:2094400004460D4692463A4B1B78042B18BF4402012B04D0172011460022FFF719FD19203E
:2094600021460022FFF714FD044600285CD131484FF48061FDF76CFEFF2000F09FF8FF20FD
:2094800000F09CF84FF0FC094FF00008FF27484600F094F8444606E06E1C287800F08EF87D
:2094A0000134A4B23546B4F5007FF5D3384600F085F8384600F082F8384600F07FF80446B4
:2094C00000F01F03052B05D01A484FF48061FDF70FFE29E0FFF7AEFC0446012805D115489F
:2094E0004FF48061FDF704FE1EE00AF1FF3313F0FF0ACCD1FD2000F061F8002808BF4FF0EA
:20950000FE0AFFF797FC30B10A484FF48061FDF7EFFD012408E007484FF48061FDF7E8FD2A
:20952000FF2000F04BF854462046BDE8F08700BF1C030020000C014010B5FF24204600F034
:209540003DF8FF28FAD1002010BD00BF1A4A138823F038031B041B0C1380042824D8DFE823
:2095600000F003080F161D00134B1A8892B21A801AE0114B1A8892B242F008021A8013E0CB
:209580000D4B1A8892B242F010021A800CE00A4B1A8892B242F018021A8005E0064B1A88CA
:2095A00092B242F038021A80034B1A8892B242F040021A80704700BF00380040F8B5074637
:2095C0000024154E022504E00134A4B2B4F5C87F1DD830462946FEF78FFA0028F4D00E48E4
:2095E0003946FEF755FA00240B4E012504E00134A4B2B4F5C87F0CD830462946FEF77CFA72
:209600000028F4D00448FEF75DFAC0B2F8BD0020F8BD0020F8BD00BF0038004070B506464D
:209620000C4D022428462146FEF766FA0028F9D008483146FEF72CFA064D01242846214661
:20964000FEF75AFA0028F9D00248FEF73BFAC0B270BD00BF0038004000B583B04FF40063F8
:20966000ADF8043003238DF8063010238DF80730034801A9FDF7E8FB03B05DF804FB00BFAF
:20968000000C014008B5FFF7E7FF03484FF40061FDF72EFD08BD00BF000C014008B5002325
:2096A000034A1380034A1380FFF7ECFF08BD00BF1E0300202003002070B58AB0194E02AC8D
:2096C00035460FCD0FC495E80F0084E80F006B46324652F8200F516803C3134D28464FF427
:2096E0000061FDF735FDD720FFF798FF0020FFF795FF0446C0F3C2030AAA1A4412F8281C93
:209700000A4A11700AAA02EB830353F8202C084B1A6028464FF40061FDF7EAFC20460AB0DD
:2097200070BD00BF088B0108000C0140401300204413002008B509484FF40061FDF708FDBF
:20974000FF20FFF76BFFFFF7B7FF10F0800FFAD002484FF40061FDF7CBFC08BD000C0140CA
:2097600038B504460D461A484FF40061FDF7F0FC72B6012C15D15320FFF750FF154C20788D
:20978000C0F1100025FA00F0C0B2FFF747FF2078083805FA00F0C0B2FFF740FF0020FFF7C7
:2097A0003DFF0B4C20464FF40061FDF7A1FC20464FF40061FDF7CCFCFFF77EFF10F0800FB3
:2097C000FAD062B602484FF40061FDF791FC38BD000C01404013002038B504460D461A4897
:2097E0004FF40061FDF7B4FC72B6012C15D18320FFF714FF154C2078C0F1100025FA00F071
:20980000C0B2FFF70BFF2078083805FA00F0C0B2FFF704FF0020FFF701FF0B4C20464FF48E
:209820000061FDF765FC20464FF40061FDF790FCFFF742FF10F0800FFAD062B602484FF4B3
:209840000061FDF755FC38BD000C014040130020F8B504460F4616461D4615484FF40061A1
:20986000FDF776FC72B6012C1AD1D420FFF7D6FE0020FFF7D3FEC7F30720FFF7CFFEF8B24F
:20988000FFF7CCFE0020FFF7C9FE0024274605E03846FFF7C3FE05F8010B0134B442F7D382
:2098A00062B603484FF40061FDF722FCF8BD00BF000C01402DE9F04F83B0894601924FEAAB
:2098C000122A060AC5B208B900252E4601203146FFF746FFC5F58074019B9C4228BF1C4627
:2098E0000120294622464B46FFF7B2FF711C264600250127AB4612E001F101083846FFF7A0
:209900002FFF384659464FF4807209EB0403FFF79FFF04F5807406F5807601354146554503
:20992000EAD3019BB3420BD99E1B09D00120FFF717FF01200021324609EB0403FFF788FF04
:2099400003B0BDE8F08F00BFF8B504460F4616461D4612484FF40061FDF7FAFB72B6012C2A
:2099600015D18420FFF75AFE0020FFF757FEC7F30720FFF753FEF8B2FFF750FE002404E086
:2099800015F8010BFFF74AFE0134B442F8D362B602484FF40061FDF7ABFBF8BD000C0140D8
:2099A0002DE9F04F83B08A4601924FEA122B10B1060AC1B201E000210E46C1F58074019B66
:2099C0009C4228BF1C46012022465346FFF7BCFF01203146FFF700FF0136274600254FF0F8
:2099E000010813E0404600214FF480720AEB0403FFF7AAFF06F1010940463146FFF7ECFE16
:209A000004F5807407F5807701354E465D45E9D3019BBB420BD9DA1B09D0012000210AEBBC
:209A20000403FFF791FF01203146FFF7D5FE03B0BDE8F08F30B4002303E08C4208BF2A7048
:209A40000133C518C45C002CF7D130BC704700BF03463038C0B2092812D9A3F16102D2B2C5
:209A6000052A03D8A3F15700C0B27047A3F14102D2B2052A03D8A3F13700C0B27047184611
:209A8000704700BF2DE9F04106460024254611E073555BB2252B0BD1B7187878FFF7D8FFB0
:209AA0008046B878FFF7D4FF00EB081070550234013501342246335D002BE9D17355BDE834
:209AC000F08100BF30B585B00446012918D0022918D0032918D0042918D0052918D009295C
:209AE00018D00A2918D00C2918D00B2918D0082918D00D2918D00E29184D18BF002514E067
:209B0000174D12E0174D10E0174D0EE0174D0CE0174D0AE0174D08E0174D06E0174D04E0CD
:209B2000174D02E0174D00E0174D01A817490DF0CFFC204629460DF013FD204601A90DF077
:209B4000EBFC20460DF014FD02462118104B1868A0501B790B7105B030BD00BF208E010836
:209B6000348B0108888B0108C48B0108008C01083C8C01088C8C0108E08C01081C8D0108FB
:209B8000608D0108A88D0108E48D0108608E0108E0B50108F8B505460C4608464D490DF057
:209BA0002AFD20B920464C490DF025FD10B101232B70F8BD204649490DF01DFD10B1022361
:209BC0002B70F8BD204646490DF015FD20B9204644490DF010FD10B103232B70F8BD2046BE
:209BE00041490DF008FD20B9204640490DF003FD10B104232B70F8BD20463D490DF0FBFCFC
:209C000010B105232B70F8BD20463A490DF0F3FC064628B9204638490DF0EDFC074610B12E
:209C200008232B70F8BD204634490DF0E4FC20B9204633490DF0DFFC10B10C232B70F8BD16
:209C4000204630490DF0D7FC20B920462E490DF0D2FC10B10B232B70F8BD07B916B10823E3
:209C60002B70F8BD204629490DF0C5FC20B9204627490DF0C0FC10B109232B70F8BD2046F3
:209C800024490DF0B8FC20B9204623490DF0B3FC10B10A232B70F8BD204620490DF0ABFC9E
:209CA00020B920461E490DF0A6FC10B10D232B70F8BD20461B490DF09EFC20B920461A491B
:209CC0000DF099FC10B10E232B70F8BD00232B70F8BD00BF648E0108989001086C8E01084F
:209CE000748E01087C8E0108848E01088C8E0108948E010818B001089C8E0108A48E01089E
:209D0000AC8E0108B48E0108B88E0108BC8E0108C48E0108CC8E0108D48E0108DC8E010877
:209D2000E48E0108EC8E0108F48E010838B50546084624490DF078FC044610B900232B7065
:209D400038BD21490DF002FC20B120461F490DF0FDFB38B901232B7000201A490DF064FC85
:209D6000044625E020461A490DF0F0FB20B1204618490DF0EBFB38B902232B70002011493D
:209D80000DF052FC044613E0204613490DF0DEFB20B1204611490DF0D9FB38B900201049D7
:209DA0000DF042FC044603232B7001E000232B7014B900232B7038BDA81C21460DF0D0FB4B
:209DC00038BD00BFDC8C0108FC8E0108008F0108048F01080C8F0108148F01081C8F010893
:209DE000308B010810B5ADF5B76D014670B168460DF0B6FB684607490DF016FC04460649AA
:209E00000DF0A4FB00B10134204600E000200DF5B76D10BD248F0108288F010870B504467C
:209E20000E46002305E003FB06F50134FFF710FE2B18207808B12028F5D198B270BD00BFBC
:209E40002DE9F04188B003460E46684619460DF087FB68460024104D0A274FF0100816E0AD
:209E600029460DF0E1FB0378302B08D14378782B05D102304146FFF7D1FFC0B203E0394664
:209E8000FFF7CCFFC0B230550134E4B20020032CE6D908B0BDE8F0812C8F0108F8B50F469D
:209EA00015461E460DF0A7FB044638460DF060FB0444204629460DF09EFB001B85B23046A9
:209EC00021462A460DF072FB00237355F8BD00BF70B584B00C46002301930293ADF80C300A
:209EE000054600283FD000293FD02249224A01ABFFF7D4FF01A80A21FFF790FF0646284649
:209F00001E490DF078FB04300023835521460DF072FB054658B320460DF02AFB01302C1817
:209F2000204626210DF005FB034618B920460DF01FFB2318181B83B28BB11A46104D002321
:209F40005355284621460DF031FB2846FFF79AFD28462B212022FFF76DFD284608E008485E
:209F60000023037004E0002002E0002000E0002004B070BD308F01087C920108E0B50108E7
:209F800048130020704700BF704700BF014B185C704700BF340300200023074906E0CA5C4E
:209FA000824201D1D8B204E00133DBB2072BF6D9FF2040B2704700BF3403002010B54001F7
:209FC00000F584742046082101F0CEFF204601F0ADFF0028FAD1012010BD00BF30B583B08C
:209FE00005460C46009208460549064A0DF070FA82B22846214602F0ADFA03B030BD00BFDE
:20A0000058900108A88D010838B505461C46B3F5C87F0FD0B3F5CA7F13D0C82B19D1A1F166
:20A020000803DBB2012B13D9104B186849B2FFF749FD0EE00D4B18680D4976220DF0FBF8BA
:20A0400007E00A4B18680B4999220DF0F4F800E000244CB1054B1C6820460DF089FA82B25D
:20A060002846214602F076FA38BD00BF28030020448F0108BC8F01082DE9F04383B0804638
:20A080000F46164699460A9DFFF786FF0446B0F1FF3F7CD000EBC0023E4B03EB0212D2F897
:20A0A0008820C2B9B5F5006F3CD300EBC00003EB0010C0F88490C0F88850451C2846002160
:20A0C00080220DF0C1F8284639460DF049FA002740F2FF7529E000EBC0032E4901EB0313FE
:20A0E000D3F88C50551BB5F5006F26BF002740F2FF75012700EBC001264B03EB01112648CB
:20A100000131012205F054F9244B187060B904EBC403204A02EB03131F48D3F88C1005F0B2
:20A12000EFFB02E0002700E000251B4831462A460DF1060305F0F0F9184B187018B96B1CB5
:20A140000022F25400E000252DB140463146AAB202F000FA00E0012767B10E4AE1000819F5
:20A1600002EB00100023C0F88430C0F88830C0F88C3009E0074BE200111903EB0111D1F85F
:20A180008C301D44C1F88C50034805F0A9FB03B0BDE8F0833C030020501B0020741F0020C1
:20A1A0002DE9F0418CB005460C4600230B9303930493059306930793089309930A93FFF7FC
:20A1C000EBFEB0F1FF3F00F0C980664B1A68664B1A602378032B00F2BA80DFE803F0020A65
:20A1E0000A7F284600210A464FF4C873FFF70CFFB4E0A01CFFF7F6FD06465C490DF0A6F9B2
:20A2000038B95B4B03CB306071601A889B783281B372304657490DF099F930B9564B07CBEA
:20A2200030607160B2601B783373304653490DF08DF938B9524F0FCF30607160B260F360A7
:20A240003B883382601C3146FFF7A4FC6378082B1CD130464B4B19680BAA00F097F968B127
:20A260000B9B40F2BE72934208D828463E4A1168444A12689BB2FFF7B1FE6FE028460821D2
:20A2800000224FF4CA73FFF7BFFE67E03E483146012205F08DF83D4B187030B93A4BDA68C8
:20A2A0000B92D3F81080012201E000229046002A14BFC8274FF4CA77284661780B9A3B46CD
:20A2C000FFF7A2FEC82F49D1274B1A680B9B0093284631464346FFF7CFFE3FE0A01C234932
:20A2E0002B4A03ABFFF7DAFD601C03A9FFF752FC6378082B23D103A821461B4B1A680BAB50
:20A3000000F0A0F9044690B10B9B40F2BE7293420DD828461B4A1168134A12689BB2FFF701
:20A320005DFE022C1AD11B4B1B68984716E02846082100224FF4CA73FFF766FE0EE02846FC
:20A3400000210A464FF4CA73FFF75EFE06E0284600210A464FF4C873FFF756FE0CB0BDE8CC
:20A36000F08100BF4C1B002028030020288F010864900108709001087490010884900108EB
:20A380008C900108481B0020501B0020741F0020A09001084C00002010B40023054C03E017
:20A3A000CA5CE2540133DBB28342F9D35DF8044B704700BF3403002010B5044C206004489D
:20A3C000016010461946FFF7E7FF10BD481B00204C1B002008B1034A106009B1024B1960BE
:20A3E000704700BF4C0000204800002070B582B006465B4B1A685B4B1A605B4B1A685B4B5A
:20A400001A60FFF7C3FD04464501083505F5407001F08CFD1338092800F29680DFE800F0E0
:20A42000909A9A9A05949494948C05F50075284601F07CFD10F0010F03D02846012101F032
:20A4400093FD06EBC6031B01494AD35C032B46D0042B5BD0002B7DD1204601F02BFE82B209
:20A4600013B2002B76DDB3F5006F20463D4B1968C8BF4FF4006202F00DF985B215F4004F60
:20A4800068D1384B186808F0C7FA30B106EBC60633010421364AD1545CE0324B19682DB212
:20A4A00000234B55314D2868FFF740FC20462968FFF776FE06EBC6032D4A02EB0313D3F839
:20A4C00088302BB106EBC60633010321D15441E006EBC60633010421254AD1543AE0254B59
:20A4E0001A680023009320461946FFF7C5FD06EBC6031F4A02EB0313D3F8883053BB06EBFF
:20A50000C606360104221A4B9A5523E01849F000821901EB02120023C2F88830C2F88C30C4
:20A52000C2F88430304400010B54134B1B6898472046FFF743FD0DE02046FFF73FFD09E00F
:20A54000204601F015FF05E0204601215022002301F082FE084B1B68984702B070BD00BFCA
:20A560004C1B00202C030020481B0020300300203C0300202803002048000020024B1A684E
:20A5800001321A60704700BF24030020F0B583B004460F46164602AA002522F8025D07F03D
:20A5A00087FF00283BD1204621490CF0CFFF30B938460DF1060107F01FF9012032E0204633
:20A5C0001C490CF0C3FF30B938460DF1060107F06FFA012026E0204617490CF0B7FF30B904
:20A5E00038460DF1060107F017FB01201AE0204612490CF0ABFF30B938460DF1060107F0EA
:20A60000F7FB01200EE020460D490CF09FFF40B938460DF1060107F0C3FB012002E001208E
:20A6200000E0002010B1BDF80630336003B0F0BDA8900108B4900108BC900108CC90010833
:20A64000E0900108F0B583B0054617461E4602AB002423F8024D8C1C214608F055F90028E5
:20A660005AD1284631490CF071FF58B9204607F0CFFB014605203A460DF1060307F07EFDBE
:20A6800002204CE028462A490CF060FF58B9204607F086FC0246384626490CF019FF0120D6
:20A6A000ADF806003BE0284623490CF04FFF58B9204607F0BDFC024638461E490CF008FF59
:20A6C0000120ADF806002AE028461C490CF03EFF58B9204607F0E4FC0246384615490CF02A
:20A6E000F7FE0120ADF8060019E0284614490CF02DFF20B9204607F013FD01200FE02846E9
:20A7000010490CF023FF48B9204607F01FFD0023ADF80630022002E0012000E0002010B164
:20A72000BDF80630336003B0F0BD00BFE8900108F4900108289C010800910108109101085D
:20A74000209101083491010838B50E4A0023D3701D2111710121917105780B4C25704578BC
:20A7600065708578A570C078E07048F6B8040748048007480088A2F86B000220152201F077
:20A780006BFD38BD801F0020781F00207C1F0020288F010810B59AB001AC074B0FCB84E817
:20A7A0000F00022021460F2201F0D4FE0120034BD8701AB010BD00BF50910108801F002057
:20A7C0002DE9F843814600241F4FDFF888801F4E12E02CB9484641460CF026FF054604E047
:20A7E000002039460CF020FF054628460A210CF0DBFC3055FDB10134032CEADD0025144B06
:20A800001D80DFF850802F461C460FE0384641460CF00AFF064623881B0223800A210CF046
:20A82000C3FC2388184420804EB10135012DEDDD0020BDE8F8834FF0FF30BDE8F8834FF078
:20A84000FF30BDE8F88300BF64910108DC240020E02400206091010870B5B6B0064604468D
:20A860008D490BE05AB20D6815446A7802F00302012A5BB208BF203304F8013B23785DB230
:20A88000202D0ED0002BEDD1844D0BE020460CF06FFE0246204631460CF072FE28B1043576
:20A8A00000E07E4D2C68002CF0D15CB904A87C4932460CF00DFE82B2022004A901F04AFE2B
:20A8C0000020EFE2774BDB78E3B9744BEB1A9B10022B17D0082B15D0A3B104AC724D0FCD9C
:20A8E0000FC40FCD0FC495E8030044F8040B24F8021B090C2170022004A9262201F02AFEFC
:20A900000020CFE220460CF033FE341800E0013494F90030202BFAD0604BED1AAD101C2DE8
:20A9200000F2B182DFE815F01D009E023E004B006901EC017E02AF02A500CE00F8002D01BF
:20A94000BB02880188015E025E029E029E029E029E0279019E029E0299009401B3015901F2
:20A96000F80020460CF004FE421E0023A354023823544E4821460CF0F3FD04AC4C4D0FCD42
:20A980000FC495E8070003C42270022004A9182201F0E0FD041E80F28482022001F026FC61
:20A9A000E0B27FE220460CF0E3FD421E0023A354023823542046FFF7EDFE012072E2204615
:20A9C0000CF0D6FD421E0023A3540238235494F90030413B282B34D8DFE803F0152433338C
:20A9E000333333332433333333333333333333333333333333333333333333331524333333
:20AA00003333333324000022264B9A7004A8294922460CF05DFD82B2022004A901F09AFD42
:20AA200001203FE201251F4B9D7004A8214922460CF04EFD82B2022004A901F08BFD284688
:20AA400030E204A81C4922460CF042FD82B2022004A901F07FFD012024E204A817497522F6
:20AA60000CF0E9FB022004A9742201F073FD012018E2134B04AC0FCB07C424F8023B1B0CE2
:20AA80002370022004A90E2201F064FD022001F019FD012006E200BF20020020500000202F
:20AAA00068910108801F002084910108871F0020AC910108C8910108E0910108F89101083D
:20AAC0007092010820460CF053FD421E0023A35402382354A4480CF04BFD012805D1A34874
:20AAE000A34922460CF0F4FC06E0A04A1046A149643A23460CF0ECFC9C4C04A89E49224638
:20AB00000CF0E6FC82B2022004A901F023FD092304F8CB3C0120C5E120460CF029FD421E65
:20AB20000023A354023823548F480CF021FD012805D18E488E4922460CF0CAFC06E08B4AC8
:20AB400010468C49643A23460CF0C2FC874C04A88A4922460CF0BCFC82B2022004A901F0A7
:20AB6000F9FC0A2304F8CB3C03208549854B1A8801F036FC012840F095810022824B1A7042
:20AB800090E12046FFF71CFEB0F1FF3F0FD104AC7E4D0FCD0FC495E8030044F8040B218079
:20ABA000022004A9152201F0D5FC01207AE1784B01269E715E7104AC764D0FCD0FC495E8EA
:20ABC0000F0007C424F8023B1B0C2370022004A91E2201F0BFFC304664E1634C04A86E4900
:20ABE00022460CF075FC82B2022004A901F0B2FC1B2304F8673C012054E15B4C04A86649A9
:20AC000022460CF065FC82B2022004A901F0A2FC042304F8673C012044E104AC5F4D0FCD99
:20AC20000FC495E80F0007C42380022004A91D2201F090FC012035E104A859494A4A0CF0A7
:20AC400047FC82B2022004A901F084FC012029E154490A784B788D78CC7853490988080AA8
:20AC6000C9B2009501940290039104A84F490CF02FFC82B2022004A901F06CFC032001F02E
:20AC800021FC434B00229A71012058710AE120460CF06EFC421E0023A354821EA3540328FF
:20ACA0001DDD20462F210CF093FC0146002301F8013B204605F02EF8021E05DD04A83C4906
:20ACC0000CF006FC024614E004AC3A4D0FCD0FC495E8030044F8040B2170142209E004AC29
:20ACE000344D0FCD0FC495E8030044F8040B21701422022004A992B201F02CFC0120D1E094
:20AD000020460CF035FC421E0023A354821EA354032855DD03381E46235420462F210CF06A
:20AD200057FC0546014601F8016B204604F0F2FF2F232B70024678B904A81D490CF0C8FB47
:20AD4000094D284621460CF00BFC04A81A492A460CF0BEFB02463EE004A8184922460CF0BA
:20AD6000B7FB024637E000BFEB1F00204F20002080920108849201088C920108D09201087E
:20AD8000DC240020E0240020BD07002010930108801F002028930108489301088493010858
:20ADA000A4930108781F00207C1F0020C8930108F8930108049401081C94010850940108A2
:20ADC0003A4D284621460CF0CBFB04A838492A460CF07EFB0246022004A992B201F0BAFB42
:20ADE00001205FE020460CF0C3FB421E0023A35402382354204605F0A1F830B104A82D49B1
:20AE000022460CF065FB024605E004A82A4922460CF05EFB0246022004A992B201F09AFB84
:20AE200001203FE020460CF0A3FB421E0023A35402382354204605F025F830B104A81F493A
:20AE400022460CF045FB024605E004A81C4922460CF03EFB0246022004A992B201F07AFBB2
:20AE600001201FE004AC174D0FCD0FC40FCD0FC495E8030084E80300022004A9272201F048
:20AE800069FB01200EE004A80F4922460CF020FB82B2022004A901F05DFB012002E001204C
:20AEA00000E0012040B236B070BD00BFEB1F00201C940108689401088C940108B09401086F
:20AEC000D0940108E4940108689101082DE9F04182B005460023ADF806304FF4527001F0CA
:20AEE00025F81C287ED8DFE800F0657D7D7D7D7D7D7D7D7D7D7D7D7D7D7D7D7D7D737D7D48
:20AF00007D0F7D7D7D7D5E00964B1B78DBB9964B1A88964B1A8028469549964A964B0CF044
:20AF2000D7FA28460CF024FB82B20220294601F011FB041E04DA022001F058F9E4B2D8E142
:20AF40000122884B1A70022001F0B4F80446ADF80600002846D0284600214FF400720CF03F
:20AF600073F9B4F5007F84BF40F2FF13ADF8063002202946BDF8062001F08CFB044600238A
:20AF80002B54BDF80630834209D0002800F0AA81002804DA022001F029F9E4B2A9E128469D
:20AFA000FFF75AFC1EE0022001F08CFA012819D0C4B29EE1022001211522002301F04CF9D3
:20AFC000044602280ED0022001F010F9E4B290E1022001F0CDF9012801D0C4B289E1002227
:20AFE000604B1A704FF45A7000F0A0FF04461C2800F27A81DFE810F02801780178017801AA
:20B000007801780178017801780178017801780178017801780178017801780178015E01BA
:20B020007801780178011D0078017801780178012101524B1B7813B90122504B1A70504BA3
:20B040001B79043B172B00F25181DFE813F018004F014F014F014F013D009F004F014F0179
:20B060004F014F014F014F014F014F014F014F014F014F014F014F014F014F0118003B4CD1
:20B08000204629460DF1060204F05AFD28460CF06FFA82B2ADF806200320294601F05AFAE1
:20B0A0001D2304F8673C032001F00CFA2846354922460CF00DFA82B2ADF8062002202946B0
:20B0C00001F048FA002414E12F4C2046A4F16501012204F06DF984F8240468BBA4F59A735E
:20B0E000D3F840414FF4007603F59A77A7F59A78FDF7C2FD2846002132460CF0A5F8B4F598
:20B10000007F94BFA2B232463846294601AB04F003FA88F8580548B903202946BDF80420BE
:20B1200001F018FABDF80430E41AE1D1164C204604F0D6FB84F82404114C1D2323710320EE
:20B1400001F0C0F928460F4904F1CF020CF0C0F982B2ADF806200220294601F0FBF900246B
:20B16000C7E000BFBC070020288F0108EB1F00200C9501082C95010834950108BD07002072
:20B18000801F002038950108B42000205B4C2046A4F165010A2204F00BF984F8240400282E
:20B1A00036D12746A4F59A78032000F083FF044610B34FF40076FDF75FFD284600213246BE
:20B1C0000CF042F8B4F5007F94BFA2B232460320294601F05FFA02463846294601AB04F041
:20B1E00055FA88F85805BDF80430E41A08B9002CE1D10028D8D005E04FF45A7000F096FE57
:20B200001728D1D03D4C204604F06AFB84F824043B4C1D232371032001F054F928463949B6
:20B2200004F1CF020CF054F982B2ADF806200220294601F08FF900245BE0032001F042F948
:20B24000012855D0C4B254E02D4B5B79012B50D12B4B9B79E3B9032001212B4B1A880023B7
:20B2600000F0FAFF0546032804D0032000F0BEFFECB23EE0244A138801339BB213804CF2B4
:20B280005032934212D948F6B8021F4B1A800DE0032001211422002300F0DEFF05460328A2
:20B2A00004D0032000F0A2FFECB222E00222144B5A711EE0124B9B7933B9032001F058F859
:20B2C00001280BD0C4B214E003201049104B1A8801F086F8012801D0C4B20AE000240D4B42
:20B2E0001C7006E0002404E0002402E0002400E00024204602B0BDE8F08100BFB4200020C5
:20B30000801F0020389501087C1F0020DC240020E0240020BD07002008B54FF47060084994
:20B32000042200F073FE4FF4A0600649042200F06DFE4FF480700449042200F067FE08BDB3
:20B34000D0070020C0070020CC07002008B50020802100F009FE002000F0E8FDFFF7DCFFE1
:20B360004FF410600249062200F050FE08BD00BFE424002008B50020802100F0F5FD00203D
:20B3800000F0D4FD4FF410600249062200F03EFE08BD00BFE424002010B40B4C0B4B1C6001
:20B3A0000B4C0C4B1C600C4C0C4B1C60034608B10648036009B1074B19600AB1074B1A6079
:20B3C0005DF8044B704700BF19B30008D00000204DB30008CC00002075B30008D400002077
:20B3E00010B582B04FF410606946062200F0DCFD32490A68012313700A6853700A6806239F
:20B40000937008680022C27009682D480068040E0C71C0F307444C71C0F307248C71C871B9
:20B420000A8180208872CA720A734A738A73CA730A744A748A74CA740A754A758A75CA7543
:20B440000A764A768A76CA761E4A107808775078487790788877D078C877107981F82000C6
:20B46000527981F82120002003E0CA1810770133DBB20F2BF9D90023184604E0CA1882F84D
:20B480002C000133DBB23F2BF8D90023184604E0CA1882F86C000133DBB213F0800FF7D03D
:20B4A000632381F8EC30822281F8ED20532281F8EE2081F8EF3002B010BD00BFF42400203D
:20B4C000EC240020E4240020F0B585B0FFF788FF504B1968352381F8F030012381F8F130F2
:20B4E00081F8F2303D2281F8F320072281F8F42081F8F530484B1A7881F8F6205A7881F873
:20B50000F7209A7881F8F82093F803E081F8F9E01F7981F8FA705E7981F8FB600C2381F8E3
:20B52000FC30002381F8FD3012223C4807E0541CC55C0A4482F8EC5001339BB2A2B2C45CED
:20B54000002CF4D1541CA4B20A4482F8ECE0601C80B20C4484F8EC70421C92B2084480F864
:20B56000EC60D51A0D44033385F8E830531C9BB20A44372082F8EC00581C80B20B44062290
:20B5800083F8EC20431C9BB20844012480F8EC40181980B20B44032483F8EC40431C9BB237
:20B5A000084480F8EC205A1C92B20B440F2083F8EC00531C9BB20A443A2082F8EC005A1CDC
:20B5C00092B20B443B2083F8EC00531C9BB20A44FF2082F8EC00002004E0CA1882F8EC003B
:20B5E00001339BB2B3F59C7FF7D3FF238DF80C308DF80D308DF80E308DF80F30084B18782E
:20B60000432300934FF4097203AB01F0BBF805B0F0BD00BFF4240020E4240020DC000020A4
:20B62000F8240020F0B585B0FFF7DAFE7E4B1B78033BDBB2012B1BD87C4B1B6800229A7268
:20B64000DA727B4A117819735178597391789973D278DA73774B1A788DF80C205A788DF827
:20B660000D209A788DF80E20DB788DF80F3008E0FF238DF80C308DF80D308DF80E308DF8EC
:20B680000F306A4B1968352381F8F030012381F8F130032281F8F2203D2281F8F3200722C2
:20B6A00081F8F42081F8F530634B1A7881F8F6205A7881F8F7209A7881F8F82093F803E01D
:20B6C00081F8F9E01F7981F8FA705E7981F8FB609DF80F30FF2B26D1322381F8FC300422DD
:20B6E00081F8FD20524B187881F8FE00587881F8FF00987881F80001DB7881F801313623E7
:20B7000081F8023181F803214A4B1A7881F804215A7881F805219A7881F80621DB7881F82C
:20B7200007311C2200E010228B180C2083F8EC00501C02320844002380F8EC303F4D05E037
:20B74000541C0A4482F8EC000133A2B2E85C0028F6D1541CA4B20A4482F8ECE0601C80B202
:20B760000C4484F8EC70421C92B2084480F8EC60D01A0844033380F8E830531C9BB20A44E9
:20B78000372082F8EC005A1C92B20B44082083F8EC00531C9BB20A44012082F8EC001A1891
:20B7A00092B20B44032083F8EC00531C9BB20A44062082F8EC005A1C92B20B440F2083F823
:20B7C000EC00531C9BB20A443A2082F8EC005A1C92B20B443B2083F8EC00531C9BB20A44DE
:20B7E0001F2082F8EC005A1C92B20B44212083F8EC00531C0A44FF2082F8EC009BB2002044
:20B8000003E0CA1882F8EC000133B3F59C7FF8DB0B4B1878432300934FF4097203AB00F0F8
:20B82000B1FF05B0F0BD00BFBE070020F4240020D0070020F0240020E4240020DC000020CB
:20B84000F824002000B585B0FFF7CAFD374B196800238B72CB72352381F8F030012381F817
:20B86000F130042281F8F2203D2081F8F300072081F8F40081F8F5302D4B187881F8F60084
:20B88000587881F8F700987881F8F800D87881F8F900187981F8FA005B7981F8FB30322354
:20B8A00081F8FC3081F8FD20224B187881F8FE00587881F8FF00987881F80001DB7881F83B
:20B8C0000131362381F8023181F803211A4B1A7881F804215A7881F805219A7881F80621DC
:20B8E000DB7881F80731FF2381F808311D23002003E0CA1882F8EC000133B3F59C7FF8DB1B
:20B90000FF238DF80C308DF80D308DF80E308DF80F300A4B1878432300934FF4097203ABB1
:20B9200000F030FF05B05DF804FB00BFF4240020E4240020D0070020F0240020F824002059
:20B940002DE9F04387B0684B187800F0B3FB0246002800F0B780644B1878644B19680DF182
:20B960000E03009304AB00F0B1FFBDF80E30432B40F0A5805D4B1B68197F5D4A1278914257
:20B9800040F0A280597F5A4A5278914240F09E80997F574A9278914240F09A80D97F544A18
:20B9A000D278914240F0968093F82010504A1279914240F0918093F821104D4A527991423F
:20B9C00040F08C8080B203F1F00103440020494F494E9846DFF82CC1484D494C6CE00A78E4
:20B9E000062A34D005D8012A13D06AB1032A1AD05DE0352A0AD002D8332A3CD057E0362AA6
:20BA00004BD0FF2A57D052E0013155E08878033152E08A782A70CA786A700A79AA704A79A4
:20BA2000EA70063148E04A7891F8029084F8009091F8039084F8019091F8049084F8029010
:20BA400091F8059084F803901144023134E04A7891F8029087F8009091F8039087F8019005
:20BA600091F8049087F8029091F8059087F803901144023120E08A78CCF8002091F80390DE
:20BA800009EB022291F8049009EB02294A7902EB0922CCF8002006310EE08A783270CA7888
:20BAA00072700A79B2704A79F270063104E08A1C4978114400E04146994290D300E000205E
:20BAC000C0B20CE000200AE0002008E0002006E0002004E0002002E0002000E0002040B2D8
:20BAE00007B0BDE8F08300BFF8240020F4240020E4240020D4070020F0240020C007002006
:20BB0000CC070020D800002030B583B04FF4D85000F00CFA05464FF4D850032100F024FAD9
:20BB2000104B187841F2883300930F4911220F4B00F028FE04464FF4D850294600F014FA7C
:20BB400014F10D0F0AD0FFF77DFE094B19681A4613685B1A012BFBD9002000E0012003B080
:20BB600030BD00BFF824002038960108D0070020C40700200023044A13600521034A11605C
:20BB8000034A1370704700BFC4070020C8000020D807002010B5214B93F90030012B23DC75
:20BBA0001F4B1A681F4B1B689A4234D21E4B93F90030022B06D0042B07D0012B07D1FFF7A2
:20BBC00083FC04E0FFF72EFD01E0FFF72BFD154B00221A601A680532114B1A600F4B1A786B
:20BBE00001321A70012417E00F4B93F90030022B07D0042B05D0012B09D100240A4B1C7043
:20BC000006E0FFF761FC0124074B1C7000E00124FFF7B0FF00E00124204610BDD807002007
:20BC2000C8000020C4070020BE07002010B5654B93F90030062B00F0C280634B1878400139
:20BC400000F5427000F072F9222806D05E4B187802214422002300F0FFFAFFF771FEC0B21D
:20BC6000584B93F90030042B00F2A280DFE803F0030F274A6A00554B00221A705A709A705B
:20BC8000DA70FFF721FC01244E4B1C7095E0022811D14F4B1A68117C4C4B1970517C59701D
:20BCA000917C9970D27CDA70FFF7BCFC0222454B1A70012481E0FFF76DFF04467DE005282E
:20BCC00016D1FFF721FF48B1424B1B689847FFF751FF03223B4B1A7001246EE0FFF74AFF52
:20BCE0003D4B1B6898470022364B1A70012464E0062803D10124334B1C705EE0FFF74AFF16
:20BD000004465AE0354B1B68B3F1FF3F52D0344A1268B2EB530F4FD92C4A1178314B197075
:20BD20005178597091789970D278DA702E4B1A6801321A60FFF776FCFFF71CFF0424214B16
:20BD40001C703AE0052826D10022284B1A70254B1A781E4B1B789A4211D1224B5A781B4B99
:20BD60005B789A420BD11F4B9A78184B9B789A4205D11C4BDA78154BDB789A4204D01C4B11
:20BD80001B689847032400E00424FFF7F3FE03220C4B1A7011E0062806D1FFF7EBFE01222D
:20BDA000084B1A70042408E0FFF7F4FE044604E0012402E0042400E00424204610BD0520F1
:20BDC00010BD00BFBE070020F8240020D0070020F4240020D0000020D4000020D8000020AB
:20BDE000C4070020C8070020EC240020D8070020CC000020F0B583B006460D4600238DF82F
:20BE000004308DF805308DF806308DF80730224C4FF410602146062200F0C6F894F800E0F3
:20BE20006378A778E078217962794EEA03033B4303430B4313430ED1002222700821617008
:20BE4000DC21A170E270227162714FF410602146062200F0DBF8114B1E70114B1D60114AF9
:20BE6000114B1A604FF4706001A9042200F0CEF84FF4706001A9042200F0C8F84FF480708D
:20BE800001A9042200F0C2F8FFF774FE0022074B1A7003B0F0BD00BFE4240020F82400203F
:20BEA000F424002078563412EC240020BE070020024B1A6801321A60704700BFC407002044
:20BEC000044B1A7802705A7842709A788270DB78C3707047D0070020044B1A7802705A782E
:20BEE00042709A788270DB78C3707047CC070020044B1A7802705A7842709A788270DB782E
:20BF0000C3707047C0070020044B1A7802705A7842709A788270DB78C3707047D40700203D
:20BF2000014B1868704700BFD800002038B505460C4CA368984723699847E369C5F3074097
:20BF40009847E369C5F307209847E369E8B29847A3699847054663699847E36898472846BA
:20BF600038BD00BFE8000020F8B505460E460D4CA36898472369984745F00407E369C5F3C7
:20BF800007409847E369C5F307209847E369F8B29847E3693046984763699847E368984726
:20BFA000F8BD00BFE8000020F8B507460E461546154CA368984723699847E369C7F3074059
:20BFC0009847E369C7F307209847E369F8B29847236A43B1626A6AB907E0BB6998473055C2
:20BFE0000134A4B203E0002400E00024064FAC42F3D302E0304629469847034C6369984702
:20C00000E3689847F8BD00BFE80000202DE9F04107460E461546154CA36898472369984781
:20C0200047F00408E369C7F307409847E369C7F307209847E3695FFA88F09847636A5BB9A8
:20C0400005E0FB69305D98470134A4B201E00024064FAC42F5D302E0304629469847034C9B
:20C0600063699847E3689847BDE8F081E8000020F8B50025400100F1080606F5005706F56E
:20C0800004563846FFF752FF000284B23046FFF74DFF204484B24CB13846FFF747FF00023E
:20C0A00085B23046FFF742FF284485B2A542E8D12846F8BDF8B50025400100F1080606F529
:20C0C000185706F51C563846FFF730FF000284B23046FFF72BFF204484B24CB13846FFF708
:20C0E00025FF000285B23046FFF720FF284485B2A542E8D12846F8BD2DE9F8430D461446F4
:20C1000032B34FEA800909F10106F60006F510573846FFF70BFF804606F514563046FFF70A
:20C1200005FF00EB08201FFA80F809F10200C00000EB082029462246FFF768FF4444A4B276
:20C140003846210AFFF710FF3046E1B2FFF70CFFBDE8F8832DE9F8430D46144632B34FEAEB
:20C16000800909F10106F60006F520573846FFF7DDFE804606F524563046FFF7D7FE00EB17
:20C1800008201FFA80F809F10300C00000EB082029462246FFF708FF4444A4B23846210ABB
:20C1A000FFF7E2FE3046E1B2FFF7DEFEBDE8F883F8B50F46400100F1080505F52056304687
:20C1C000FFF7B4FE044605F524552846FFF7AEFE00EB0420C419A4B23046210AFFF7C4FE4F
:20C1E0002846E1B2FFF7C0FEF8BD00BF70B50546082827D84601083606F58074204610216C
:20C20000FFF7B2FE2046FFF791FE0028FAD106F500701F21FFF7A8FE0122AA400B4B19884F
:20C2200021EA02021A800023094A22F81530094A535506F540742046FFF778FE0028FAD111
:20C24000012000E0FF2040B270BD00BFDC070020E8070020E00700202DE9F04105460F46E0
:20C2600014461E4608286BD800296BD0022901D9042967D116F0060F66D1A6B1012F02D014
:20C28000022F04D00FE016F0210F0CD15EE016F0200F02D016F0800F5AD016F0100F02D09C
:20C2A00016F0800F56D02846FFF7A0FF4FEA451808F1080826F00F0140463943FFF754FEB1
:20C2C00064B9264A1488631C9BB213804FF6F072934203D14FF44042204B1A8008F58060DF
:20C2E000210AFFF741FE08F5A060E1B2FFF73CFE08F5807420460121FFF736FE2046FFF71F
:20C3000015FE0028FAD106F00106AE40144B1A8816431E800122AA40124B198821EA02021A
:20C320001A800023104A22F81530104A535508F540742046FFF7FAFD0028FAD0E8B20AE00B
:20C34000FF2008E0FB2006E0FA2004E0FA2002E0FA2000E0FA2040B2BDE8F081E4000020BB
:20C36000DA070020DC070020E8070020E007002070B5064608282BD8440108342046FFF722
:20C38000D5FD00F00F00012824D104F540752846FFF7CCFD13281FD104F580742046022132
:20C3A000FFF7E2FD2046FFF7C1FD0028FAD108E02046FFF7BBFD20B93046FFF717FFFC2028
:20C3C0000BE02846FFF7B2FD1428F1D1012004E0FF2002E0FB2000E0FD2040B270BD00BF65
:20C3E0002DE9F04107460D46904608285AD8440108342046FFF79AFD00F00F00012853D15E
:20C4000004F540763046FFF791FD13284ED12A786B7803EB0223AA7802EB0323EA7802EBFD
:20C420000323013B13F1030F42D8B8F1000F41D004F5406029460422FFF7E8FD04F58050CF
:20C440004FEA1821FFF790FD04F588505FFA88F1FFF78AFD04F5807528460421FFF784FDCF
:20C460002846FFF763FD0028FAD1154B1B8843FA07F717F0010F0CD01EE02046FFF756FD27
:20C4800010F0080F07D020460821FFF76DFDF32013E004F500743046FFF748FD1728ECD19F
:20C4A00001200AE0FF2008E0FB2006E0FD2004E0F42002E0F52000E0002040B2BDE8F08155
:20C4C000DA07002070B50646082837D8450108352846FFF72BFD00F00F00012830D105F579
:20C4E000807420460821FFF73FFD2046FFF71EFD0028FAD10122B240144B198821EA0202F9
:20C500001A80134B1B88334113F0010F0BD019E02846FFF70BFD10F0080F08D03046FFF75E
:20C5200065FEF3200FE005F5407405F500752046FFF7FCFC0028EBD1012004E0FF2002E03B
:20C54000FB2000E0002040B270BD00BFDC070020DA0700202DE9F84F06468B4614460828DA
:20C560007DD880464FEA401A0AF1080A5046FFF7DDFC00F00F00012875D1002C77D00AF5BB
:20C5800040773846FFF7D2FC172801D01C2872D13E4B1B88334113F0010F1DD00AF50075F7
:20C5A0002846FFF7C3FC10F0100F0BD028461021FFF7DAFC0121B140344B1A8822EA0102B0
:20C5C0001A8009E010F0080F59D03046FFF70EFE6FF00C00BDE8F88F0AF5F850FFF7A6FCAA
:20C5E000850205F47C45A54228BF2546DFF8A0903046FFF73DFD04463846FFF797FC172884
:20C6000008D01C2806D03046FFF7F0FD6FF00600BDE8F88FB9F8003043FA08F313F0010F12
:20C6200001D0A5422ED8A542E2D8304659462A46FFF762FD0AF5807A50462021FFF794FC6B
:20C640005046FFF773FC0028FAD1012303FA06F60E4B1A8816431E802846BDE8F88F4FF004
:20C66000FF30BDE8F88F6FF00400BDE8F88F6FF00D00BDE8F88F6FF00600BDE8F88F002087
:20C68000BDE8F88F0020BDE8F88F00BFDC070020DA0700202DE9F04F83B0054601911446A0
:20C6A000082860D880464FEA401B0BF1080B5846FFF73CFC00F00F00012857D1002C58D039
:20C6C0000BF5F050FFF732FC800200F47C43A34228BF234600930BF540770BF5F85ADFF819
:20C6E000A0902846FFF7E6FC04463846FFF71EFC172818D01C2810D1FCB92846FFF7B8FCD3
:20C7000006465046FFF712FCB6EB802F0BD12846FFF76CFD6FF006002FE02846FFF766FDFF
:20C720006FF0060029E0B9F8003043FA08F313F0010F00D004B3002CD3D0009B9C4228BFA9
:20C740001C46284601992246FFF704FD0BF5807B58464021FFF708FC5846FFF7E7FB00287E
:20C76000FAD1204609E04FF0FF3006E06FF0040003E06FF00D0000E0002003B0BDE8F08FC2
:20C78000DA0700202DE9F84F06468B4691461D46BDF82840082878D880464FEA401A0AF1F3
:20C7A000080A5046FFF7C2FB00F00F00022801D004286ED1B9F1000F6FD02B68002B70D0C3
:20C7C000002C72D00AF540773846FFF7AFFB422801D022286DD10AF5406029460422FFF72A
:20C7E00015FC0AF58050210AFFF7BEFB0AF58850E1B2FFF7B9FB0AF5F850FFF797FB850215
:20C8000005F47C454D4528BF4D46DFF8BC903046FFF72EFC04463846FFF788FB00284CD014
:20C82000B9F8003043FA08F313F0010F01D0AC4247D3AC42EBD3304659462A46FFF75CFC74
:20C840000AF5807420462021FFF78EFB2046FFF76DFB0028FAD10AF5007A5046FFF766FBA2
:20C8600010F0100F06D050461021FFF77DFB2846BDE8F88F10F0080FEFD050460821FFF769
:20C8800073FB6FF00C00BDE8F88F4FF0FF30BDE8F88F6FF00400BDE8F88F6FF00D00BDE859
:20C8A000F88F6FF00B00BDE8F88F6FF00A00BDE8F88F6FF00600BDE8F88F6FF00300BDE82E
:20C8C000F88F0020BDE8F88FDA0700202DE9F04F85B00546009193460193082800F2D88037
:20C8E00006464FEA401909F108094846FFF71EFB824600F00F03022B02D0042B40F0CB803F
:20C90000BBF1000F00F0CA80694B33F81530CBB909F54077DFF8A0812846FFF7CBFB044659
:20C920003846FFF703FB002800F0BB80B8F80030334113F0010F02D0002C00F0B580002C7C
:20C94000EAD000E0002400225A4B5A550AF0070ABAF1020F03D0BAF1040F41D077E0544B44
:20C9600033F8153083BB284602A90822FFF7F2FB09F5807420464021FFF7F6FA2046FFF7E8
:20C98000D5FA0028FAD19DF80830019A13709DF8093053709DF80A3093709DF80B30D37074
:20C9A0009DF80C209DF80D3003EB02220E9B1A809DF80E209DF80F3003EB02223C4B23F844
:20C9C000152080223B4B5A55394B33F815405C4528BF5C46284600992246FFF7BBFB3DE0E5
:20C9E000334B33F8153033BB284602A90222FFF7B1FB09F5807420464021FFF7B5FA2046B8
:20CA0000FFF794FA0028FAD19DF808209DF8093003EB02239BB2264A22F8153040F2EA5277
:20CA2000934205D92846FFF7E1FB6FF47A703CE08022204B5A551E4B33F815405C4528BF6D
:20CA40005C46284600992246FFF784FB06E028462146FFF7ADFB164B23F8154009F580792F
:20CA600048464021FFF780FA4846FFF75FFA0028FAD10F4A32F815301B1B9BB222F81530DD
:20CA800023B10C4B5A5D42F001025A5520460CE04FF0FF3009E06FF0040006E06FF00D0072
:20CAA00003E06FF0030000E0002005B0BDE8F08FE8070020E0070020DA07002070B50446D2
:20CAC0001546082800F28D800C2900F28C80DFE801F0071019222F388A48585D626A7C0059
:20CAE00040010830FFF722FA20F00F00287001207EE0400100F5B0500830FFF717FA287068
:20CB0000012075E0400100F5A8500830FFF70EFA287001206CE04401083404F59050FFF7E6
:20CB200005FA04F59850FFF701FA287001205FE0400100F6084011460422FFF735FA0120EA
:20CB400056E04401083404F58050FFF7EFF9064604F58850FFF7EAF900EB062028800120A7
:20CB600046E0440108342046FFF7E0F900F00F0001283AD104F53C50FFF7D8F92880012091
:20CB800036E0FFF775FA2880012031E0FFF792FA288001202CE0400100F54270FFF7C6F94C
:20CBA0002870012024E040010830FFF7BFF9012805D12046FFF77EFA2880012018E00D4BA5
:20CBC00033F814302B80012012E040010830FFF7ADF900F00F00012809D1074B1B5D2B70AC
:20CBE00006E0FF2004E0FE2002E0FB2000E0FB2040B270BDE8070020E0070020704700BF8B
:20CC0000704700BF704700BF704700BF007870470170704700207047704700BF704700BF98
:20CC2000704700BF00B129B9044B054A1A61054A5A617047014B186159617047E8000020D3
:20CC400005CC000809CC0008094A138803F400739BB2002BF9D000B129B9054B054A9A6158
:20CC6000054ADA617047024B9861D961704700BFE800002015CC000819CC0008094A1388B1
:20CC800003F400739BB2002BF9D000B129B9054B054A1A62054A5A627047024B18625962F7
:20CCA000704700BFE80000201DCC000821CC000800B587B04FF4106001A90622FFF774F93C
:20CCC0004FF4807005A90422FFF76EF94FF4A06004A90422FFF768F94FF4706003A904229E
:20CCE000FFF762F900208021FFF73EF90020FFF71DF94FF4106001A90622FFF787F94FF48B
:20CD0000807005A90422FFF781F94FF4A06004A90422FFF77BF94FF4706003A90422FFF784
:20CD200075F907B05DF804FB70B506460D46FFF7BFFF3EB91DE059B2715C0A44D2B2013330
:20CD4000DBB201E00022134659B20729F3DD52B2102A31DC002409E063B2580100F5F850DC
:20CD60000830F15CFFF700F90134E4B263B2072BF2DD00201DB306E059B2695C0A44D2B2E6
:20CD80000133DBB201E00022134659B20729F3DD52B2102A12DC002409E063B2580100F5CF
:20CDA000F0500830E95CFFF7DFF80134E4B263B2072BF2DD002002E0FF2000E0FF2040B2F6
:20CDC00070BD00BF10B50146040A4FF4A85001F0F001FFF7C9F84FF4B8502146FFF7C4F815
:20CDE00010BD00BF10B54FF4A850FFF79FF800F0F0044FF4B850FFF799F8000280B20444E8
:20CE0000A0B210BD10B50146040A4FF4B050C9B2FFF7AAF84FF4C0502146FFF7A5F810BD69
:20CE200010B54FF4B050FFF781F804464FF4C050FFF77CF804EB002080B210BD08B54FF466
:20CE40003850FFF773F800F0010008BD08B54FF43850FFF76BF800F03000003018BF01200A
:20CE600008BD00BF08B54FF43850FFF75FF800F07F014FF43850FFF777F84FF43850FFF7F8
:20CE800055F860F07F014FF43850C9B2FFF76CF808BD00BF08B50378012B14BF0021402198
:20CEA0004378012B03D141F03801C9B20FE0C378012B07D18378012B0CBF41F0180141F037
:20CEC000080104E08378012B08BF41F010014FF43850FFF749F8FFF7C5FF08BD10B50446A5
:20CEE0004FF43850FFF722F8C0F38013237000F03803202B01D0382B02D10122627001E02B
:20CF000000226270182B03D0202B01D0102B02D10122A27001E00022A270182B03D0202B32
:20CF200001D0082B02D10123E37010BD0023E37010BD00BF10B504464FF43850FEF7F6FF10
:20CF400010F0400F1CD000F0C701012C0CBF41F0300141F038014FF43850FFF705F8FFF766
:20CF600081FF4FF43850FEF7E1FF012C0CBF00F0300000F03800002814BF0020FF2000E037
:20CF8000FF2040B210BD00BF30B583B00C460023009301930F2809D8DFE800F00A0E1D1824
:20CFA00022272C394755595E7763676FFF2071E0FFF77EFE00206DE019B1009101F1080418
:20CFC000019400980199FFF7AFFE63E00888FFF7F9FE00205EE0FFF705FF2080002059E0D6
:20CFE0000888FFF70FFF002054E0FFF719FF208000204FE009884FF49850090AFEF7B4FFD5
:20D000004FF4A0502178FEF7AFFF002042E04FF49850FEF78BFF05464FF4A050FEF786FFBD
:20D0200000EB05202080002034E01C4B9A780A70DA784A701A798A705A79CA709B790B71E3
:20D040000020487126E0FFF70DFF002022E00846FFF720FF00201DE00846FFF73FFF0020AB
:20D0600018E00878FFF766FF14E0FFF7EFFEC0B2FF280CD0207000200CE0FFF7DFFEC0B2B0
:20D08000FF2806D02070002004E0002002E0FF2000E0FF2040B203B030BD00BFE800002086
:20D0A00010B504464FF4106021460622FEF7AEFF4FF4807004F10E010422FEF7A7FF4FF442
:20D0C000A06004F10A010422FEF7A0FF4FF47060A11D0422FEF79AFFA27C064B1A70E27CBA
:20D0E0005A70227D9A70627DDA70A27D024B1A7010BD00BFFC070020F807002010B50446C1
:20D100004FF4106021460622FEF74EFF4FF4807004F10E010422FEF747FF4FF4A06004F1BB
:20D120000A010422FEF740FF4FF47060A11D0422FEF73AFF064B1A78A2745A78E2749A7832
:20D140002275DB786375034B1B78A37510BD00BFFC070020F807002010B5044630F03A03DA
:20D160000AD10020FEF7E2FE40EA04010020C9B2FEF7FAFE002000E0FF2040B210BD00BF8B
:20D1800008B50020FEF7D2FE08BD00BF10B504464FF4D8502178FEF7E7FE61884FF4C85038
:20D1A000090AFEF7E1FE4FF4D050A178FEF7DCFE10BD00BF38B504464FF4D850FEF7B6FE66
:20D1C00020704FF4C850FEF7B1FE05464FF4D050FEF7ACFE00EB0520608038BD10B50C4677
:20D1E000052821D8DFE800F003080D11161B0846FFF756FF002018E00846FFF77FFF002065
:20D2000013E00878FFF7A8FF0FE0FFF7B9FF207000200AE00846FFF7B9FF002005E0084678
:20D22000FFF7C8FF002000E0FF2040B210BD00BF03463038C0B2092812D9A3F16102D2B2DA
:20D24000052A03D8A3F15700C0B27047A3F14102D2B2052A03D8A3F13700C0B270471846F9
:20D26000704700BF70B504460E46002305E003FB06F50134FFF7DCFF2B18207808B1202892
:20D28000F5D198B270BD00BF30B400231D4603E08A4208BF25700133C418C25C002AF7D1FD
:20D2A00030BC704730B4084C9DF808502570074C20600748016007490A80074A13600122CD
:20D2C000064B1A7030BC7047202500201C25002004250020222500200025002010080020DD
:20D2E00082B002AB03E90300009B044A1360BDF804201344024A136002B070470C2500205B
:20D300002825002010B5094B1C68094B1B689C4209D220460AF02CF9C0B2421C2244034B6A
:20D320001A60204610BD002010BD00BF0C2500202825002010B50446194B1878FEF7BAFE26
:20D34000002829D0164B1878164B19680522FFF7A1F9052822D1134B1A68117821701A6886
:20D36000527862801868807842EA002262801868C378A380007943EA0023100A40EA02224A
:20D3800092B26280180A40EA03239BB2A380064809F0FAFF012010BD002010BD002010BD7D
:20D3A00020250020002500204C960108074B188850B9074A138801339BB2138013B90122EE
:20D3C000034B1A80024B1888704700BFFC24002012080020014B1868704700BF24250020DD
:20D3E0002DE9F84F83460F4690461E460B9D484B1878400100F54270FEF798FD172804D028
:20D4000044480AF04DF8BDE8F88F17B9FFF7CEFF0746390A41EA072189B21FFA86FA1FFAB2
:20D4200085F973190AEB0900C3F3072242EA002292B2394C206880F800B02068417020687D
:20D44000090A81702168CA702168120A0A71334859463A4609F098FF2D4B18782168052203
:20D46000FFF778F80746BBF1000F4BD0EEB13C2009F0A2FF00244FF0200B0AE018F8040002
:20D4800010B109F099FF02E0584609F095FF0134A4B2B442F2D322480AF002F81C4B187892
:20D4A00041465246FFF756F80744EDB13C2009F083FF00244FF020080AE00A9B185D10B1F9
:20D4C00009F07AFF02E0404609F076FF0134A4B2AC42F2D3124809F0E3FF0D4B18780A9906
:20D4E0004A46FFF737F8074405367219BA4209D00C48394609F048FF054B1878FEF7E2FFC8
:20D50000BDE8F88FFFF766FF074B1860BDE8F88F202500205C960108002500206C960108DE
:20D5200024B601087C960108102500202DE9F04389B00290ADF80C100023049305930693D8
:20D54000079302AB93E80300FFF7CAFEFFF7DAFE0546002800F0EB80764909F0F7FF38B90D
:20D560000021009101911420734A4523FFF738FFFFF7C8FE0446002800F0D9800A21FFF749
:20D5800071FEC6B228466D4909F0E0FFB0B9304600F084FB034604A86949324609F098FFAB
:20D5A000044604A82021FFF76FFE002100910191142004AAA3B2FFF713FFB8E0284661499E
:20D5C00009F0C4FFB0B9304600F080FB034604A85D49324609F07CFF044604A82021FFF791
:20D5E00053FE002100910191142004AAA3B2FFF7F7FE9CE02846554909F0A8FFC8B954482F
:20D6000009F04EFF304600F093FB034604A85149324609F05DFF044604A82021FFF734FE15
:20D62000002100910191142004AAA3B2FFF7D8FE7DE02846484909F089FF60B9474809F025
:20D640002FFFFFF75FFE04460A21FFF70BFE0146304600F077FB2846414909F077FF002827
:20D6600033D039E0FFF74EFE0446394609F06EFF20B93046002100F03DFB1DE0204641469B
:20D6800009F064FF20B12046494609F05FFF20B93046012100F02EFB0EE02046314909F0C0
:20D6A00055FF20B93046022100F024FB04E02E483146224609F068FEFFF724FE044658B192
:20D6C0000A21FFF7CFFDC6B204E0284FDFF8AC80DFF8AC90002CC5D1FFF714FE044630B37D
:20D6E0002846234909F032FF78B920460A21FFF7B9FDC4B23046012100F0FCFA3046211C11
:20D7000018BF012100F0CEFA11E02846194909F01DFF40B920460A21FFF7A4FDC1B2304678
:20D7200000F0DEFA03E01448294609F02DFE09B0BDE8F0838C9601081001002094960108EF
:20D7400098960108A4960108A8960108B4960108B8960108E0960108EC960108F0960108C5
:20D7600018970108289701082C9701081C970108489701084C97010850970108209701081D
:20D780002497010870B584B002A8FFF7D3FD002875D09DF80810142965D8DFE801F00B6441
:20D7A000646464641464646464646464641E646464641E00BDF80C30052B5CD1314B18787F
:20D7C000FEF780FE5BE0BDF80A100022009201921046C823FFF704FE4DE0BDF80C40FF2CF3
:20D7E00009D929482146FF2209F0CEFD254B1878FEF768FE43E0234B1878244B19682246B6
:20D80000FEF748FF844203D0214809F049FE36E0BDF80C301D4A12680024D4543E2009F0FF
:20D82000CBFD1A4D20260AE02B68185D10B109F0C3FD02E0304609F0BFFD0134A4B2BDF8BA
:20D840000C30A342F0D8134809F02AFEBDF80A30114C23800D4B1868BDF80C10FFF766FE71
:20D860000023238007E00D4809F08EFD054B1878FEF728FE03E0FFF7ADFD094B186004B024
:20D8800070BD00BF2025002068970108002500209097010824B60108FC240020A497010853
:20D8A0001825002010B5044648B10C4B1B6883B9FFF790FD2044094B1860002010BDFFF757
:20D8C00089FD064B1B68984205D30020034B186010BD002010BD012010BD00BF0C080020BB
:20D8E0002DE9F04184B0FFF775FD04460020FFF7D9FF8046002840F09980504B1B78CBB924
:20D90000FFF754FD06464E4B18804E4B1D68284609F02EFE03460022009201920220314669
:20D920002A46FFF75DFD0122444B1A70FFF752FD454B1860FFF74EFD434B1B6803F59C5365
:20D940000833984208D202A8FFF7F4FC002870D000223A4B1A7005E00123ADF80C300022A3
:20D96000364B1A709DF808305BB9BDF80A20344B1B889A4205D1BDF80C30C82B43D00B2BDB
:20D9800041D0BDF80C10012903D1304809F088FD30E0092903D12E4809F082FD2AE02D482E
:20D9A00009F0F2FCFF228DF808200024ADF80A40ADF80C40284B19680A701A68BDF80A10EF
:20D9C00051701A68BDF80A1091701A68BDF80C10D1701B68BDF80C201A71204F1E4E0525AC
:20D9E00006E0387831682A46FEF7B4FD0134E4B2092CF6D9194B1878FEF764FD41F28830DE
:20DA0000FFF750FF16E0FFF7E5FC154B1860154D2860154B1860154809F042FD29681448D8
:20DA2000091B09F0B1FC4FF0010803E04FF0000800E08046404604B0BDE8F0810808002084
:20DA4000000800201C25002004080020C0970108CC970108E097010800250020202500201B
:20DA6000102500201825002014250020FC9701080498010870B586B0764B1B78002B00F090
:20DA8000E680754B1878400100F54270FEF74EFA1C2800F2DC80DFE810F0AE00DA00DA00F0
:20DAA000DA00DA00DA00DA00DA00DA00DA00DA00DA00DA00DA00DA00DA00DA00DA00DA00C6
:20DAC000C300DA00DA00DA001D00DA00DA00DA00DA00A500604B1878400100F50270FEF7F3
:20DAE00025FA10F0010F30D05B4C2078400100F502700121FEF738FA2078400100F60840B0
:20DB000005A90422FEF750FA2078400100F580500830FEF70BFA05462078400100F5885031
:20DB20000830FEF703FA00EB052085B29DF814209DF815309DF816609DF8170021780096EB
:20DB400001900295454809F01FFC454B1B786BB9FFF7C6FE434B1870002878D00122404BC7
:20DB60001A7041483C4B197809F00EFC3D4B1B780BB1FFF707FEFFF72DFC04463B4B196835
:20DB8000431A43F6A40293420CD9394809F0FCFB0023334A1370334A13702F4B1878FEF7FC
:20DBA00091FC54E042F21072934206D8314B1A68821A42F210739A4249D92F4B1A68A21A34
:20DBC00040F2DC539A4242D92C4809F069FC002300930193062019461A46FFF701FC264B88
:20DBE0001C6034E01C4C2648217809F0CDFB2078FEF768FC2BE00023194A1370194A13707A
:20DC0000154C20781F490A88551C0D800121FEF723FB217888421AD11B4809F0B5FB16E08E
:20DC20000D4E1A48317809F0AFFB194D2868017842788378C0780090164C208801901648F6
:20DC400009F0A2FB307829682288FEF7C9FB06B070BD00BF1008002020250020189801089A
:20DC6000140800200908002044980108182500206C98010810250020142500209098010809
:20DC80009C98010858010020B8980108D498010804250020222500203098010808B502F0D0
:20DCA00005FF08BD08B5084B03449974012902D102F0D0FE02E009B902F0E2FE02484FF477
:20DCC000DB7103F003FD08BDD428002008B50E2886BF0E38C0B2002003F086FD08BD00BF1A
:20DCE00008B503460A460248194609F04DFB08BDF098010808B521B90C4B034401229A702C
:20DD00000CE0022904D1094B034401229A7005E0012903D1054B034402229A7002F070FE47
:20DD200002484FF4DB7103F0D1FC08BDD428002010B504460248214609F026FB204610BD5C
:20DD40002099010808B503460A460248194609F01BFB08BD3899010810B586B004F05EFE09
:20DD600004460DF10600FEF7ABF80DF10E00FEF7B3F80DF10A00FEF7BBF80DF11200FEF75C
:20DD8000C3F8684604F12101062204F0F3FE04F127000DF10601042204F0F0FE04F12B00AD
:20DDA0000DF10E01042204F0E9FE04F12F000DF10A01042204F0E2FE04F14F000DF11201D9
:20DDC000042204F0DBFE94F84D301BB102238DF8163002E001238DF8163000206946FFF7F5
:20DDE000FDF906B010BD00BF704700BF04E00A7802701A4601310130531E002AF7D17047C0
:20DE0000C9B202E001701A460130531E002AF9D1704700BF70B40346002001E02946334672
:20DE2000541E32B15E1C18784D1C0B782246C01AF4D070BC704700BF00E00130037813B19F
:20DE40005AB28A42F9D158B2704700BFCA7E8B7E43EA02230278032A05D1487D0A7D42EA08
:20DE6000002243EA02431846704700BF8176C1F30723C376090C0175090A4175704700BF62
:20DE8000F0B40C7804F03F04013C04EB440304EB830401260023154F4FF6FF7CFA5C551C05
:20DEA0004D5D8A5C42EA052236B1FE2C14D820F814201646013401E062450FD101330C2BD2
:20DEC000ECD90B7813F0400F0AD0FE2C0AD8002320F81430012006E0002004E0002002E036
:20DEE000012000E00020F0BC704700BF449A01082DE9F0014B730F23CB7200240C738C761F
:20DF0000CC76531E03EB430603EB860623464FF6FF77DFF84480BB421CBF30F81630013661
:20DF200018F804504B550135C3F3072C01F805C0002B08BF3B4601340C2CECD94FF6FF74A3
:20DF4000A34202D030F816300BB942F040020A70BDE8F001704700BF449A0108F0B583B01F
:20DF6000064617461C460B22FFF740FF052C13D816E0023711460CE003F0010505EB440475
:20DF80005B0814F4803F1CBF84F4883484F0210401310F29F0D900E000223B88002BE8D1D3
:20DFA000072100E0114604F00F0202F13003392B88BF02F137034A1E02A8084400F8083C65
:20DFC0002409EFD17E2002AB134403F8080C0023881E07E07F31C9B27D2902D8984206D098
:20DFE00001330133934202D2F15C2029F2D12024591C3344072A05D802A8104410F8080C5F
:20E00000013200E0204618700B460729F0D903B0F0BD00BF0B220023D90141EA5303017872
:20E020000B4403F0FF030130013AF5D11846704710B4046824B94FF0FF3323E0013200E0C1
:20E0400022461378D9B21F2902D959B23A29F5D15BB23A2B15D1611C94F90030303B092BBA
:20E0600006D8914207D1012B08D80132026009E04FF0FF3306E04FF0FF3303E04FF0FF3371
:20E0800000E0002318465DF8044B70472DE9F0410446037913B3C56A00F130074078394663
:20E0A0002A460123FAF70CFED8B900232371236AEA1AA3699A4217D2E6784FF0010808E099
:20E0C000A2691544607839462A464346FAF7F8FD013E012EF4D80020BDE8F0810020BDE871
:20E0E000F0810120BDE8F0810020BDE8F08100BF70B504460D46C36A8B4212D0FFF7C6FF2A
:20E10000064678B9607804F130012A460123FAF7BBFD002818BF012618BF4FF0FF35E56290
:20E1200000E00026304670BD10B50446002303714FF0FF33C362FFF7DBFF58BB94F82F223A
:20E1400094F82E3243EA022212B2154B9A4223D194F8692094F868301B0443EA026394F818
:20E16000672043EA022294F866301A4322F07F420C4B9A4212D094F884301B0494F88300F2
:20E1800094F8822043EA002313430648181A18BF012010BD032010BD022010BD002010BD9A
:20E1A00055AAFFFF4641540008B588B103688BB1197889B1D988828891420FD15878FAF740
:20E1C00061FD00F0010000280CBF0020032008BD092008BD092008BD092008BD092008BD3D
:20E1E0002DE9F04184B005461746002303600846FFF71EFF061EC0F29781894B53F82640A2
:20E20000002C00F093812C60237883B16078FAF739FD10F0010F0AD1002F00F0898100F070
:20E220000400C0B2002814BF0A2000209FE1002323707C4B13F816006070FAF721FD10F026
:20E24000010F40F077811FB110F0040F40F0748120460021FFF768FF012822D0002844D142
:20E26000704B03EB46035B78EBB900273EE004EB031292F8F21102F5F77251B1D07A917AA8
:20E28000090441EA0061507A41EA0021127A114300E0294604A800EB830242F8101C0133EA
:20E2A00003E0002300E000230025032BDFD95D4B03EB46035D7805B1013D4FF00208594BB5
:20E2C00003EB460604AA02EB850353F8107C27B120463946FFF728FF00E0404673782BB9FB
:20E2E00020B10135032DEDD900E00027032800F02581002840F0248194F83C2094F83B307D
:20E3000043EA02231BB2B3F5007F40F01B8194F8472094F8463053EA02230DD194F85720B3
:20E3200094F856301B0443EA026394F8552043EA022294F854301343A36194F84020E27020
:20E34000511EC9B2012900F2FF8003FB02FC94F83D00A070002800F0F980421E104240F0F0
:20E36000F78094F8421094F8412042EA0121218111F00F0F40F0EE8094F8445094F843209F
:20E3800052EA05250DD194F8535094F85220120442EA056294F8515042EA052594F85020E4
:20E3A000154394F83F8094F83E2052EA082800F0D38008EB0C0606EB1116B542C0F0CE800F
:20E3C000AD1BB5FBF0F0002800F0CA8040F6F575A8428CBF022501254FF6F572904288BF9C
:20E3E0000325821C6261E76107EB080020623E44A662032D18D1002940F0B48094F85F00B5
:20E4000094F85E10090441EA006194F85D0041EA002094F85C1001436162920012E000BFF3
:20E420001C0A00205C010020002900F09D8060446062022D0FBF520002EB420102F0010209
:20E4400002EB510202F2FF12B3EB522FC0F08E804FF0FF332361E36080236371032D5AD190
:20E4600094F8612094F8603043EA02231BB2012B51D12046791CFFF73BFE00284BD1002375
:20E48000637194F82F2294F82E3243EA022212B2384B9A423FD194F8332094F832301B046F
:20E4A00043EA026394F8312043EA022294F830301A43314B9A422ED194F8172294F8163263
:20E4C0001B0443EA026394F8152243EA022294F814321A43294B9A421DD194F81B2294F8B5
:20E4E0001A321B0443EA026394F8192243EA022294F818321343236194F81F2294F81E32AE
:20E500001B0443EA026394F81D2243EA022294F81C321343E3602570194A138801339BB2A7
:20E520001380E380002022E00B2020E00C201EE000201CE003201AE00A2018E0012016E0FC
:20E540000D2014E00D2012E00D2010E00D200EE00D200CE00D200AE00D2008E00D2006E0EB
:20E560000D2004E00D2002E00D2000E00D2004B0BDE8F08155AAFFFF5252614172724161AE
:20E58000180900202DE9F0410F4601F109040369002B3FD0456900234FF02E0C21E05A1C38
:20E5A000EB5C5EB2202E1BD0052E08BFE523092A04BF84F800C00134D9B2A1F14106F6B256
:20E5C000192E0BD895F80C80092A34BF0826102618EA060F1CBF01F12003DBB22370013412
:20E5E00013460A2BDBD9EB7A3B72EA7FAB7F1B0443EA02636A7F43EA02232A7F13433B60AE
:20E600006A7E2B7E43EA0223BB80EA7DAB7D43EA0223FB8000232370BD6975B303690BB352
:20E62000FB690BB3028C4FF6FF739A421ED0C3690024A04611E0414602F0AEF80346B8B1B1
:20E64000FF2803D9C0F307222A550134FA69013AA2420FD92B55334601349E1C188800280D
:20E66000E9D108E0002406E0002404E0002402E0002400E0002400232B55BDE8F08100BF40
:20E680002DE9F04F83B000908B460D6800E001352B785AB22F2AFAD05C2AF8D00099D1F884
:20E6A0001C80002426464FF00109DFF850A2731CA85780B21F2837D92F2835D05C2833D022
:20E6C000FE2C00F20C81C0B200F17F02D2B27D2A15D85E1CEB5CA3F14102D2B2192A0AD953
:20E6E000A3F16102D2B2192A05D903F17F02D2B27D2A00F2F68003EB002080B200E01E46F2
:20E70000494602F049F80746002800F0EC807F2806D850463946FFF78FFB002840F0E5808F
:20E7200028F814700134C2E72B44CBF800301F288CBF002604266FF0004207E0A31838F8A0
:20E740001330202B01D02E2B02D1013C002CF5D1002C00F0CC80002528F81450009A90695B
:20E7600020210B22FFF74CFB2B4600E0013338F81320202AFAD02E2AF8D023B146F00306BF
:20E7800001E0013C01E06FF0004154B1621838F812202E2AF5D14FF008094FF0000AD34629
:20E7A00004E04FF008094FF0000AD34601945F1C38F81350002D67D0202D03D02E2D05D16B
:20E7C000A74203D046F003063B46F0E7CA4501D2A74215D1B9F10B0F02D146F0030653E02C
:20E7E000A74218BF46F00306A7424DD84FEA8B0B5FFA8BFB019B4FF00B094FF0080AD6E761
:20E800007F2D08D9284601F0E3FF002101F0C4FF054646F00206FF2D11D909F1FF335345F2
:20E8200004D846F003063B46CA46C0E7009B9A690AF10103C5F3072102F80A101DE025B121
:20E840002D482946FFF7F8FA20B146F0030653465F2512E0A5F141039BB2192B03D84BF04C
:20E86000020B534609E0A5F161039BB2192B9EBF4BF0010B203DADB2534600998A6903F105
:20E88000010AD5543B4692E7009A93691A78E52A04BF05221A70B9F1080F04BF4FEA8B0B4C
:20E8A0005FFA8BFB0BF00C030C2B03D00BF00302032A01D146F0020616F0020F0AD10BF03B
:20E8C000030BBBF1010F08BF46F01006042B08BF46F0080600998B69DE72002008E0062016
:20E8E00006E0062004E0062002E0062000E0062003B0BDE8F08F00BF7C990108709901082E
:20E900002DE9F84F82460D460F7827F04007013F07EB470307EB830701260024DFF874808C
:20E920004FF6FF7918F804305A1CA85CEB5C43EA002076B101F04CFF0646FE2F1BD807F101
:20E94000010B3AF8170001F043FFB04216D15F4601E0484515D101340C2CE3D92B7813F08E
:20E96000400F11D09EB13AF81700D0F1010038BF0020BDE8F88F0020BDE8F88F0020BDE8B9
:20E98000F88F0020BDE8F88F0120BDE8F88F0120BDE8F88F449A010870B50546FFF776FB4C
:20E9A0000446002855D12B78032B4AD16B79012B47D105F13006304600214FF40072FFF73D
:20E9C0001FFA552385F82E32AA2385F82F32522385F8303085F83130612385F83230412228
:20E9E00085F83320722185F8141285F8151285F8162285F817322B6985F81832C3F30722B8
:20EA000085F81922C3F3074285F81A221B0E85F81B32EB6885F81C32C3F3072285F81D22DA
:20EA2000C3F3074285F81E221B0E85F81F32EA690132EA62687831460123FAF741F9002388
:20EA40006B71687800210A46FAF760F9002818BF0124204670BD00BF02394369023B8B42D8
:20EA600083BF8278836A01FB02300020704700BFF8B505460C4601295AD943698B4259D957
:20EA80000378022B28D0032B37D0012B54D101EB5106016A01EB5621FFF72AFB00284DD1DE
:20EAA000771CC6F308062E4496F83060296A284601EB5721FFF71CFB002842D1C7F30807F6
:20EAC0003D4495F8300046EA002014F0010F14BF0009C0F30B00F8BD016A01EB1421FFF7C3
:20EAE00007FB88BB640004F4FF742B1993F8310093F8303043EA0020F8BD016A01EBD411D9
:20EB0000FFF7F6FA18BBA40004F4FE7404F130032B44D8789A78120442EA0062587842EA95
:20EB200000202C4494F83030184320F07040F8BD0120F8BD0120F8BD0120F8BD4FF0FF3099
:20EB4000F8BD4FF0FF30F8BD4FF0FF30F8BD4FF0FF30F8BDF8B505460E46E9808468012CC9
:20EB600034D003685A69A24232D91CB91A78032A08BF5C6A24B91A89B2422BD9586A17E022
:20EB80009F783F010EE028682146FFF771FF0446B0F1FF3F20D0012820D92B685B6983427C
:20EBA0001ED9F61BBE42EED228682146FFF754FFEC60B8B100EB161028612B6806F00F0660
:20EBC00003EB461330336B610020F8BD0220F8BD0220F8BD0220F8BD0120F8BD0220F8BDB8
:20EBE0000220F8BD0220F8BD2DE9F04105460C46164601297CD943698B427BD90378022B33
:20EC000042D0032B54D0012B76D101EB5107016A01EB5721FFF76CFA034600286DD107F107
:20EC20000108C7F3080714F0010409D0EB1993F83020F3B202F00F0242EA0313DBB200E0EA
:20EC4000F3B22F4487F8303001232B71296A284601EB5821FFF74CFA034600284DD1C8F311
:20EC6000080814B1C6F3071608E005EB080292F8302022F00F02C6F303261643A84488F863
:20EC8000306001222A7138E0016A01EB1421FFF72FFA034688BB640004F4FF742A1982F84B
:20ECA0003060C6F3072682F8316001222A7124E0016A01EBD411FFF71BFA0346E8B9A4003C
:20ECC00004F4FE7404F130022A44D17809062C4401F070410E4384F83060C6F307215170CC
:20ECE000C6F307419170360ED67001222A7104E0022302E0022300E002231846BDE8F08141
:20ED00002DE9F0410546884631B9C66886B14369B34298BF01260CE0FFF7AAFE012844D955
:20ED2000B0F1FF3F4CD06B69834249D8464600E001263446022701346B69A34202D8012EF1
:20ED400036D93C4628462146FFF792FE38B1B0F1FF3F30D0012830D0B442ECD12FE02846A6
:20ED600021466FF07042FFF73FFF034640B9B8F1000F05D0284641462246FFF735FF034648
:20ED80005BB9EC602B69B3F1FF3F0BD0013B2B616B7943F001036B7104E0012B14BF0124FB
:20EDA0004FF0FF342046BDE8F0810120BDE8F0810020BDE8F081BDE8F081BDE8F0810020AC
:20EDC000BDE8F0812DE9F84304460E46C5880135ABB2002B66D00369002B66D015F00F0705
:20EDE00057D101330361C16821B903681B89AB425ED94EE000688378013B13EA151348D112
:20EE0000FFF736FE8046012855D9B0F1FF3F55D020684369434535D8002E52D0E168FFF74F
:20EE20006FFF804600284FD0012850D0B0F1FF3F50D02068FFF72AF900284ED1206830303F
:20EE400000214FF40072FEF7DBFF266830464146FFF702FEF06200264FF001090BE083F865
:20EE600004902068FFF712F9002839D12368DA6A0132DA62013623689A78B242EFD8DA6A32
:20EE8000921BDA62C4F80C8020684146FFF7E4FD2061E580236803EB47133033636100205B
:20EEA000BDE8F8830420BDE8F8830420BDE8F8830420BDE8F8830220BDE8F8830120BDE85E
:20EEC000F8830420BDE8F8830720BDE8F8830220BDE8F8830120BDE8F8830120BDE8F88368
:20EEE0000120BDE8F88300BF2DE9F84F04460021FFF730FE002861D14FF6FF7323844FF02F
:20EF0000FF0A57469946D0464FF00B0B20682169FFF7EEF8064600284DD165692B78002BE5
:20EF200048D0EA7A02F03F01E52B04D012F0080F05D00F2903D0A4F82090474632E00F2923
:20EF40001DD1E06970B313F0400F06D095F80DA003F0BF03E28822841F46BB4209D16B7B0E
:20EF6000534508D12946FFF7CBFC30B1013FFFB218E0474616E0474614E0474612E027B9C7
:20EF80002846FFF747F8504515D0A169CB7A13F0010F04D128465A46FEF73CFF58B1A4F83A
:20EFA0002090474620460021FFF70CFF06460028ACD000E004263046BDE8F88FBDE8F88FC4
:20EFC00010B582B0044601910B785AB22F2A01D05C2A01D1013101910023A360019B1B7834
:20EFE0001F2B07D820460021FFF7B4FD03460022626123E0204601A9FFF742FB0346E8B95C
:20F000002046FFF771FFA369DA7A034640B1042814D102F00402D2B2002A08BF05230DE0F7
:20F0200012F0040F0AD16169CB7A13F0100F04D02068FEF70BFFA060DCE70523184602B059
:20F0400010BD00BF2DE9F04104460F460021FFF781FD0246C8B90025A84601262068216994
:20F06000FFF746F8024680B963691B78E52B00D01BB90135BD4201D107E045462046314672
:20F08000FFF7A0FE02460028E8D0042A14BF10460720BDE8F08100BF2DE9F04385B0054698
:20F0A0008769C66901A839460C22FEF79FFE9DF80F3013F0010F1BD00023FB72EB61012476
:20F0C0000BE0384601A932462346FEF747FF2846FFF70AFF804610B90134632CF1D9642CE7
:20F0E00063D0B8F1040F62D19DF80F30FB72EE619DF80F3013F0020F03D101260CE001335B
:20F1000000E0002336F81320002AF8D103F11906294AA2FB0636B60828463146FFF792FF0F
:20F12000044630BB013E24D0E9882846891BFFF711FD0446E8B9A869FEF76CFF81464FF07E
:20F140000108002728682969FEF7D2FF044680B9E8696969F2B24B46FEF7CAFE2A6882F8F3
:20F16000048028463946FFF72DFE044608B9013EE8D1C4B928682969FEF7BAFF044690B91A
:20F18000686900212022FEF73BFE6869A9690B22FEF72CFE6B69AA69D27A02F018021A7312
:20F1A0002B6801221A71204602E0072000E0404605B0BDE8F08300BF4FECC44E2DE9F04713
:20F1C000044689464FF0FF0A56460425D04600274BE02068FEF78CFF054600284AD1616941
:20F1E0000B78002B45D0CA7A02F03F02E52B31D02E2B31D022F02000082814BF00200120F4
:20F2000048452BD10F2A1BD113F0400F06D091F80DA003F0BF03E28822841E46B34209D1EA
:20F220004B7B534508D1E069FEF72AFE30B1013EF6B214E0464612E0464610E046460EE001
:20F2400026B90846FEF7E6FE504513D04FF6FF7323840FE0464602E0464600E04646204617
:20F260003946FFF7AFFD054620B921690029B0D100E004250DB1002323612846BDE8F0871D
:20F280002DE9F8430446C788018C4FF6FF73994208BF3946FFF75EFC054610BB00264FF054
:20F2A00020094FF0E50820682169FEF721FF0546A0B9606931464A46FEF7A2FD636983F883
:20F2C0000080236801221A71E388BB4206D220463146FFF777FD05460028E4D0042D08BFCF
:20F2E00002252846BDE8F8832DE9F04104460D46012926D943698B4225D90027B8461CE0B4
:20F3000020462946FFF7B4FB064608B301281CD0B0F1FF3F1BD0204629464246FFF764FCDA
:20F320000746A8B92369B3F1FF3F05D001332361637943F00103637135466369AB42DFD852
:20F3400006E0022704E0022702E0022700E001273846BDE8F08100BF10B584B00190009110
:20F36000144604A840F8041DFEF762FE002816DB0E4B53F820300BB100221A70019B0BB10C
:20F3800000221A70019B094A42F820304BB1012C09D101A869460022FEF722FF04E00B20A6
:20F3A00002E0002000E0002004B010BD1C0A00202DE9F043ADF50F7D0191154604460028AE
:20F3C00000F0A4800023036002F01F0885A801A902F01E02FEF704FF0646002840F09480E1
:20F3E00082AB8B9302AB8C9385A80199FFF7E8FD8A9F064610B9002F08BF062615F01C0FC4
:20F400004AD04EB1042E03D185A8FFF745FE064648F008088A9F0BE0FB7A13F0110F06D150
:20F4200005F00405EDB2002D18BF082600E00726002E40D118F0080F3DD0F9F7ABFCB873C3
:20F44000C0F30723FB73C0F307433B74000E78740025FD723D777D77BD77FD77859839463B
:20F46000FEF7F4FC814638462946FEF7FFFC859801220271B9F1000F1DD0C56A4946FFF7F6
:20F4800033FF0646B8B9859809F1FF33C3602946FEF72EFE06460EE06EB9FB7A13F0100F89
:20F4A00008D115F0020F06D003F00103002B18BF072600E0042646B918F0080F18BF48F02A
:20F4C0002008859BDB6AE3612762EEB984F806804FF0000884F80780859D28463946FEF7DB
:20F4E000B5FC2061FA7FBB7F1B0443EA02637A7F43EA02233A7F1343E360C4F80880C4F8D9
:20F5000018802560EB88A380304600E009200DF50F7DBDE8F08300BF2DE9F04F83B0044682
:20F520000F4690461E4600233360FEF73DFE002840F0A780E079002840F0A580A37913F0E2
:20F54000010F00F09F80A368E568ED1A454528BF454604F1240301938EE0A368C3F3080248
:20F56000002A72D1206890F802A00AF1FF3A5FFA8AFA1AEA532A11D10BB9206902E06169FF
:20F58000FFF776FA012802D80220E0717BE0B0F1FF3F02D10120E07175E06061D4F80080AE
:20F5A00040466169FFF758FA814610B90220E07169E0D1445FEA552B25D00AEB0B0298F802
:20F5C00002309A4288BFCAEB030B98F8010039464A465B46F9F758FB10B10120E07152E02A
:20F5E000A37913F0400F0BD0A369C9EB0300584506D207EB402001994FF40072FEF7F6FB03
:20F600004FEA4B2B2FE0A2694A451CD0A37913F0400F0DD098F8010001990123F9F750FBD1
:20F6200010B10120E0712EE0A37923F04003A3712368587801994A460123F9F725FB10B189
:20F640000120E0711FE0C4F81890A168C1F30801C1F5007BAB4528BFAB46214438462431DE
:20F660005A46FEF7C3FB5F44A3685B44A36033685B443360CBEB0505002D7FF46EAF00207D
:20F6800001E000E0072003B0BDE8F08F2DE9F04F83B004460F4615461E4600233360FEF71A
:20F6A00083FD002840F0C580E079002840F0C380A37913F0020F00F0BD80A3685A19934289
:20F6C00088BF002504F124030193A4E0A368C3F30802002A40F08480206890F802B00BF1A3
:20F6E000FF3B5FFA8BFB1BEA532B1DD133B9236943B90021FFF704FB034603E06169FFF70A
:20F70000FFFA0346002B00F08980012B02D10220E07190E0B3F1FF3F02D10120E0718AE010
:20F720006361226902B92361A37913F0400F0ED0236858780199A2690123F9F7C1FA10B15F
:20F740000120E07177E0A37923F04003A371D4F8008040466169FFF77FF9814610B902209E
:20F76000E07168E0D9445FEA552A25D00BEB0A0298F802309A4288BFCBEB030A98F80100DB
:20F7800039464A465346F9F79BFA10B10120E07151E0A369C9EB030151450AD2019807EB17
:20F7A00041214FF40072FEF721FBA37923F04003A3714FEA4A2A25E0A3694B450ED0A26865
:20F7C000E3689A420AD298F8010001994A460123F9F75AFA10B10120E0712CE0C4F8189060
:20F7E000A068C0F30800C0F5007AAA4528BFAA462044243039465246FEF7F8FAA37943F04C
:20F800004003A3715744A3685344A360336853443360CAEB0505002D7FF458AFA368E268D1
:20F82000934288BFE360A37943F02003A371002001E000E0072003B0BDE8F08F38B50446CD
:20F84000FEF7B2FC0346002845D1A27912F0200F41D012F0400F0DD0214651F8243B587814
:20F86000A2690123F9F72CFA002836D1A37923F04003A3712068E169FEF73AFC034650BB3D
:20F88000256AEB7A43F02003EB72237B2B77A3891B0A6B77A37BAB77E37BEB772846216956
:20F8A000FEF7E4FAF9F776FAA875C0F30723EB75C0F307432B76000E68760023AB74EB7490
:20F8C000A37923F02003A371236801221A712068FFF762F80346184638BD012038BD00BF40
:20F8E00010B50446FFF7AAFF034630B92046FEF75BFC034608B900222260184610BD00BFDE
:20F90000F8B504460D46FEF74FFC0746002840F0A580E079002840F0A180E368AB4206D2B1
:20F92000A27902F00202D2B2002A08BF1D46A2680023A360002D5CD02068867876026AB13C
:20F94000691EB1FBF6F1013AB2FBF6F3994205D373421A40A260AD1A616911E0216971B9C2
:20F96000FFF7CEF90146012802D10220E071F8BDB0F1FF3F02D10120E071F8BD2061616143
:20F9800019BB002538E0A27912F0020F05D02068FFF7B6F9014620B91AE02068FFF768F82E
:20F9A0000146B1F1FF3F02D10120E071F8BD012903D9226852698A4202D80220E071F8BD0D
:20F9C0006161A2683244A260AD1BB542DBD800E03546A2682A44A260C5F308025AB1206847
:20F9E000FFF73AF810B90220E071F8BD00EB552502E0002500E00025A368C3F3080313B3EB
:20FA0000A269AA421FD0A37913F0400F0ED0214651F8243B58780123F9F752F910B1012094
:20FA2000E071F8BDA37923F04003A371214651F8243B58782A460123F9F726F910B10120D6
:20FA4000E071F8BDA561A368E268934204D9E360A37943F02003A3713846F8BDF8BD00BF23
:20FA600030B5ADF5077D0191054600282FD085A801A90022FEF7B4FB044618BB859B2B6012
:20FA800082ABAB6102ABEB6128460199FFF798FA0446A0B9696949B1CB7A13F0100F04D0FA
:20FAA0008598FEF7D3F9A86000E005243CB9859BDB88AB8028460021FFF74CF80446042C71
:20FAC00008BF05240CB100232B60204600E009200DF5077D30BD00BFF0B5ADF5057D044617
:20FAE0000F46FEF761FB054628BB2FB920460021FFF730F805461EE081ABA36101ABE3613C
:20FB000020460021FFF75AFB0646042802D1002323612E4676B920463946FEF733FD20460E
:20FB20000021FFF74FF90546042804D100232361354600E0354628460DF5057DF0BD00BF3F
:20FB40002DE9F04798B003460F46604A16924FF48072179207A81946FFF782FF024600284D
:20FB600040F0B0800026DFF8A0A1DFF8A091DFF8A08107A810A9FFF7AFFF0246002840F03B
:20FB8000A1809DF84930002B00F09C805BB22E2BEFD0169D2B780BB90DF14905BDF844205B
:20FBA000C2F34313013B0B2B66D8DFE803F0060E161E262E363E464E565E454B93E803006A
:20FBC00003908DF81010042456E0424B93E8030003908DF8101004244EE03F4B93E80300EE
:20FBE00003908DF81010042446E03C4B93E8030003908DF8101004243EE0394B93E80300FA
:20FC000003908DF81010042436E0364B93E8030003908DF8101004242EE0334B93E8030005
:20FC200003908DF81010042426E0304B93E8030003908DF8101004241EE02D4B93E8030011
:20FC400003908DF81010042416E02A4B93E8030003908DF8101004240EE0274B93E803001D
:20FC600003908DF81010042406E0244B93E8030003908DF81010042403A82044514602F059
:20FC80001F0207F025FC2044BDF84420520A03AB1844494602F2BC7207F01AFC9DF848307D
:20FCA00013F0100F14BF164B164B1B88BB5301360095B8194146109A03AB07F009FC04461A
:20FCC000064456E7104618B0BDE8F08718080020849901088C990108949901089C9901085B
:20FCE000A4990108AC990108B4990108BC990108C4990108CC990108D4990108DC990108F4
:20FD0000E8990108EC990108E4990108289C0108F099010810B592B003460C461C4A10923C
:20FD20004FF480721192027822B901A81949FFF797FE03E001A81946FFF792FEE0B901A84D
:20FD40000AA9FFF7C9FED0B99DF83130D3B15BB22E2BF4D0109803780BB90DF13100214689
:20FD600007F0F4FB03460028E9D19DF8302012F0100F09D10A9B07E04FF0FF3304E04FF072
:20FD8000FF3301E04FF0FF33184612B010BD00BF1C090020288F01082DE9F04F83B002ABF9
:20FDA00043F8040D8A461446104619460022FEF717FA2568804600285FD12B696C69A21E1C
:20FDC000934202D8CAF8003057E02F78012F11D10224002628462146FEF74AFEB0F1FF3F55
:20FDE0003FD0012840D000B9013601346B699C42F0D33BE0296A00231A461E464FF4007BCE
:20FE000052B901F101092846FEF772F9804668BB05F1300349465A46022F09D193F801C075
:20FE2000187850EA0C2008BF01360233023A15E093F803C09878000440EA0C6093F801C024
:20FE400040EA0C2093F800C020F0704020F0FF0050EA0C0008BF01360433043A013CCFD19C
:20FE600004E04FF0010801E04FF002082E616B7943F001036B71CAF80060404603B0BDE8A6
:20FE8000F08F00BF30B5ADF5197D01908FA801A90122FEF7A5F9044600284BD183AB9593FB
:20FEA00003AB96938FA80199FFF78AF80446002840D1949931B1CB7A03F00103002B18BF52
:20FEC000072400E00624FCB9CB7A13F0100F1DD08F98FDF7BBFF0546D0B186A88FA9242297
:20FEE000FDF784FF889586A80221FEF733FE044678B986A80021FFF761F9002808BF0720C7
:20FF0000042818BF044604E0002502E0002500E002247CB98FA8FFF7B3F9044628B925B16F
:20FF20008F982946FFF7E0F904461CB98F98FEF733FD044620460DF5197D30BD2DE9F04F67
:20FF4000ADF50F7D0190F8F725FF054685A801A90122FEF745F90446002840F0A18082AB67
:20FF60008B9302AB8C9385A80199FFF729F8002808BF0820042840F0928085980021FEF701
:20FF8000BFFEB0F1000908BF0724B9F1010F08BF0224B9F1FF3F08BF01241CB98598FEF7A6
:20FFA00075F80446002C59D1859E30464946FEF753FD074606F1300A504600214FF40072DD
:20FFC000FDF71EFF504620210B22FDF719FF4FF02E0B86F830B0102386F83B3086F84650FA
:20FFE000C5F3072386F84730C5F3074386F848302B0E86F8493050464946FDF737FF06F1BC
:020000040801F1
:200000005008404651462022FDF7F0FE86F851B08799859B1A78032A03D15B6A8B4208BF9C
:2000200000214046FDF722FF859B9E784FF0010B12E0859807F10108C76280F804B0FEF729
:2000400025F8044650B9504600214FF40072FDF7D7FE013EF6B24746002EEAD11CB985A89C
:20006000FFF71AF8044624B185984946FFF73CF916E08A981023C3728575C5F30723C375EE
:20008000C5F3074303762D0E45764946FDF7EEFE859801230371FEF77FFC044600E00446E7
:2000A00020460DF50F7DBDE8F08F00BF2DE9F04F8DB009900C461546012988BF132000F2FB
:2000C000688309A8FDF7B4FF0028C0F23683BE4B53F82060002E00F03B8300233370BB4BCE
:2000E00013F8107003EB400393F801803846F8F7C7FD10F0010F40F02D8310F0040F40F0D4
:200100002B83B8F1000F34D0384606F1300100220123F8F7B9FD002840F0208396F82F220A
:2001200096F82E3243EA022212B2A94B9A4240F0178306EB081393F8E22103F5EF73002A04
:2001400000F01083D97A9A7A120442EA0162597A42EA01211A7A41EA020AD97B9A7B1204A5
:2001600042EA0162597B42EA01221B7B13430A9314E0384601210AAAF8F7C8FD002840F0F0
:20018000F3820A9B7F2B40F2F182002C0CBF4FF03F0A4FF0000ACAEB03030A936B1E2B42E0
:2001A00018BF00257DB94FF4FA600A9BB3FBF0F00023884900E0013331F813208242FAD843
:2001C000854A32F81350B5F5007F28BF6D0A002D08BF0125812D28BF80250A9AB2FBF5F3AF
:2001E00040F6F5794B458CBF4FF002094FF001094FF6F5718B4288BF4FF00309B9F1030F27
:2002000009D19B0003F207235B0A0193002104912023029312E0B9F1010F05D103EB43030D
:2002200001335B08033301E002335B0003F2FF135B0A0193202104910123029302995144C1
:2002400003918B46019B9B4404998B440BEB0503CAEB03039A42C0F08B82384603210BAAA9
:20026000F8F754FD20B90B9B13B1B3F5004F01D901230B930B9B0BEB0302013A5B4213409C
:20028000CBEB03030B93B9F1030F06D1029A1A44029203991944039102E0019A1A440192E8
:2002A0000A9B02995A1A0199521A0499521AB2FBF5F20592B9F1020F05D140F6F572059984
:2002C000914240F25782B9F1030F05D14FF6F5720599914240F25082B9F1030F0DD0B9F14A
:2002E000010F02D1B3F5803F0AD3B3F5803F2CBF4FF0060B4FF0040B04E04FF00C0B01E0CC
:200300004FF0010BB8F1000F10D006EB081888F8E2B1384606F1300100220123F8F7D0FC2F
:20032000002840F02B824FF0F80859E0002C55D106F13004204600214FF40072FDF760FD36
:20034000012386F8EF3186F8F031002286F8F12186F8F2B1FE2186F8F3110A990AEB010E21
:2003600043F6C160BEFBF0F00B904FEA900E4EF03F0E86F8F4E186F8F5013F2086F8F601F2
:2003800086F8F72186F8F82186F8F92186F8FA11C1F3072086F8FB01C1F3074086F8FC0144
:2003A000090E86F8FD11552186F82E12AA2186F82F1238462146F8F783FC002840F0E081D0
:2003C0004FF0F8080CE000BF1C0A00205C01002055AAFFFF58990108549A01084FF0F0084B
:2003E00006F1300B584600214FF40072FDF708FD5846D3490B22FDF7F9FC002386F83B3082
:20040000022386F83C3086F83D50029A86F83E20C2F3072386F83F30012386F84030B9F1C2
:20042000030F4FF0000386F8413018BF022386F842300A9BB3F5803F06D286F84330C3F302
:20044000072386F844300CE086F85030C3F3072286F85120C3F3074286F852201B0E86F832
:20046000533086F845803F2386F84830002386F84930FF2286F84A2086F84B3086F84CA0D8
:20048000CAF3072386F84D30CAF3074386F84E304FEA1A6386F84F30F8F77CFC0B90B9F118
:2004A000030F3CD186F87300C0F3072386F87430C0F3074386F87530000E86F87600019B6F
:2004C00086F854301946C3F3072386F85530C1F3074386F856300B0E86F85730022386F815
:2004E0005C30002386F85D3086F85E3086F85F30012286F8602086F86130062286F86220D1
:2005000086F86330802386F87030292386F8723006F177008B491322FDF768FC1FE086F851
:200520005700C0F3072386F85830C0F3074386F85930000E86F85A00019A86F84620C2F363
:20054000072386F84730802386F85430292386F8563006F15B007C491322FDF747FC55238C
:2005600086F82E32AA2386F82F323846594652460123F8F7A5FB002840F00481B9F1030FF0
:2005800006D1384659460AF106020123F8F798FB0023029368F0FF010691CAB20792089565
:2005A000039D62E0584600214FF40072FDF728FCB9F1030F13D0B9F1010F644A18BF6FF090
:2005C000FF0242EA08030B9386F83030FF2286F8312086F832201B0E86F833301CE0069B00
:2005E0000B93079986F83010FF2386F8313086F8323086F8333086F8343086F8353086F8FA
:20060000363086F8373086F8383086F8393086F83A300F2386F83B306C1C384659462A46AA
:200620000123F8F74DFB002840F0AE80584600214FF40072FDF7E4FB01230B9322460CE07C
:20064000541C384659460123F8F73AFB002840F09D800B9B01330B9322460B9B01998B4263
:20066000EED31546029A01320292029B002B99D00395089D0499B9F1030F08BF2946049169
:200680000124039A0D4602F10108384659462346F8F716FB00287BD14246013DF3D1B9F11B
:2006A000030F41D1522386F8303086F83130612386F83230412286F83320722186F8141215
:2006C00086F8151286F8162286F81732059A531E86F81832C3F3072386F81932531EC3F350
:2006E000074286F81A221B0E86F81B32022386F81C32002386F81D3286F81E3286F81F3285
:20070000552386F82E32AA2386F82F32384659460AF101020123F8F7D3FA384659460AF1C4
:2007200007020123F8F7CCFA384600210A46F8F7EDFA003018BF01202BE00B2029E000BFEC
:20074000109A01081C9A0108309A010800FFFF000C201EE003201CE00A201AE0012018E0D0
:200760000E2016E00E2014E0012012E0012010E00E200EE00E200CE00E200AE0012008E0B8
:20078000012006E0012004E0012002E0012000E001200DB0BDE8F08F7F2815D971B1FF2869
:2007A0009DBF8038094B33F810000020704731F81320824206D001339BB201E000230349F8
:2007C0007F2BF4D98033D8B2704700BF6C9A0108A0F161039BB2192B9CBF203880B27047BE
:2007E00070B592B001200146F6F794FF4FF4C0600121F6F7B5FFF023ADF8443000248DF8AF
:200800004740374811A9F6F71FFB364D2846F5F7CDFF354B0693354B0793089404260996D0
:200820000A9480230B934FF480730C934FF480630D9320230E934FF400530F931094284610
:2008400006A9F6F76FF828460121F6F713F9019401258DF808508DF809504FF4602303933A
:2008600004948DF81460224C20460DEB0601F5F793FD204607212A460323F5F71FFF204604
:20088000062102220323F5F719FF2046052103221346F5F713FF2046314632460323F5F774
:2008A0000DFF20462946F5F745FE20462946F5F717FE2046F5F764FE2046F5F77DFE0028A9
:2008C000FAD10B48F5F796FE094C2046F5F7AEFE0028FAD106480121F5F7C6FE12B070BD25
:2008E00000080140080002404C2401402C2500200024014010B5044672B6F6F7E3F9352089
:20090000F6F7F4F92046F6F72DFA042804D1F6F7E5F962B6002010BD4FF0FF3010BD00BFB8
:200920002DE9F04105460F46904672B6960812F0030F18BF0136F6F7C5F93520F6F7D6F956
:20094000002408E0284657F82410F6F739FA042809D104350134B442F4DBF6F7BFF962B684
:200960004046BDE8F0814FF0FF30BDE8F08100BF10B4002302E0C45CCC5401339342FAD3B9
:2009800018465DF8044B7047194B1B88FF2B17D9184B4FF000621A6002F5C0425A604FF409
:2009A00000621A8140225A810C221A7303225A733122DA81104A1A61A2F500625A61704762
:2009C0000C4B4FF000621A6002F5C0425A604FF480621A8180225A8118221A7303225A73FC
:2009E0006522DA81054A1A61A2F580625A617047E0F7FF1F3425002000F0010800F80108F8
:200A000010B582B004460F4B53F820000121F6F7A7FE0D4B33F81430ADF804300B4B2344BF
:200A20009B78012B0CBF282310238DF8073003238DF80630064B53F8240001A9F6F704FA3C
:200A400002B010BD6C9B0108AC9B0108D42800206001002008B50346064A02449278022A48
:200A600007D1054A52F82000044A32F81310F6F73FFB08BDD428002060010020AC9B010871
:200A800008B50346064A02449278022A07D1054A52F82000044A32F81310F6F759FB08BD52
:200AA000D428002060010020AC9B010808B502460D4B03449B78012B08D10C4B53F82000CB
:200AC0000B4B33F81210F6F75BFA08BD022B08D1064B53F82000064B33F81210F6F7ACFA79
:200AE00008BD002008BD00BFD428002060010020AC9B010870B582B00E461546052806D196
:200B00001048694601AAFFF747F9044609E0431EDBB2032B05D80C48694601AAFFF73CF9E8
:200B2000044664B9019B5A69023A9B7803FB02F1009A02FB03F34A0832605B082B602046EA
:200B400002B070BDCC9B0108D09B010808B5F8F747F9F8F73DFA02280BD060B90748084902
:200B60000022FEF7F9FB0122064B1A60064B187808BD002008BD002008BD00BF4C250020BC
:200B8000D09B0108301300201C03002008B5F8F785FD0F480F490022FEF7DEFBF8F714F877
:200BA00001280CBF012200220B4B1A60094800214FF40072FFF77AFAF8F706F8012801D1B3
:200BC000F8F718F80122044B1A60052008BD00BF4C250020CC9B01082C13002010B5F6F76F
:200BE0000FFC4FF48030F6F72BFCF6F737FE012830D11020F6F74EF80220F6F737F80020D6
:200C0000F6F7C4FC4FF48060F6F704FD4FF48060F6F7E0FC4FF480304FF48011F6F73EFC3C
:200C20000120F6F787FC39242046F6F7E5FD0028FAD00220F6F78EFCF6F7A0FC0828FBD181
:200C40004FF410300121F6F7B1FD44F23D000121F6F786FD10BD00BF0160436082600023BA
:200C60000361C3600120704738B504460568C2680369D21A43689A420DDAC268013B02EA2F
:200C80000300A26802FB005006F0D5FAE3680133E360012038BD002038BD00BFF8B5044692
:200CA0000F46D0F800E0C1680369C91A436899420BDBC1680269891A1D488B42CCBF00213E
:200CC000012106F061FB0020F8BDC6680169761A9E1BC168581E0840811999422CBFC0EBF8
:200CE00003053546761BAA42B8BF1546521BB242B8BF1646A26802FB00E0394602FB05F294
:200D000006F099FAE3682B44E36020686268013A1340A26802FB030002FB057102FB06F2FB
:200D200006F089FAE3683344E360A819F8BD00BFD49B010838B504460568C26803699A4272
:200D40000ED003694268013A13408268084602FB035106F070FA236901332361012038BDCE
:200D6000002038BDF8B504460F460168C0682369984231D0E6682369F61A23696568681E51
:200D800003409819A8422CBFC3EB05053546761BAA42B8BF1546521BB242B8BF1646A268CA
:200DA000384602FB031102FB05F206F044FA23692B44236121686268013A1340A26802FB15
:200DC000057002FB031102FB06F206F034FA236933442361A819F8BD0020F8BD08B503489A
:200DE0004FF48051F6F7B4F908BD00BF000C014008B503484FF48051F6F77AF908BD00BF74
:200E0000000C014070B506460C4D022428462146F6F772FE0028F9D008483146F6F738FE88
:200E2000064D012428462146F6F766FE0028F9D00248F6F747FEC0B270BD00BF00380040D1
:200E400008B5FFF7DFFF08BD08B5FF20FFF7DAFF08BD00BF30B58DB005460C464FF6FF7397
:200E6000ADF800302D4B01930023079308930593049209934FF440520A920B932848F5F704
:200E800095FC2848F5F792FC9DB102940024039480230693224801A9F5F744FD0DEB0403BC
:200EA00002931023039306941E4801A9F5F73AFD11E000AB0293002303930693184801A97A
:200EC000F5F730FD02941023039380230693154801A9F5F727FD12480121F5F7CBFD1148BE
:200EE0000121F5F7C7FD104803210122F6F79AFD4FF400542046F5F703FE0028FAD00848D1
:200F00000021F5F7B7FD07480021F5F7B3FD064803210022F6F786FD0DB030BD0C380040D2
:200F200044000240580002400038004008B503460A4601201946FFF78DFF08BD08B50346F6
:200F40000A4600201946FFF785FF08BD70B586B04FF40053ADF8143003238DF8163018237D
:200F60008DF817302B4D284605A9F5F76DFF4FF40043ADF81430284605A9F5F765FF4FF49B
:200F80008043ADF8143004238DF81730284605A9F5F75AFF4FF48053ADF8143010238DF89A
:200FA0001730284605A9F5F74FFF0023ADF800304FF48272ADF80220ADF804300222ADF8FC
:200FC00006200124ADF808404FF40072ADF80A20ADF80C30ADF80E300723ADF810300E4E26
:200FE00030466946F6F75CFC30462146F6F7EEFC28462146F6F7ACF82046F7F7DDFD2846D1
:201000002146F6F775F820462146F6F783FB06B070BD00BF000C01400038004010B586B075
:20102000FFF7E6FE14481549FBF7FCFD14481549FBF70AFE14481549FBF720FE144B01ACA7
:20104000186859689A68DB680FC4012001A9FBF79BFFB0F1FF3F02D10E4806F021FA0F2494
:2010600020460DF11701FBF78FFF9DF81730002BF6D006B010BD00BFDD0D0108F10D01086B
:20108000490E0108410E01082D0F01083D0F0108F09B0108009C010808B50128044B03BFCE
:2010A00018891B69C0181869FFF762FC08BD00BF3425002070B50E4615460128074B03BF50
:2010C0001C891B69E4181C692046FFF713FC204631462A46FFF724FC70BD00BF3425002033
:2010E00008B54FF080400121F6F76EFF40B34FF080400121F6F70CFF4FF080400121F6F79E
:20110000D1FF104B1A88013292B21A801A8892B240F2E6339A420BD90B4B1A780132D2B261
:201120001A70F9F72BFAFAF7C3FE0022054B1A80054B1B78DBB23A2B02D90022024B1A70A9
:2011400008BD00BF240A0020260A002010B584B001200146F6F72AFB1C238DF800300124E1
:201160008DF801408DF802408DF803406846F5F78BF84FF47A73ADF808300023ADF80430F4
:20118000ADF80A30ADF806304FF0804001A9F6F7E7FC4FF0804047212246F6F75FFE4FF0C4
:2011A00080402146F6F78AFD4FF0804021462246F6F7E8FD04B010BDF8B505460F461646CA
:2011C0001C4640F227710022F7F720F9384631462246FFF763FD0446284640F22771012262
:2011E000F7F714F92046F8BD08B5044806F0C0F980B20028014808BF002008BD90270020FB
:2012000008B50021044B1980044B198004484FF4967206F019F808BD280A00202C1200200D
:201220009027002010B5184840F22551F7F706FA48B3154840F22551F7F77CFA134B1C88B6
:20124000134B1B889C4203D9E21AB2F5957F04DC9C4207D2621C934204D10B484021F7F7BB
:201260004BF910BD0848F7F773F90A4B1855074B1B88B3F5957F03D80133044A138010BD83
:201280000022024B1A8010BD00380140280A00202C1200209027002070B506460648314642
:2012A000F7F72AF9044D802428462146F7F772F90028F9D0304670BD003801400B480C4945
:2012C00003880A889342FBD0B3F5957F07D801339BB2064A1380013B064AD05C70470022C1
:2012E000024B1A80034B93F82B0170472C120020280A002090270020F8B50D46174638B17E
:201300000CE0FFF7DBFF287001360134013501E000263446BC42F4DB3046F8BD05F048FF22
:20132000092303604FF0FF30F8BD00BF70B51546012809D0022812D015E04E1C0878FFF7D9
:20134000ABFF0134314600E00024AC42F5DB11E04E1C0878FFF7A0FF0134314600E0002455
:20136000AC42F5DB06E005F023FF092303604FF0FF3070BD284670BD30B585B00023364D2D
:2013800008E00A6855F82340A24202D10092012303E00133092BF4D9002313B94FF4E13378
:2013A00000930B79082B02D0092B04D008E00023ADF8043009E04FF48053ADF8043004E069
:2013C0000023ADF8043008230B718B79012B02D0022B04D008E00023ADF8063009E04FF455
:2013E0000053ADF8063004E00023ADF8063001238B714B79012B07D013B1022B09D00DE03F
:201400000023ADF808300DE04FF4C063ADF8083008E04FF48063ADF8083003E00023ADF806
:2014200008304B714B7913B1012B04D008E00023ADF80C3007E04FF44073ADF80C3002E0A4
:201440000023ADF80C300C23ADF80A306946F6F785FE05B030BD00BFA001002030B585B01F
:2014600001F0DCFA05464FF49053ADF8043018238DF8073003238DF80630164C204601A911
:20148000F5F7E2FC04238DF807304FF44063ADF80430204601A9F5F7D7FC0023ADF8083011
:2014A000ADF80A304FF40072ADF80C20ADF80E3004F54054204605F13301FFF75DFF20460F
:2014C00002A9F6F721FF20460121F6F76BFF05B030BD00BF00080140F8B505460F46164622
:2014E0001C4640F225510022F6F790FF384631462246FFF737FC0446284640F2255101223B
:20150000F6F784FF2046F8BD70B582B005460C46164640F22771F7F791F888B130460DF102
:201520000701FFF707FC28B128469DF80710F6F7E3FF05E0284640F227710022F6F766FF57
:20154000284640F22551F7F779F870B1E2682369D21A63689A4208DA2846F6F7F9FF02A9AC
:2015600001F8010D2046FFF77FFB02B070BD00BF08B503480349044AFFF7C6FF08BD00BF0F
:2015800000440040BC2800207C270020F0B585B001F044FA07462A482A4901224FF480637C
:2015A000FFF75AFB2848294901224FF48063FFF753FB26238DF8003000248DF801408DF804
:2015C000024001258DF803506846F4F75DFE0623ADF8043018238DF8073003238DF80630FD
:2015E0001B4E304601A9F5F72FFC04238DF807300923ADF80430304601A9F5F725FCADF891
:201600000840ADF80A404FF40073ADF80C30ADF80E40104C204607F13B01FFF7ADFE20460C
:2016200002A9F6F771FE204640F225512A46F6F7EDFE20462946F6F7B5FE05B0F0BD00BFB7
:20164000BC2800202C0E00207C2700202C0A0020000801400044004008B502460B460248A6
:201660000249FFF739FF08BD00440040BC28002008B502460B4602480249FFF79DFD08BD64
:20168000004400407C270020024BD8681B69C01A704700BF7C27002008B504480449012266
:2016A0004FF48063FFF7D8FA08BD00BF7C2700202C0A002008B503460A46034948691946ED
:2016C000FFF756F908BD00BF3425002070B506460D46054B5C692046FFF70CF920463146B1
:2016E0002A46FFF71DF970BD342500202DE9F0413A4C20464FF4DB71FFF7DCFF2378AA2BC5
:2017000002D16378012B3ED0344BAA221A7001225A7002219970D970197159719971D97102
:20172000197259729A72DA721A735A739A73DA731A745A7400232948194603E0C218917436
:201740000133DBB20F2BF9D90024DFF890801927234E11E004EB840505EB8505454422353D
:20176000284600213A4605F06FFD28463146224605F0AEFE0134E4B20F2CEBD917484FF49F
:20178000DB71FFF7A3FF17480121F5F711FD0024124D0AE02B199B78013BDBB2FD2B02D85B
:2017A0002046FFF72DF90134E4B20F2CF2D900240A4D0FE02B199B78022B09D12B199B7CB3
:2017C0001BB92046FFF75CF902E02046FFF742F90134E4B20F2CEDD9BDE8F081D42800200D
:2017E0001C9C010800043000024B33F8100080B2704700BF2C2500202DE9F04FC9B04290B3
:20180000439101F00BF90023ADF81C31ADF81831ADF814314FF0040A08264FF007094FF009
:2018200009084FF0050C4FF0060E012502274FF0030B7FE01A46991D00EBC101D1F803105A
:20184000B1F5165F39D00ED8B1F5966F44D003D8B1F5167F45D04AE0B1F5166F37D0B1F592
:20186000965F2FD043E0B1F5614F17D006D8B1F5964F1DD0B1F5164F15D038E0B1F5E13FF0
:2018800007D0B1F5613F32D148A9194401F8048C31E048A9194401F8046C2CE048A919442F
:2018A00001F8049C27E048A9194401F804EC22E048A9194401F804CC1DE048A9194401F8F4
:2018C00004AC18E048A9194401F804BC13E048A9194401F8047C0EE048A9194401F8045C0A
:2018E00009E0002448A9194401F8044C03E048A9114401F8046C00EBC20191F83710092902
:2019000004D148A9114401F8085C04E0002448A9114401F8084C00EBC20191F83910022909
:2019200048A90A440EBF02F80C5C002102F80C1C0133DBB2012B7FF67DAF827FC37F90F89D
:2019400020B000F1050A90F8029090F8038090F804C090F821E090F82270279790F823102A
:20196000289190F82470299790F825102A9190F826702B9790F84D102C9190F827702D97F5
:2019800090F828102E9190F829702F9790F82A10309190F82B70319790F82C10329190F864
:2019A0002D70339790F82E10349190F82F70359790F83010369190F83170379790F83210F2
:2019C000389190F84F70399790F850103A9190F851703B9790F852103C919DF81C713D97AC
:2019E0009DF818113E9190F838703F979DF8146190F83A509DF81D419DF8191190F840704E
:201A000040979DF81571419790F84200CDF800B0CDF804A0CDF80890CDF80C80CDF810C011
:201A2000CDF814E0279F0697289F0797299F08972A9F09972B9F0A972C9F0B972D9F0C970E
:201A40002E9F0D972F9F0E97309F0F97319F1097329F1197339F1297349F1397359F1497C6
:201A6000369F1597379F1697389F1797399F18973A9F19973B9F1A973C9F1B973D9F1C9726
:201A80003E9F1D973F9F1E971F9620952194229140992391419F249725904298034905F058
:201AA00017FD439F388049B0BDE8F08F2C9C01082DE9F04FBDB0834688460020FEF7F6FF27
:201AC00082460120FEF7F2FF81460220FEF7EEFF2E900320FEF7EAFF2F900420FEF7E6FFF0
:201AE00030900520FEF7E2FF31900620FEF7DEFF32900720FEF7DAFF33900820FEF7D6FF06
:201B000034900920FEF7D2FF35900A20FEF7CEFF36900B20FEF7CAFF37900C20FEF7C6FF05
:201B200038900D20FEF7C2FF39900E20FEF7BEFF3A900F20FEF7BAFF3B90354B9A7821929A
:201B4000DA7822921A7923925A7924929A792592DA7926921A7A27925A7A28929A7A29922F
:201B6000DA7A2A921A7B2B925A7B2C929A7B2D92DF7B1E7C5D7C0020F6F7D2FF0446012086
:201B8000F6F7CEFF2E9B00932F9A0192309B0293319A0392329B0493339A0592349B0693E3
:201BA000359A0792369B0893379A0992389B0A93399A0B923A9B0C933B9A0D92219B0E93C0
:201BC000229A0F92239B1093249A1192259B1293269A1392279B1493289A1592299B1693DD
:201BE0002A9A17922B9B18932C9A19922D9B1A931B971C961D951E941F9058460549524626
:201C00004B4605F065FCA8F800003DB0BDE8F08FD428002064A001082DE9F04FBDB0834678
:201C200088460020FEF742FF82460120FEF73EFF81460220FEF73AFF2F900320FEF736FF42
:201C400030900420FEF732FF31900520FEF72EFF32900620FEF72AFF33900720FEF726FF68
:201C600034900820FEF722FF35900920FEF71EFF36900A20FEF71AFF37900B20FEF716FF68
:201C800038900C20FEF712FF39900D20FEF70EFF3A900E20FEF70AFF3B900F20FEF706FF68
:201CA0003D4A91780E91D3780F93177910975179119193791293D7791397117A149192F800
:201CC00009C092F80AE0D37A1793167B557B947BD17B177C1C97537C2F9F0097309F019733
:201CE000319F0297329F0397339F0497349F0597359F0697369F0797379F0897389F099764
:201D0000399F0A973A9F0B973B9F0C970D90CDF854C0CDF858E0189619951A941B911D9379
:201D200002F122031E9302F13B031F9302F15403209302F16D03219302F18603229302F1BF
:201D40009F03239302F1B803249302F1D103259302F1EA03269302F20313279302F58E73F2
:201D6000289302F23513299302F5A7732A9302F267132B9302F5C0732C9302F299132D936D
:201D80005846064952464B4605F0A2FBA8F800003DB0BDE8F08F00BFD4280020F8A301086B
:201DA0002DE9F04184B007460C460020FFF71CFD06460120FFF718FD05460220FFF714FDEE
:201DC00080460320FFF710FDCDF80080019064230293C82303933846044932462B4605F0FB
:201DE00077FB208004B0BDE8F08100BF00A9010838B505460C46FFF7F7F902462846034924
:201E000005F066FB2080FFF7FBF938BDB4A90108F0B583B0054600F001FE044690F827304C
:201E20008DF8043090F828308DF8053090F829308DF8063090F82A308DF8073028464C4912
:201E4000F8F746F8064680B1671D38460021192205F0FAF9304605F08BFBC2B2192A38466C
:201E6000314628BF182205F0E6F928464149F8F72FF850B1312105F05CFB18B1012384F8E0
:201E80004D3002E0002384F84D3094F84D309BBB28463949F8F71CF898B104F12701F7F721
:201EA000CFFF94F827308DF8043094F828308DF8053094F829308DF8063094F82A308DF80F
:201EC000073028462D49F8F703F818B104F12B01F7F7B6FF28462A49F7F7FAFF18B104F1EA
:201EE0002F01F7F7ADFF28462649F7F7F1FF18B104F14F01F7F7A4FF28462349F7F7E8FF0F
:201F000040B10A21F7F78AFFC0B2204B53F82030C4F8333028461E49F7F7DAFF20B10A21FF
:201F2000F7F77CFF84F8370028461A49F7F7D0FF20B10A21F7F772FF84F83800284616491B
:201F4000F7F7C6FF20B10A21F7F768FF84F8390028461249F7F7BCFF20B10A21F7F75EFF0F
:201F600084F83A0000F0FCFD01A803B0F0BD00BFDCA90108E8A90108F0A90108F4A901088A
:201F8000F8A90108FCA9010800AA0108C80100200CAA010814AA01081CAA010824AA010821
:201FA00038B505461F49F7F793FF20B10A21F7F735FFC4B200E0002428461B49F7F788FF22
:201FC00020B10A21F7F72AFFC5B200E00025A4F15A00C0B2012807D8012D02D1F6F790FD8E
:201FE0001EE0F6F77DFD1BE02246104B23449B78022B15D1012D07D10C4B1A44002393744C
:202000002046FEF73DFD06E0084B1A44012393742046FEF71FFD05484FF4DB71FFF756FBCF
:20202000284638BD30AA010834AA0108D428002070B505461649F7F74BFF28B30A21F7F75C
:20204000EDFEC4B228461349F7F742FF0546A8B104EB840606EB86060F4B1E443046002139
:20206000192205F0F1F8284605F082FAC2B2192A3046294628BF182205F0DDF807484FF44F
:20208000DB71FFF723FB00E00024204670BD00BF30AA010834AA0108F6280020D428002066
:2020A00038B504461B49F7F713FF20B10A21F7F7B5FEC5B200E0002520461749F7F708FFB1
:2020C00020B10A21F7F7AAFEC4B200E00024022C07D1124B2B4402229A702846FEF790FC05
:2020E00010E0012C07D10D4B2B4401229A702846FEF786FC06E02846FEF7C2FC074B1D4458
:202100000023AB7005484FF4DB71FFF7DFFA204638BD00BF30AA010838AA0108D4280020D2
:2021200038B50949F7F7D4FE0546002430B938BD285DFFF7B1F80134A4B2FFE7284605F05B
:2021400017FA8442F4D338BD3CAA010808B50949F7F7BEFE68B10A21F7F760FEC0B2012819
:2021600007D10548FF23037043704FF4DB71FFF7ADFA08BD44AA0108D4280020F0B585B014
:2021800007460C4616461D4600F048FC90F84D10012907D130460B49BD2205F04CF8BC2305
:2021A0002B800CE023786078A178E278009001910292304604493A4605F08AF9288005B0D4
:2021C000F0BD00BF50AA010810AB0108F0B583B007460E4614461046FEF768FC0346094AAE
:2021E0001119897804EB840505EB85052A4422320091019238460449224605F069F93080A2
:2022000003B0F0BDD428002094AC010870B506460D4614461046FFF7E7FA034630460349A3
:20222000224605F055F9288070BD00BF04AD01082DE9F04F8FB006460D4600F0EFFB04464E
:20224000827FC37F90F820B000F1050A90F8029090F8038090F804C090F821E090F82270CF
:2022600090F8230094F824100C9194F825100D9194F82640CDF800B0CDF804A0CDF80890CA
:20228000CDF80C80CDF810C0CDF814E0069707900C9908910D9909910A943046034905F098
:2022A00017F928800FB0BDE8F08F00BF44AD01082DE9F04F97B006460D4600F0AFFB0446AB
:2022C00090F8272090F8283090F829B090F82AA090F82B9090F82C8090F82DC090F82E10EA
:2022E000119190F82F70129790F83010139190F83170149790F83210159190F84FE090F87D
:202300005070109790F8510094F8521094F84D40CDF800B0CDF804A0CDF80890CDF80C80EA
:20232000CDF810C0119F0597129F0697139F0797149F0897159F0997CDF828E0109F0B975A
:202340000C900D910E943046034905F0C1F8288017B0BDE8F08F00BFE0AD0108F0B589B06B
:2023600007460E46154600F059FB0023ADF81C30ADF81830ADF81430022D28BF1D462C4648
:20238000AB1D00EBC303D3F80330B3F5165F3ED00ED8B3F5966F4CD003D8B3F5167F53D0B1
:2023A0004DE0B3F5166F3ED0B3F5965F35D046E0B3F5614F19D006D8B3F5964F21D0B3F5A8
:2023C000164F18D03BE0B3F5E13F08D0B3F5613F35D1092108AB2B4403F8041C34E0082103
:2023E00008AB2B4403F8041C2EE0072108AB2B4403F8041C28E0062108AB2B4403F8041CC1
:2024000022E0052108AB2B4403F8041C1CE008AB1D44042305F8043C16E0032108AB2B44A7
:2024200003F8041C10E0022108AB2B4403F8041C0AE0012108AB2B4403F8041C04E00821DB
:2024400008AB234403F8041C00EBC40393F83730092B0CBF0121002108AB234403F8081C28
:2024600000EBC40393F83930022B0CBF0121002108AB234403F80C1C08AD254415F8043CD3
:2024800015F808ECA11D00EBC102107A15F80C1C927ACDF800E001900291039238460349DC
:2024A000224605F015F8308009B0F0BD88AE01082DE9F04784B00646884691460023009335
:2024C00001930293ADF80C303D4905F03FF828B940464946FFF7ACFE01206DE03046394944
:2024E00005F034F828B940464946FFF7E1FE012062E03046344905F029F830B94046494686
:202500000022FFF72BFF012056E030462F4905F01DF8F8B9404649460122FFF71FFF01200C
:202520004AE0009501950295ADF80C5068463946224604F0CDFF3046694605F007F830B957
:20254000404649462246FFF741FEE4B208E00134E4B202E0002425461D4F0F2CE1D9FF248B
:2025600014F0800F1AD1FF251FE0009701970297ADF80C70684651462A4604F0A9FF30460A
:20258000694604F0E3FF30B9404649462A46FFF73DFEEDB209E00135EDB203E000252F463D
:2025A000DFF830A0032DE0D9FF2514F0800F1DBF68B2C043C00F012004B0BDE8F08700BF5C
:2025C00030AF010840AF010850AF010864AF010878AF010888AF010838B5044600F01EFA48
:2025E000054620460E49F7F773FC044690B1053528460021192204F027FE204604F0B8FFBD
:20260000C2B2192A2846214628BF182204F013FE012400E000240CB100F0A2FA204638BD3B
:2026200098AF010870B5064600F0F8F9054630462049F7F74DFC60B1312104F07AFF18B1FE
:20264000012485F84D4005E0002385F84D30012400E0002495F84D303BBB30461649F7F75D
:2026600037FC20B105F12701F7F7EAFB012430461249F7F72DFC20B105F12B01F7F7E0FB9C
:20268000012430460E49F7F723FC20B105F12F01F7F7D6FB012430460A49F7F719FC20B1C3
:2026A00005F14F01F7F7CCFB01240CB100F058FA204670BDE8A90108A0AF0108F4A90108D0
:2026C000F8A90108FCA90108F8B504460F4600F0A5F9064620463249F7F7FAFB78B10A2164
:2026E000F7F79CFBC0B20A2828BF08202D4B53F8202006EBC703C3F83320012500E00025AB
:2027000020462949F7F7E4FB78B10A21F7F786FBC0B2A0F1080303F0FF03022B28BF082012
:2027200006EBC70383F83700012520461F49F7F7CFFB58B10A21F7F771FBC0B2032828BF6E
:20274000002006EBC70383F83800012520461849F7F7BEFB70B10A21F7F760FBC0B2431EEF
:2027600003F0FF03022B28BF012006EBC70383F83900012520460F49F7F7AAFB58B10A2115
:20278000F7F74CFBC0B2042828BF002006EBC70686F83A0001250DB100F0E2F92846F8BD17
:2027A000A4AF0108C80100200CAA010814AA01081CAA0108ACAF010838B505461449F7F798
:2027C00087FBF8B10A21F7F729FBC4B20F2C1CD828461049F7F77CFB38B10A21F7F71EFBA5
:2027E000C0B2032828BF022000E000200A4D2A1990702046FEF704F928464FF4DB71FEF74F
:2028000065FF00E00024E0B200E0FF2040B238BD30AA010834AA0108D428002038B50546BA
:202820001849F7F755FB30B30A21F7F7F7FAC4B20F2C23D828461449F7F74AFB38B10A214E
:20284000F7F7ECFAC0B2022828BF012000E000200E4A22449074012803D12046FEF7FAF8F4
:2028600003E010B92046FEF70BF908484FF4DB71FEF72CFF00E00024E0B200E0FF2040B2C7
:2028800038BD00BF30AA010834AA0108D428002070B505461849F7F71BFB38B30A21F7F7C5
:2028A000BDFAC4B20F2C24D828461449F7F710FB0546A8B104EB840606EB8606104B1E4499
:2028C00030460021192204F0BFFC284604F050FEC2B2192A3046294628BF182204F0ABFC6F
:2028E00008484FF4DB71FEF7F1FE00E00024E0B200E0FF2040B270BD30AA010834AA010897
:20290000F6280020D4280020F8B504460F4616461D46394904F01AFE50B93846FFF75CFEED
:2029200002463046354904F0D3FD28800120F8BD2046334904F00AFE50B93846FFF772FE4E
:20294000024630462D4904F0C3FD28800120F8BD20462C4904F0FAFD58B938460021FFF7A5
:20296000B3FE02463046254904F0B2FD28800120F8BD2046244904F0E9FD58B938460121FB
:20298000FFF7A2FE024630461C4904F0A1FD28800120F8BD20461D4904F0D8FD50B9384652
:2029A000FFF70AFFC2B23046144904F091FD28800120F8BD2046164904F0C8FD50B93846CC
:2029C000FFF72CFFC2B230460C4904F081FD28800120F8BD20460F4904F0B8FD50B93846B9
:2029E000FFF756FFC2B23046044904F071FD28800120F8BD0020F8BDB4AF0108289C010867
:202A0000C4AF0108D4AF0108E8AF0108FCAF01080CB0010820B001080020704700487047E6
:202A200030120020F8B53D4C852323800127A7700223E37000252571DFF8E4C066460FCE3D
:202A4000C4F80500C4F80910C4F80D20C4F8113003CEC4F81500C4F8191033786377A777D0
:202A6000E77784F82070C02184F82710A82284F828200B2384F82930642084F82A0084F821
:202A80002B1084F82C2084F82D3084F82E70FF2384F82F3084F8303084F8313084F832508C
:202AA00084F83350636B03F07F4343F4E1736363082384F8373084F8385084F8397084F890
:202AC0003A5084F83B50E26B02F07F4242F4E172E26384F83F3084F8405084F8417084F8F7
:202AE00042500CF11C0203CAC4F84300C4F847101288A4F84B2084F84D5084F84E5084F8FA
:202B00004F3084F8503084F8513084F8523004F153002946322204F097FBF8BD3012002097
:202B200034B0010810B50D4C012021468522FEF7B3FA2288013A92B24FF6FD739A4206D920
:202B4000FFF770FF012021468522FEF7B3FA034B01229A77DA7783F8202010BD3012002082
:202B600008B5012002498522FEF7A4FA08BD00BF3012002008B504F05EFB08BD08B504F08C
:202B80005AFB08BD38B50446154D05F1210021460622FFF7F3FF05F12700A11D0422FFF7FD
:202BA000EDFF05F12B0004F10E010422FFF7E6FF05F12F0004F10A010422FFF7DFFF05F1EE
:202BC0004F0004F112010422FFF7D8FFA37D012B07BF00222B460122014B83F84D2038BDBA
:202BE0003012002038B50546144C04F121010622FFF7C0FFA81D04F127010422FFF7BAFF30
:202C000005F10E0004F12B010422FFF7B3FF05F10A0004F12F010422FFF7ACFF05F11200CD
:202C200004F14F010422FFF7A5FF94F84D3013B10223AB7538BD0123AB7538BD30120020ED
:202C400030B58BB0012004A9FAF7C8FA9DF810109DF811209DF812309DF813509DF81440A0
:202C60009DF815000095019402901A4804F08CFB9DF816109DF817209DF818309DF81900FF
:202C80000090154804F080FB9DF81E109DF81F209DF820309DF821000090104804F074FB5B
:202CA0009DF81A109DF81B209DF81C309DF81D0000900B4804F068FB9DF822109DF8232019
:202CC0009DF824309DF825000090064804F05CFB0BB030BD5CB0010884B001089CB00108D9
:202CE000B4B00108CCB0010810B586B0FFF796FE0446684604F121010622FFF73BFF0DF1F8
:202D0000060004F127010422FFF734FF0DF10E0004F12B010422FFF72DFF0DF10A0004F1CF
:202D20002F010422FFF726FF0DF1120004F14F010422FFF71FFF94F84D301BB102238DF814
:202D4000163002E001238DF8163000206946FAF745FA06B010BD00BF10B50446FFF75EFEBA
:202D60002368C0F82130A388A0F8253010BD00BFBFF34F8F044AD16801F4E061034B0B4332
:202D8000D360BFF34F8FFEE700ED00E00400FA0510B4002304E0CC5C4440CC5401339BB2A3
:202DA0009342F8D35DF8044B704700BF10B4002304E0CC5C4440CC5401339BB29342F8D3A1
:202DC0005DF8044B704700BF2DE9F041CEB0054688461446FFF722FE074628460B210DF5A2
:202DE0009B72F9F76BFEB4F80560BDF83621964257D10DF10A030093284627A9062203AB9E
:202E0000F9F764FD607810F0800F06D000F07F0027A9BDF83621FFF7C9FF27A807F1210132
:202E2000062204F0F9F900283BD16FF0740363710023A371552323713B4653F8210F0490D3
:202E40009B88ADF814300DF116003946852204F0F2F9607810F0800F05D000F07F0004A9F5
:202E60008B22FFF795FF20682990A288A379ADF8A8208DF8AA300DF1AB0004A98B2204F0D1
:202E8000DAF9A37823B94046FF21042204F0DCF9B8F804300093284629A992224346F9F7EF
:202EA00071FC4EB0BDE8F0812DE9F043A5B0054688461446FFF7B2FD074628460B210DF1F6
:202EC0008E02F9F7FBFDB4F80560BDF88E20964240F0FC80E378A13B042B00F2F780DFE8EC
:202EE00003F0AE03207B9A000DF13E030093284602A9072210ABF9F7E9FC607810F0800FEE
:202F000006D000F07F0002A9BDF88E20FFF74EFF02A8B91C032204F07FF9002800F08F80E4
:202F2000D4E00DF13E030093284602A90C2210ABF9F7CCFC607810F0800F06D000F07F00A5
:202F400002A9BDF88E20FFF731FF9DF8082097F821309A4200F2BA809DF8091097F8222019
:202F6000914200F2B3809DF80A0097F82310884200F2AC809DF80B6097F82400864200F2A3
:202F8000A5809DF80CC097F82560B44500F29E809DF80D9097F826C0E14500F297809DF823
:202FA0000E904B4500F292809DF80F309A4200F28D809DF81030994200F288809DF81130B0
:202FC000984200F283809DF812309E427ED89DF813309C4533D979E00DF13E0300932846B7
:202FE00002A9212210ABF9F771FC607810F0800F06D000F07F0002A9BDF88E20FFF7D6FE47
:203000007E1D02A804F0B4FA024602A8314604F003F9A0B15AE00DF13E030093284602A9FA
:20302000342210ABF9F752FC607810F0800F06D000F07F0002A9BDF88E20FFF7B7FE0C23AD
:2030400063710023A371552323713B4633F8022F9B78ADF844208DF846303B4633F81E2F6C
:203060009B78ADF847208DF8493057F8213FCDF84A30BB88ADF84E30607810F0800F05D0A3
:2030800000F07F0011A90C22FFF782FE20681490A288A379ADF854208DF8563011AB07CB3F
:2030A000CDF85700CDF85B10CDF85F20A37823B94046FF21042204F0C7F8B8F80430009393
:2030C000284614A913224346F9F75CFB25B0BDE8F08300BF2DE9F04190B00546884614461A
:2030E000FFF79CFC074628460B210DF13E02F9F7E5FCB4F80560BDF83E2096425BD10DF126
:203100000A030093284606A9172203ABF9F7DEFB607810F0800F06D000F07F0006A9BDF832
:203120003E20FFF743FE06A807F12101062204F073F800283FD10DF11F0007F1430104F026
:2031400005FA002837D1062363710023A3715523237157F8210F0490BB88ADF814306078E9
:2031600010F0800F05D000F07F0004A90622FFF70FFE20680C90A288A379ADF834208DF8BC
:20318000363010AB53F8300DCDF837009B88ADF83B30A37823B94046FF21042204F054F854
:2031A000B8F80430009328460CA90D224346F9F7E9FAFFF7DDFD10B0BDE8F0812DE9F041FD
:2031C000F4B0054688461446FFF728FC074628460B210DF5E772F9F771FCB4F80560BDF859
:2031E000CE2196426ED10DF10E030093284628A99C2204ABF9F76AFB607810F0800F06D0E9
:2032000000F07F0028A9BDF8CE21FFF7CFFD28A807F12101062203F0FFFF002852D10DF1BC
:20322000A70007F1430104F091F900284AD138460DF1B7018522FFF7A1FC0123BB77FB77B4
:2032400087F82030FFF78CFC6FF0740363710023A371552323713B4653F8210F05909B8880
:20326000ADF818300DF11A003946852203F0E3FF607810F0800F05D000F07F0005A98B2248
:20328000FFF786FD20684F90A288A379ADF840218DF842310DF2431005A98B2203F0CBFFA0
:2032A000A37823B94046FF21042203F0CDFFB8F80430009328464FA992224346F9F762FA26
:2032C000FFF756FD74B0BDE8F08100BF2DE9F043B7B0054688461446FFF7A0FB8146FFF73B
:2032E0009DFB074628460B210DF1C202F9F7E6FBB4F80560BDF8C220964240F0B4800DF1DA
:203300000A03009328461CA94F2203ABF9F7DEFAE378D12B40F0A780607810F0800F06D008
:2033200000F07F001CA9BDF8C220FFF73FFD1CA807F12101062203F06FFF002840F09380BE
:203340000DF1770007F1430104F000F9002840F08A800DF1C40E4E4656F8210F7168B26898
:20336000F368AEE80F00338AAEF80030FFF7DAFB0DF1C40EBEE80F00C9F821007160B260A5
:20338000F360BEF800303382FFF7EAFB20680490A288A379ADF814208DF81630D8F800305E
:2033A000CDF81730B8F80430ADF81B30DDF88730CDF81D30BDF88B30ADF821300DF18D039B
:2033C0000DF123020DF1BD01D3F800C0D3F804E09E68D868C2F800C0C2F804E09660D06050
:2033E000103310328B42EFD11B881380002004A94522FDF75FFE062363710023A371552354
:20340000237157F8210F1690BB88ADF85C30607810F0800F05D000F07F0016A90622FFF7F7
:20342000B7FC20681890A288A379ADF864208DF8663036AB53F8800DCDF867009B88ADF872
:203440006B30A37823B94046FF21042203F0FCFEB8F804300093284618A90D224346F9F7D3
:2034600091F9FFF785FC37B0BDE8F0832DE9F04190B0054688461446FFF7D0FA07462846D7
:203480000B210DF13E02F9F719FBB4F80560BDF83E2096425FD10DF10A030093284606A9D7
:2034A000172203ABF9F712FA607810F0800F06D000F07F0006A9BDF83E20FFF777FC06A8A4
:2034C00007F12101062203F0A7FE002843D10DF11F0007F1430104F039F800283BD1FFF72E
:2034E000A1FAFFF73DFB062363710023A3715523237157F8210F0490BB88ADF814306078AC
:2035000010F0800F05D000F07F0004A90622FFF73FFC20680C90A288A379ADF834208DF8EA
:20352000363010AB53F8300DCDF837009B88ADF83B30A37823B94046FF21042203F084FE7B
:20354000B8F80430009328460CA90D224346F9F719F9FFF70DFC10B0BDE8F08110B588B045
:2035600004460A210DF11F02F9F7A8FA9DF81F30002B51D0222B56D12046092107AAF9F750
:203580009DFABDF81C30062B4DD906AB0093204603A9072205ABF9F799F99DF80C30A52BEA
:2035A00041D19DF81030AA2B3DD19DF80F3003F0F003C02B18D004D8A02B09D0B02B0DD07C
:2035C00031E0E02B1CD0F02B20D0D02B2BD111E0204605A903AAFFF767FC24E0204605A9BE
:2035E00003AAFFF7F1FB1EE0204605A903AAFFF7E5FD18E0204605A903AAFFF767FE12E09F
:20360000204605A903AAFFF765FD0CE0204605A903AAFFF72BFF06E02046022141F6961276
:203620000023F8F719FE08B010BD00BF2DE9F04784B004460F4603F09BFF073808282DD8FC
:203640006846214603F08CFF6846194903F0ECFF044600263546DFF85C80DFF854A0B14689
:203660000EE0204603F0A0FDFF2819D807B1785506440135EDB24846514603F0D5FF044674
:203680002CB14046214600F071F80028E9D0042D08D1002E14BF0020FF2004E0FF2002E0F7
:2036A000FF2000E0FF2040B204B0BDE8F08700BF2C8F0108D17101082DE9F04387B0044692
:2036C0000F4603F055FF11282BD101A8214603F047FF01A8164903F0A7FF04460025DFF8E9
:2036E00054802E46DFF848900FE020463146102204F07AF8FF2816D807B178550135EDB200
:203700003046494603F090FF04462CB14046214600F02CF80028E8D0062D0CBF0020FF20DD
:2037200002E0FF2000E0FF2040B207B0BDE8F083E4B00108E571010810B40028BABF4042E5
:2037400001220022002308E0013292B290FBF1F008B9D0B205E001339BB21CB2FE2CF3DDC5
:20376000FF2040B25DF8044B704700BF38B50C46054658B169B10B7823B90DE040B2A84744
:2037800068B1013420780028F8D138BD4FF0FF3038BD4FF0FF3038BD4FF0FF3038BD4FF0F5
:2037A000FF3038BDF0B484460068B0B10646771C96F900500B465C1C93F90020AA4207D1B7
:2037C00015B10023337000E00027CCF8007005E02346002AEFD13E46E9E70020F0BC704713
:2037E0002DE9F84F0646DFF86491DFF86481DFF858A12AE09AF800200232121B4E4B1340BF
:2038000003D5013B63F0010301335FB24B4B53F827509DB1284603F0ABFEB8F80030181A36
:20382000431EA8F80030284603F0EEFC0022434B43F82720013C89F8004006E040484149E4
:20384000E02203F0A1FD30BFFDE799F80040012CD0D824B1B8F900303344F92BCADC3A4BE0
:203860001C78A04606F1010A504603F0C5FC334B43F82400354F1D4632E008F10203C9EBFA
:2038800003092D4B19EA030B05D50BF1FF3B6BF0010B0BF1010B4FFA8BFB55F82B90B9F193
:2038A000000F16D0484603F063FE294B1A88101A421E1A80484603F0A7FC002345F82B3018
:2038C0003B78013B3B70504603F096FC45F8280006E020481B49ED2203F056FD30BFFDE7F4
:2038E00097F80090B9F1000F03D055F82830002BC3D0124B53F8240030B917481149F0223A
:2039000003F042FD30BFFDE7144903F029FE012C03D100220C4B1A7002E001340A4B1C702F
:2039200009F10109094B83F80090094B1A88324401321A80BDE8F88F0100008020130020EB
:20394000E4B10108B0B101081D130020281300201E13002008B201082CB20108B8120020CF
:2039600070B59AB0044619903D2103F0E2FD18B10322B44BDA7510E020463F2103F0D9FDFA
:2039800018B10122AF4BDA7507E020462D2103F0D0FD10B10222AB4BDA7519A8AA49FFF7C3
:2039A00001FF064678B9FD2096E15DB20C682C44647804F00304022C06BF2B46203B5BB260
:2039C00002F8013B01E00246A0491378002BECD1304603F0CDFD0A280BD896F90030412BB9
:2039E00007D196F90130542B03D196F902302B2B3FD096F90030412B36D196F90130542B45
:203A000032D1B378002B2FD18E4BDB7D5AB2012A21D18F4B1B78012B05D88E480821FDF78A
:203A200027FE022058E18C4B1B78012B84BF023BDBB28A4A52F82340204603F099FD0246AB
:203A400068468749234603F043FDC1B26846FDF70FFE022040E1002B40F03D8181480521DF
:203A6000FDF706FE022037E17F48314603F078FD03E07D48F11C03F073FD19A87B49FFF7DB
:203A800091FE0446002800F0188103F071FD232816D96C48002380F8443080F82030C3753E
:203AA000037680F8A43080F8903080F87C3080F8683020306E49012203F00AFDFB200BE1AA
:203AC0006C48214603F04CFD19A86849FFF76AFE0446002800F0F38003F04AFD232816D976
:203AE0005848002380F8443080F82030C375037680F8A43080F8903080F87C3080F86830E6
:203B000020305B49022203F0E3FCFB20E4E05A48214603F025FD19A85449FFF743FE0446DF
:203B2000002800F0CE8003F023FD132816D94548002380F8443080F82030C375037680F855
:203B4000A43080F8903080F87C3080F8683020304749032203F0BCFCFB20BDE047482146C7
:203B600003F0FEFC19A84149FFF71CFE0446002800F0A98003F0FCFC132816D931480023C1
:203B800080F8443080F82030C375037680F8A43080F8903080F87C3080F86830203034493B
:203BA000042203F095FCFB2096E03548214603F0D7FC19A82D49FFF7F5FD0446002800F09F
:203BC000848003F0D5FC132816D91E48002380F8443080F82030C375037680F8A43080F841
:203BE000903080F87C3080F8683020302049052203F06EFCFB206FE02248214603F0B0FCBA
:203C000019A81A49FFF7CEFD044600285FD003F0AFFC132838D90B48002380F8443080F85A
:203C20002030C375037680F8A43080F8903080F87C3080F8683020300D49062203F048FCC6
:203C4000FB2049E0902E002050B20108200200202813002054B201081D13002020130020E8
:203C600060B2010870B20108A82E002064910108289C0108B02E0020D42E0020F82E0020D7
:203C80000C2F0020202F00201548214603F068FC199B1B78EBB1134B002283F8442083F882
:203CA0002020DA751A7683F8A42083F8902083F87C2083F86820FB200EE000200CE000202C
:203CC0000AE0002008E0002006E0002004E0002002E0002000E0FC2040B21AB070BD00BF22
:203CE000342F0020902E002008B510480021642203F0AAFA00230E48194604E05AB240F810
:203D000022100133DBB25AB2012AF7DD094BFF2283F8B820012283F8CE2083F8D020064A96
:203D2000C3F8C020054AC3F8C42008BDB812002020130020902E00208C2A0020642F002091
:203D4000F8B50E469C4B93F920E093F94470003718BF012793F9685093F97C1093F99020E1
:203D600093F9A440BEF1000F0CBF3B467B1C002D18BF0133002918BF0133002A18BF013391
:203D8000002C0CBF1C465C1C5B228C4B1A70051E3DDB15B953225A701EE0032D07D1884856
:203DA00088494FF4BF7203F0EFFA30BFFDE7042D03D15722814B5A700EE0052D03D1522293
:203DC0007E4B5A7008E080487E4940F281122B4603F0DAFA30BFFDE7B6F1FF3F0FD0774886
:203DE0002C23837003307949324603F071FB30460A21FFF7A1FC033000F0FF03B9E0002C97
:203E000000F0B6802C226D4B9A700323B1E06B4B46225A702C229A70B6F1FF3F0CD0D81CC0
:203E20006A49324603F054FB30460A21FFF784FC033000F0FF0300E003235A1CD2B22C208D
:203E40005E49C8541E351C2D00F28C80DFE805F0808A8A8A8A766C62584F458A8A8A8A8ABF
:203E60008A8A8A8A3F39332D27211B150F00531CDBB23020514988547BE0531CDBB2312051
:203E80004E49885475E0531CDBB232204B4988546FE0531CDBB233204849885469E0531CD9
:203EA000DBB234204549885463E0531CDBB23520424988545DE0531CDBB236203F498854C9
:203EC00057E0531CDBB237203C49885451E0531CDBB23820394988544BE0511CC9B2374882
:203EE000312383544B1CDBB23022425441E0511CC9B23248312585544B1CDBB2455438E064
:203F0000511CC9B22D48312383544B1CDBB2322242542EE0511CC9B22848312383544B1C43
:203F2000DBB23322425424E0511CC9B22348312383544B1CDBB2342242541AE0511CC9B2C5
:203F40001E48312383544B1CDBB23522425410E0511CC9B21948322383544B1CDBB2302244
:203F6000425406E0531CDBB230201449885400E00223114A92F8202072B35E1CF6B22C2182
:203F80000E4AD154124803F0F3FA0246C5B2232D07D910480B494FF4D47203F0F5F930BF76
:203FA000FDE7064830440A49D2B203F044F97319DBB2013CE4B215E0902E0020B8120020AB
:203FC0009CB20108E8B00108D0B20108289C0108B02E002004B3010824B15A1C2C20704983
:203FE000C854D3B26F4A92F84420F2B15E1CF6B22C216B4AD1546C4803F0BAFA0246C5B273
:20400000232D07D969486A4940F2A91203F0BCF930BFFDE7624830446349D2B203F00BF95F
:204020007319DBB2013CE4B205E024B15A1C2C205B49C854D3B25B4A92F86820F2B15E1CFF
:20404000F6B22C21564AD1545A4803F091FA0246C5B2132D07D9554855494FF4D57203F0EF
:2040600093F930BFFDE74E4830445249D2B203F0E2F87319DBB2013CE4B205E024B15A1CCF
:204080002C204749C854D3B2464A92F87C20F2B15E1CF6B22C21424AD154474803F068FA46
:2040A0000246C5B2132D07D94048414940F2AB1203F06AF930BFFDE7394830443E49D2B2F7
:2040C00003F0B9F87319DBB2013CE4B205E024B15A1C2C203249C854D3B2324A92F8902002
:2040E000F2B15E1CF6B22C212D4AD154334803F03FFA0246C5B2132D07D92C482C494FF460
:20410000D67203F041F930BFFDE7254830442B49D2B203F090F87319DBB2013CE4B205E032
:2041200024B15A1C2C201E49C854D3B21D4A92F8A420E2B15D1CEDB22C21194AD154204843
:2041400003F016FA0246C4B2132C07D91748184940F2AD1203F018F930BFFDE71048284433
:204160001749D2B203F067F82B19DBB205E024B15A1C2C200A49C854D3B25A1CD2B2084C7A
:204180005D21E1540023A354204603F0F1F901462046FDF76DFA0B480221FDF769FAF8BD85
:2041A000B8120020902E0020D42E002004B30108E8B00108F82E00200C2F0020202F0020A4
:2041C000342F00207C92010810B5844BDB7DB3B9824B002283F8442083F82020DA751A7685
:2041E00083F8A42083F8902083F87C2083F868206FF003004FF0FF31FFF7A2FD10BD5AB2FC
:20420000012A16D1754B002283F8442083F82020DA751A7683F8A42083F8902083F87C20B0
:2042200083F868206FF003004FF0FF31FFF788FD10BD5AB2022A16D1684B002283F844208F
:2042400083F82020DA751A7683F8A42083F8902083F87C2083F868206FF003004FF0FF316F
:20426000FFF76EFD10BD5AB2032A40F0AE805B4B93F82030002B45D059485A49FFF776FA0E
:20428000D8B15648002380F8443080F82030C375037680F8A43080F8903080F87C3080F84F
:2042A000683020305049012203F012F96FF004004FF0FF31FFF744FD10BD4A4802F074FF8F
:2042C000C4B263B2102B01DC002B1CDC4348002380F8443080F82030C375037680F8A430B9
:2042E00080F8903080F87C3080F8683020303E49012203F0EDF86FF005004FF0FF31FFF7B7
:204300001FFD10BDFF24354B93F84430002B46D033483649FFF72AFAD8B13048002380F821
:20432000443080F82030C375037680F8A43080F8903080F87C3080F8683020302A490222F1
:2043400003F0C6F86FF004004FF0FF31FFF7F8FC10BD264802F028FFC1B24BB2012B02DC22
:2043600011F0800F1CD01D48002380F8443080F82030C375037680F8A43080F8903080F8D8
:204380007C3080F8683020301749022203F0A0F86FF005004FF0FF31FFF7D2FC10BDFF217E
:2043A0000E4B002283F8442083F82020DA751A7683F8A42083F8902083F87C2083F8682085
:2043C00060B249B202F04AFD10BD0948094940F259325BB202F0D8FF30BFFDE7902E0020E3
:2043E000D1710108B02E0020289C0108D42E002030B30108E0B3010810B5844BDB7DB3B9A5
:20440000824B002283F8442083F82020DA751A7683F8A42083F8902083F87C2083F86820B0
:204420006FF003004FF0FF31FFF78AFC10BD5AB2012A16D1754B002283F8442083F82020C8
:20444000DA751A7683F8A42083F8902083F87C2083F868206FF003004FF0FF31FFF770FCC6
:2044600010BD5AB2022A16D1684B002283F8442083F82020DA751A7683F8A42083F8902098
:2044800083F87C2083F868206FF003004FF0FF31FFF756FC10BD5AB2032A40F0AD805B4BE0
:2044A00093F82030002B45D059485A49FFF75EF9D8B15648002380F8443080F82030C3751A
:2044C000037680F8A43080F8903080F87C3080F8683020305049012202F0FAFF6FF0040051
:2044E0004FF0FF31FFF72CFC10BD4A4802F05CFEC4B263B2102B01DC002B1CDC4348002310
:2045000080F8443080F82030C375037680F8A43080F8903080F87C3080F8683020303E49A7
:20452000012202F0D5FF6FF005004FF0FF31FFF707FC10BDFF24354B93F84430002B45D017
:2045400033483649FFF712F9D8B13048002380F8443080F82030C375037680F8A43080F813
:20456000903080F87C3080F8683020302A49022202F0AEFF6FF004004FF0FF31FFF7E0FB1E
:2045800010BD264802F010FEC1B24BB2022B01DC002B1CDC1D48002380F8443080F8203007
:2045A000C375037680F8A43080F8903080F87C3080F8683020301849022202F089FF6FF0E4
:2045C00005004FF0FF31FFF7BBFB10BDFF210F4B002283F8442083F82020DA751A7683F85E
:2045E000A42083F8902083F87C2083F8682060B249B202F00FFC10BD09480A494FF4517231
:204600005BB202F0C1FE30BFFDE700BF902E0020D1710108B02E0020289C0108D42E002034
:2046200030B30108D4B3010808B5154BDB7D83B900204FF0FF31FFF783FBBFF34F8F114A5F
:20464000D16801F4E061104B0B43D360BFF34F8FFEE70B4B002283F8442083F82020DA7539
:204660001A7683F8A42083F8902083F87C2083F868206FF003004FF0FF31FFF761FB08BD3E
:20468000902E002000ED00E00400FA0508B5164BDB7D93B9144B002283F8442083F820208F
:2046A000DA751A7683F8A42083F8902083F87C2083F8682002F09EFB08BD0B4B002283F854
:2046C000442083F82020DA751A7683F8A42083F8902083F87C2083F868206FF003004FF0B7
:2046E000FF31FFF72DFB08BD902E002010B5FEF795F90446C24BDB7D13B90122C04BDA7589
:20470000BF4BDB7D5AB2012A60D1BD4B93F82030002B45D0BB48BC49FFF728F8D8B1B84805
:20472000002380F8443080F82030C375037680F8A43080F8903080F87C3080F868302030E9
:20474000B249012202F0C4FE6FF004004FF0FF31FFF7F6FA10BDAC4802F026FDC1B24BB289
:20476000052B01DC002B1CDCA548002380F8443080F82030C375037680F8A43080F8903010
:2047800080F87C3080F868302030A049012202F09FFE6FF005004FF0FF31FFF7D1FA10BD99
:2047A000FF21974B002283F8442083F82020DA751A7683F8A42083F8902083F87C2083F860
:2047C0006820934849B202F077FA10BD5AB2022A40F0B2828A4B93F82030002B00F08282E0
:2047E00088488949FEF7C2FFD8B18548002380F8443080F82030C375037680F8A43080F8BF
:20480000903080F87C3080F8683020307F49012202F05EFE6FF004004FF0FF31FFF790FAC9
:2048200010BD794802F0C0FCC0B243B2052B01DC002B1BDC7248002380F8443080F8203015
:20484000C375037680F8A43080F8903080F87C3080F8683020306D49012202F039FE6FF03E
:2048600005004FF0FF31FFF76BFA10BD43B2012B64D164486749FEF779FFD8B16048002329
:2048800080F8443080F82030C375037680F8A43080F8903080F87C3080F8683020305B4907
:2048A000022202F015FE6FF004004FF0FF31FFF747FA10BD574802F077FC0023564908E04B
:2048C00051F82320824203D1C4F83B00012303E001330A2BF4D90023D3B9494880F8443054
:2048E00080F82030C375037680F8A43080F8903080F87C3080F8683020304449022202F094
:20490000E7FD6FF004004FF0FF31FFF719FA10BD3B4B002283F8442083F82020DA751A76EA
:2049200083F8A42083F8902083F87C2083F86820374804F13B0102F047FA10BD43B2022B21
:204940006CD130483349FEF711FFD8B12C48002380F8443080F82030C375037680F8A43050
:2049600080F8903080F87C3080F8683020302749022202F0ADFD6FF004004FF0FF31FFF783
:20498000DFF910BD234802F00FFCC3B25AB2092A01DC072A1BDC1A48002380F8443080F868
:2049A0002030C375037680F8A43080F8903080F87C3080F8683020301449022202F088FDF6
:2049C0006FF005004FF0FF31FFF7BAF910BD84F83F000B4B002283F8442083F82020DA7572
:2049E0001A7683F8A42083F8902083F87C2083F86820074804F13B0102F0E6F910BD00BFC6
:204A0000902E0020D1710108B02E0020289C010800440040D42E0020A001002043B2032B18
:204A200040F08180BD48BE49FEF7A0FED8B1BD48002380F8443080F82030C375037680F818
:204A4000A43080F8903080F87C3080F868302030B549022202F03CFD6FF004004FF0FF31A7
:204A6000FFF76EF910BDAF4B93F84530ABB9AD4B93F844305AB2AD4909680A44527802F03A
:204A80000302022A5BB208BF203BDBB25AB24E2A1FD04F2A1DD0452A1BD0A248002380F871
:204AA000443080F82030C375037680F8A43080F8903080F87C3080F8683020309A490222FA
:204AC00002F006FD6FF004004FF0FF31FFF738F910BD5AB24E2A03D1002384F840300CE0C8
:204AE0005AB24F2A03D1012384F8403005E05BB2452B04BF022384F840308A4B002283F8A5
:204B0000442083F82020DA751A7683F8A42083F8902083F87C2083F86820854804F13B0115
:204B200002F052F910BD43B2042B5DD181487C49FEF71CFED8B17B48002380F8443080F8A9
:204B40002030C375037680F8A43080F8903080F87C3080F8683020307349022202F0B8FCC6
:204B60006FF004004FF0FF31FFF7EAF810BD6C4802F01AFBC3B25AB2022A01DC002A1BDC58
:204B80006848002380F8443080F82030C375037680F8A43080F8903080F87C3080F8683025
:204BA00020306149022202F093FC6FF005004FF0FF31FFF7C5F810BD84F84100594B002280
:204BC00083F8442083F82020DA751A7683F8A42083F8902083F87C2083F86820544804F147
:204BE0003B0102F0F1F810BD40B205285ED151484B49FEF7BBFDD8B14A48002380F844307F
:204C000080F82030C375037680F8A43080F8903080F87C3080F8683020304349022202F071
:204C200057FC6FF004004FF0FF31FFF789F810BD3B4802F0B9FAC3B25AB2032A02DC13F054
:204C4000800F1BD03748002380F8443080F82030C375037680F8A43080F8903080F87C302B
:204C600080F8683020303049022202F031FC6FF005004FF0FF31FFF763F810BD84F8420069
:204C8000284B002283F8442083F82020DA751A7683F8A42083F8902083F87C2083F8682082
:204CA000234804F13B0102F08FF810BD1D48002380F8443080F82030C375037680F8A430D9
:204CC00080F8903080F87C3080F8683020301649022202F0FDFB6FF007004FF0FF31FFF7E0
:204CE0002FF810BD0F48002380F8443080F82030C375037680F8A43080F8903080F87C3039
:204D000080F8683020300849012202F0E1FB6FF004004FF0FF31FFF713F810BDBD7101081A
:204D2000D42E0020902E0020289C01082002002000440040D17101085AB2032A40F0DC81CF
:204D4000C34B93F82030002B4ED0C248C249FEF70DFDD8B1BE48002380F8443080F82030A7
:204D6000C375037680F8A43080F8903080F87C3080F868302030B949012202F0A9FB6FF060
:204D800004004FF0FF31FEF7DBFF10BDB24802F00BFA0023B24908E051F82320824203D1E9
:204DA000C4F83B00012303E001330A2BF4D90023D3B9A74880F8443080F82030C3750376BC
